:020000040800F2
:10000000000005201D240008CD200008D320000892
:10001000D9200008DF200008E520000800000000CB
:1000200000000000000000000000000071F2000865
:10003000EB2000080000000081F40008E9F400084B
:100040006D2400086D2400086D2400086D2400084C
:100050006D2400086D2400086D2400086D2400083C
:100060006D2400086D2400086D2400086D2400082C
:100070006D2400086D2400086D2400086D2400081C
:100080006D2400086D2400086D2400086D2400080C
:100090006D2400086D2400086D2400086D240008FC
:1000A0006D2400086D2400086D2400086D240008EC
:1000B0006D240008F92000086D2400086D24000854
:1000C0006D2400086D2400086D2400086D240008CC
:1000D0006D2400086D2400086D2400086D240008BC
:1000E0006D2400086D2400086D2400086D240008AC
:1000F0006D2400086D2400086D2400086D2400089C
:100100006D2400086D2400086D2400086D2400088B
:100110006D2400086D2400080D2100086D240008DE
:100120006D2400086D2400086D2400086D2400086B
:100130006D2400086D2400086D2400086D2400085B
:100140006D2400086D2400086D240008212100089A
:100150006D2400086D2400086D2400086D2400083B
:10016000352100086D2400086D2400086D24000866
:100170006D2400086D2400086D24000800000000B4
:100180006D2400086D2400086D2400086D2400080B
:100190006D2400086D2400086D2400086D240008FB
:1001A000492100086D2400085D2100086D24000825
:1001B0006D2400086D2400086D2400086D240008DB
:0801C0006D2400086D24000805
:1001D00010B5054C237833B9044B13B10448AFF381
:1001E00000800123237010BDE013002000000000F8
:1001F000F4C2080808B5034B1BB103490348AFF329
:10020000008008BD00000000E4130020F4C20808CC
:1002100001F0FF01102A2BDB10F0070F08D010F8B7
:10022000013B013A8B422DD010F0070F42B3F6D1BB
:10023000F0B441EA012141EA014122F007047FF0D4
:1002400000070023F0E80256083C85EA010586EA2B
:10025000010685FA47F5A3FA87F586FA47F6A5FA67
:1002600087F68EB9EED1F0BC01F0FF0102F0070273
:1002700032B110F8013B013A83EA010313B1F8D11E
:100280000020704701387047002D06BF35460338FF
:10029000073815F0010F07D1013015F4807F02BF38
:1002A000013015F4C03F0130F0BC0138704700BF89
:1002B00010F8012B11F8013B012A28BF9A42F7D010
:1002C000D01A7047034613F8012B002AFBD1181AE5
:1002D0000138704781F0004102E000BF83F0004325
:1002E00030B54FEA41044FEA430594EA050F08BFD1
:1002F00090EA020F1FBF54EA000C55EA020C7FEA95
:10030000645C7FEA655C00F0E2804FEA5454D4EB11
:100310005555B8BF6D420CDD2C4480EA020281EADB
:10032000030382EA000083EA010180EA020281EA13
:100330000303362D88BF30BD11F0004F4FEA013165
:100340004FF4801C4CEA113102D0404261EB410174
:1003500013F0004F4FEA03334CEA133302D05242FA
:1003600063EB430394EA050F00F0A780A4F10104B6
:10037000D5F1200E0DDB02FA0EFC22FA05F28018F0
:1003800041F1000103FA0EF2801843FA05F35941D6
:100390000EE0A5F120050EF1200E012A03FA0EFC55
:1003A00028BF4CF0020C43FA05F3C01851EBE3717F
:1003B00001F0004507D54FF0000EDCF1000C7EEB9C
:1003C00000006EEB0101B1F5801F1BD3B1F5001FDA
:1003D0000CD349085FEA30004FEA3C0C04F10104F9
:1003E0004FEA445212F5800F80F09A80BCF1004F22
:1003F00008BF5FEA500C50F1000041EB045141EAA4
:10040000050130BD5FEA4C0C404141EB0101013C6C
:1004100028BFB1F5801FE9D291F0000F04BF01465B
:100420000020B1FA81F308BF2033A3F10B03B3F12D
:1004300020020CDA0C3208DD02F1140CC2F10C02BD
:1004400001FA0CF021FA02F10CE002F11402D8BF1B
:10045000C2F1200C01FA02F120FA0CFCDCBF41EAE7
:100460000C019040E41AA2BF01EB0451294330BDB6
:100470006FEA04041F3C1CDA0C340EDC04F1140493
:10048000C4F1200220FA04F001FA02F340EA03006A
:1004900021FA04F345EA030130BDC4F10C04C4F1B0
:1004A000200220FA02F001FA04F340EA0300294690
:1004B00030BD21FA04F0294630BD94F0000F83F4DA
:1004C000801306BF81F480110134013D4EE77FEABD
:1004D000645C18BF7FEA655C29D094EA050F08BF09
:1004E00090EA020F05D054EA000C04BF19461046EA
:1004F00030BD91EA030F1EBF0021002030BD5FEA2E
:10050000545C05D14000494128BF41F0004130BD55
:1005100014F580043CBF01F5801130BD01F00045A9
:1005200045F0FE4141F470014FF0000030BD7FEA1C
:10053000645C1ABF194610467FEA655C1CBF0B4617
:10054000024650EA013406BF52EA033591EA030F2E
:1005500041F4002130BD00BF90F0000F04BF002126
:10056000704730B54FF4806404F132044FF0000559
:100570004FF0000150E700BF90F0000F04BF0021D2
:10058000704730B54FF4806404F1320410F0004538
:1005900048BF40424FF000013EE700BF42004FEA33
:1005A000E2014FEA31014FEA02701FBF12F07F43B0
:1005B00093F07F4F81F06051704732F07F4208BF67
:1005C000704793F07F4F04BF41F40021704730B56E
:1005D0004FF4607401F0004521F000411CE700BFBA
:1005E00050EA010208BF704730B54FF000050AE03D
:1005F00050EA010208BF704730B511F0004502D53E
:10060000404261EB41014FF4806404F132045FEA3F
:10061000915C3FF4D8AE4FF003025FEADC0C18BFE8
:1006200003325FEADC0C18BF033202EBDC02C2F1DA
:10063000200300FA03FC20FA02F001FA03FE40EA6C
:100640000E0021FA02F11444BDE600BF70B54FF070
:10065000FF0C4CF4E06C1CEA11541DBF1CEA13554E
:1006600094EA0C0F95EA0C0F00F0DEF82C4481EAB6
:10067000030621EA4C5123EA4C5350EA013518BFD6
:1006800052EA033541F4801143F4801338D0A0FBC3
:1006900002CE4FF00005E1FB02E506F00042E0FB70
:1006A00003E54FF00006E1FB03569CF0000F18BF76
:1006B0004EF0010EA4F1FF04B6F5007F64F540741E
:1006C00004D25FEA4E0E6D4146EB060642EAC621B1
:1006D00041EA55514FEAC52040EA5E504FEACE2E1E
:1006E000B4F1FD0C88BFBCF5E06F1ED8BEF1004F21
:1006F00008BF5FEA500E50F1000041EB045170BD9D
:1007000006F0004646EA010140EA020081EA0301E0
:10071000B4EB5C04C2BFD4EB0C0541EA045170BDDC
:1007200041F480114FF0000E013C00F3AB8014F156
:10073000360FDEBF002001F0004170BDC4F100049F
:10074000203C35DA0C341BDC04F11404C4F1200520
:1007500000FA05F320FA04F001FA05F240EA02007B
:1007600001F0004221F0004110EBD37021FA04F6B1
:1007700042EB06015EEA430E08BF20EAD37070BD6B
:10078000C4F10C04C4F1200500FA04F320FA05F0CA
:1007900001FA04F240EA020001F0004110EBD370CC
:1007A00041F100015EEA430E08BF20EAD37070BD3C
:1007B000C4F1200500FA05F24EEA020E20FA04F315
:1007C00001FA05F243EA020321FA04F001F00041C4
:1007D00021FA04F220EA020000EBD3705EEA430E35
:1007E00008BF20EAD37070BD94F0000F0FD101F064
:1007F0000046400041EB010111F4801F08BF013C9D
:10080000F7D041EA060195F0000F18BF704703F0DA
:100810000046520043EB030313F4801F08BF013D61
:10082000F7D043EA0603704794EA0C0F0CEA13551D
:1008300018BF95EA0C0F0CD050EA410618BF52EAD7
:100840004306D1D181EA030101F000414FF00000DD
:1008500070BD50EA410606BF1046194652EA4306EB
:1008600019D094EA0C0F02D150EA013613D195EA5F
:100870000C0F05D152EA03361CBF104619460AD1A7
:1008800081EA030101F0004141F0FE4141F47001B1
:100890004FF0000070BD41F0FE4141F4780170BDA1
:1008A00070B54FF0FF0C4CF4E06C1CEA11541DBF06
:1008B0001CEA135594EA0C0F95EA0C0F00F0A7F808
:1008C000A4EB050481EA030E52EA03354FEA013135
:1008D00000F088804FEA03334FF0805545EA131348
:1008E00043EA12634FEA022245EA111545EA106510
:1008F0004FEA00260EF000419D4208BF964244F1A7
:10090000FD0404F5407402D25B084FEA3202B61AC5
:1009100065EB03055B084FEA32024FF480104FF499
:10092000002CB6EB020E75EB030E22BFB61A75460D
:1009300040EA0C005B084FEA3202B6EB020E75EBA0
:10094000030E22BFB61A754640EA5C005B084FEA08
:100950003202B6EB020E75EB030E22BFB61A7546D5
:1009600040EA9C005B084FEA3202B6EB020E75EBE0
:10097000030E22BFB61A754640EADC0055EA060EA1
:1009800018D04FEA051545EA16754FEA06164FEAE4
:10099000C30343EA52734FEAC2025FEA1C1CC0D190
:1009A00011F4801F0BD141EA00014FF000004FF01D
:1009B000004CB6E711F4801F04BF01430020B4F1DE
:1009C000FD0C88BFBCF5E06F3FF6AFAEB5EB030C96
:1009D00004BFB6EB020C5FEA500C50F1000041EB93
:1009E000045170BD0EF0004E4EEA113114EB5C0460
:1009F000C2BFD4EB0C0541EA045170BD41F4801133
:100A00004FF0000E013C90E645EA060E8DE60CEA3A
:100A1000135594EA0C0F08BF95EA0C0F3FF43BAF57
:100A200094EA0C0F0AD150EA01347FF434AF95EA0E
:100A30000C0F7FF425AF104619462CE795EA0C0FF2
:100A400006D152EA03353FF4FDAE1046194622E7BF
:100A500050EA410618BF52EA43067FF4C5AE50EA99
:100A600041047FF40DAF52EA43057FF4EBAE12E789
:100A70004FF0FF3C06E000BF4FF0010C02E000BF6A
:100A80004FF0010C4DF804CD4FEA410C7FEA6C5C4D
:100A90004FEA430C18BF7FEA6C5C1BD001B050EAF0
:100AA000410C0CBF52EA430C91EA030F02BF90EADB
:100AB000020F0020704710F1000F91EA030F58BF9A
:100AC000994208BF90422CBFD8176FEAE37040F0FC
:100AD000010070474FEA410C7FEA6C5C02D150EA9A
:100AE000013C07D14FEA430C7FEA6C5CD6D152EA55
:100AF000033CD3D05DF8040B704700BF844610461A
:100B000062468C461946634600E000BF01B5FFF718
:100B1000B7FF002848BF10F1000F01BD4DF808EDE8
:100B2000FFF7F4FF0CBF012000205DF808FB00BFB9
:100B30004DF808EDFFF7EAFF34BF012000205DF813
:100B400008FB00BF4DF808EDFFF7E0FF94BF012060
:100B500000205DF808FB00BF4DF808EDFFF7CEFF61
:100B600094BF012000205DF808FB00BF4DF808EDA0
:100B7000FFF7C4FF34BF012000205DF808FB00BF71
:100B80004FEA410C7FEA6C5C02D150EA013C0AD189
:100B90004FEA430C7FEA6C5C02D152EA033C02D17B
:100BA0004FF0000070474FF0010070474FEA4102DC
:100BB00012F5001215D211D56FF47873B3EB6252AF
:100BC00012D94FEAC12343F0004343EA505311F0D6
:100BD000004F23FA02F018BF404270474FF0000068
:100BE000704750EA013005D111F0004008BF6FF0A6
:100BF000004070474FF00000704700BF4A0011D21C
:100C000012F5001211D20DD56FF47873B3EB625266
:100C10000ED44FEAC12343F0004343EA505323FA72
:100C200002F070474FF00000704750EA013002D1E7
:100C30004FF0FF3070474FF0000070474FEA41021D
:100C4000B2F1E04324BFB3F5001CDCF1FE5C0DD92A
:100C500001F0004C4FEAC0024CEA5070B2F1004F74
:100C600040EB830008BF20F00100704711F0804F77
:100C700021D113F13872BCBF01F00040704741F43C
:100C800080114FEA5252C2F11802C2F1200C10FA40
:100C90000CF320FA02F018BF40F001004FEAC12324
:100CA0004FEAD32303FA0CFC40EA0C0023FA02F3C8
:100CB0004FEA4303CCE77FEA625307D150EA01339E
:100CC0001EBF4FF0FE4040F44000704701F000406E
:100CD00040F0FE4040F40000704700BF80F000404C
:100CE00002E000BF81F0004142001FBF5FEA410304
:100CF00092EA030F7FEA226C7FEA236C6AD04FEA04
:100D00001262D2EB1363C1BFD21841404840414048
:100D1000B8BF5B42192B88BF704710F0004F40F4FA
:100D2000000020F07F4018BF404211F0004F41F416
:100D3000000121F07F4118BF494292EA030F3FD0E2
:100D4000A2F1010241FA03FC10EB0C00C3F12003F5
:100D500001FA03F100F0004302D5494260EB400084
:100D6000B0F5000F13D3B0F1807F06D340084FEAEF
:100D7000310102F10102FE2A51D2B1F1004F40EBE4
:100D8000C25008BF20F0010040EA0300704749004C
:100D900040EB0000013A28BFB0F5000FEDD2B0FAE9
:100DA00080FCACF1080CB2EB0C0200FA0CF0AABF0C
:100DB00000EBC25052421843BCBFD04018437047AA
:100DC00092F0000F81F4000106BF80F400000132B0
:100DD000013BB5E74FEA41037FEA226C18BF7FEA87
:100DE000236C21D092EA030F04D092F0000F08BFC9
:100DF0000846704790EA010F1CBF0020704712F0B0
:100E00007F4F04D1400028BF40F00040704712F1EE
:100E100000723CBF00F50000704700F0004343F053
:100E2000FE4040F4000070477FEA226216BF084689
:100E30007FEA23630146420206BF5FEA412390EA4C
:100E4000010F40F4800070474FF0000304E000BF42
:100E500010F0004348BF40425FEA000C08BF7047F3
:100E600043F0964301464FF000001CE050EA0102B7
:100E700008BF70474FF000030AE000BF50EA0102CC
:100E800008BF704711F0004302D5404261EB4101B9
:100E90005FEA010C02BF84460146002043F0B643DE
:100EA00008BFA3F18053A3F50003BCFA8CF2083A03
:100EB000A3EBC25310DB01FA02FC634400FA02FC0C
:100EC000C2F12002BCF1004F20FA02F243EB020013
:100ED00008BF20F00100704702F1200201FA02FC75
:100EE000C2F1200250EA4C0021FA02F243EB020068
:100EF00008BF20EADC7070477BB972B90029BEBF19
:100F000000204FF0004106E008BF00281CBF6FF032
:100F100000414FF0FF3000F029BAADF1080C6DE947
:100F200004CE002909DB002B1ADB00F0B7F8DDF84E
:100F300004E0DDE9022304B07047404261EB410167
:100F4000002B1BDB00F0AAF8DDF804E0DDE902234A
:100F500004B0404261EB4101524263EB43037047EE
:100F6000524263EB430300F099F8DDF804E0DDE959
:100F7000022304B0404261EB41017047524263EBEF
:100F8000430300F08BF8DDF804E0DDE9022304B050
:100F9000524263EB4303704753B94AB9002908BF73
:100FA00000281CBF4FF0FF314FF0FF3000F0DEB9DA
:100FB000ADF1080C6DE904CE00F070F8DDF804E046
:100FC000DDE9022304B0704707EE900AF5EEC07A1F
:100FD000F1EE10FA01D400F023B8F1EE677A08B50B
:100FE00017EE900A00F01CF8404261EB410108BD89
:100FF00038B50022002304460D46FFF799FD28B9B5
:1010000020462946BDE8384000F02AB8204605F1C0
:10101000004100F025F8404261EB410138BD00BFBE
:10102000D0B5FFF7BBFA0C4B002206460F46FFF780
:101030000DFBFFF7E3FD0446FFF78EFA074B002296
:10104000FFF704FB02460B4630463946FFF746F9E8
:10105000FFF7D4FD2146D0BD0000F03D0000F04177
:10106000D0B50C4B002206460F46FFF7EFFAFFF70C
:10107000C5FD0446FFF770FA074B0022FFF7E6FABA
:1010800002460B4630463946FFF728F9FFF7B6FD12
:101090002146D0BD0000F03D0000F0412DE9F047B1
:1010A000089D04468E46002B4DD18A42944669D94C
:1010B000B2FA82F252B101FA02F3C2F1200120FA2F
:1010C00001F10CFA02FC41EA030E94404FEA1C487D
:1010D000210CBEFBF8F61FFA8CF708FB16E341EA79
:1010E000034306FB07F199420AD91CEB030306F1FF
:1010F000FF3080F01F81994240F21C81023E634420
:101100005B1AA4B2B3FBF8F008FB103344EA0344C3
:1011100000FB07F7A7420AD91CEB040400F1FF33D8
:1011200080F00A81A74240F207816444023840EA15
:101130000640E41B00261DB1D4400023C5E900434E
:101140003146BDE8F0878B4209D9002D00F0EF80D1
:101150000026C5E9000130463146BDE8F087B3FA04
:1011600083F6002E4AD18B4202D3824200F2F980EC
:10117000841A61EB030301209E46002DE0D0C5E9EF
:10118000004EDDE702B9FFDEB2FA82F2002A40F03B
:101190009280A1EB0C014FEA1C471FFA8CFE01263E
:1011A000200CB1FBF7F307FB131140EA01410EFBE2
:1011B00003F0884208D91CEB010103F1FF3802D289
:1011C000884200F2CB804346091AA4B2B1FBF7F083
:1011D00007FB101144EA01440EFB00FEA64508D9A6
:1011E0001CEB040400F1FF3102D2A64500F2BB80E3
:1011F0000846A4EB0E0440EA03409CE7C6F1200732
:10120000B34022FA07FC4CEA030C20FA07F401FA77
:1012100006F31C43F9404FEA1C4900FA06F3B1FB00
:10122000F9F8200C1FFA8CFE09FB181140EA014165
:1012300008FB0EF0884202FA06F20BD91CEB010102
:1012400008F1FF3A80F08880884240F28580A8F15A
:1012500002086144091AA4B2B1FBF9F009FB1011AC
:1012600044EA014100FB0EFE8E4508D91CEB01014A
:1012700000F1FF346CD28E456AD90238614440EAED
:101280000840A0FB0294A1EB0E01A142C846A6466D
:1012900056D353D05DB1B3EB080261EB0E0101FAF6
:1012A00007F722FA06F3F1401F43C5E90071002653
:1012B0003146BDE8F087C2F12003D8400CFA02FCA9
:1012C00021FA03F3914001434FEA1C471FFA8CFEB9
:1012D000B3FBF7F007FB10360B0C43EA064300FBA9
:1012E0000EF69E4204FA02F408D91CEB030300F147
:1012F000FF382FD29E422DD9023863449B1B89B2FE
:10130000B3FBF7F607FB163341EA034106FB0EF386
:101310008B4208D91CEB010106F1FF3816D28B4233
:1013200014D9023E6144C91A46EA004638E72E46FF
:10133000284605E70646E3E61846F8E64B45A9D2F7
:10134000B9EB020864EB0C0E0138A3E74646EAE766
:10135000204694E74046D1E7D0467BE7023B614414
:1013600032E7304609E76444023842E7704700BF7D
:1013700080B584B000AF78607B681B680D4A9342EB
:1013800013D10D4B1B6B0C4A43F4000313630A4B40
:101390001B6B03F40003FB60FB68002205215A204D
:1013A00002F010FF5A2002F029FF00BF1037BD469F
:1013B00080BD00BF00B002400038024080B586B05A
:1013C00000AF3B1D00221A605A609A60DA601A6111
:1013D0003A4B1B68002B6DD1384B01221A60384BF9
:1013E0009B6B374A43F001039363354B9B6B03F0D0
:1013F00001033B603B684FF683737B600223BB6055
:101400000023FB6003233B610C237B613B1D1946DA
:101410002C4803F099FC48F233137B600223BB6035
:101420000023FB6003233B610C237B613B1D1946BA
:10143000254803F089FC4CF203737B600223BB60F8
:101440000023FB6003233B610C237B613B1D19469A
:101450001E4803F079FC4FF63F037B600223BB601C
:101460000023FB6003233B610C237B613B1D19467A
:10147000174803F069FC08237B600223BB6000234C
:10148000FB6003233B610C237B613B1D1946114824
:1014900003F05AFC09237B600223BB600023FB603E
:1014A00003233B610C237B613B1D19460A4803F073
:1014B0004BFC00E000BF1837BD4680BD3C14002047
:1014C000003802400010024000180240000C0240A8
:1014D00000140240001C02400008024080B582B0A7
:1014E00000AF7860FFF76AFF00BF0837BD4680BDD8
:1014F00080B500AF044A002104480AF05DFE0346AF
:10150000034A136000BF80BD98D70808151500086E
:101510004014002080B582B000AF786062F0A0FA7D
:1015200061F03CFC61F06EFCFCE7000080B590B01F
:1015300000AF07F12C0300221A605A609A60DA604B
:101540001A61AF4B1B6BAE4A43F010031363AC4BF5
:101550001B6B03F01003BB62BB6AA94B1B6BA84A51
:1015600043F040031363A64B1B6B03F040037B6205
:101570007B6AA34B1B6BA24A43F002031363A04B8D
:101580001B6B03F002033B623B6A9D4B1B6B9C4A47
:1015900043F0040313639A4B1B6B03F00403FB61DA
:1015A000FB69974B1B6B964A43F001031363944B03
:1015B0001B6B03F00103BB61BB69914B1B6B904A32
:1015C00043F4007313638E4B1B6B03F400737B6156
:1015D0007B698B4B1B6B8A4A43F008031363884B70
:1015E0001B6B03F008033B613B69854B1B6B844A13
:1015F00043F480631363824B1B6B03F48063FB60D3
:10160000FB687F4B1B6B7E4A43F4807313637C4BF8
:101610001B6B03F48073BB60BB68794B1B6B784A10
:1016200043F020031363764B1B6B03F020037B60B6
:101630007B68734B1B6B724A43F080031363704BE0
:101640001B6B03F080033B603B68012220216D4847
:1016500003F032FE00220C216B4803F02DFE012224
:1016600008216A4803F028FE01224FF480516648A1
:1016700003F022FE00224FF40051654803F01CFEE7
:101680000022C821634803F017FE0823FB620023F1
:101690003B6300237B6307F12C0319465E4803F08C
:1016A00053FB4FF4D043FB6202233B6300237B6375
:1016B0000323BB630B23FB6307F12C031946554837
:1016C00003F042FB4FF44073FB6212233B630123A0
:1016D0007B630023BB630423FB6307F12C031946E0
:1016E0004E4803F031FB4FF40043FB6202233B639F
:1016F00000237B630023BB630123FB6307F12C03FF
:101700001946474803F020FB4FF48053FB62002347
:101710003B6300237B6307F12C031946414803F028
:1017200013FB4023FB62404B3B6300237B6307F1C9
:101730002C031946334803F007FB2023FB620123E7
:101740003B6300237B630023BB6307F12C03194633
:101750002C4803F0F9FA41F20C03FB6201233B63CE
:1017600000237B630023BB6307F12C031946264843
:1017700003F0EAFA4FF40053FB6200233B630023BB
:101780007B6307F12C031946284803F0DDFA082390
:10179000FB6201233B6300237B630023BB6307F1F0
:1017A0002C031946194803F0CFFA1023FB620023DB
:1017B0003B6300237B6307F12C031946114803F0B8
:1017C000C3FA48F20403FB6200233B6300237B63FC
:1017D00007F12C0319460E4803F0B6FA0223FB6208
:1017E00002233B6300237B630023BB630523FB636E
:1017F00007F12C031946044803F0A6FA18E000BFCD
:1018000000380240000C0240002002400028024044
:10181000001C024000180240001002400004024078
:1018200000000240002402400000121000080240A4
:101830004FF40053FB6201233B6300237B630023CF
:10184000BB6307F12C031946534803F07DFA0123CB
:10185000FB6202233B6300237B630023BB63022301
:10186000FB6307F12C0319464C4803F06DFA4FF463
:101870000053FB624A4B3B6300237B6307F12C035D
:101880001946464803F060FA3023FB6212233B639B
:1018900000237B630323BB630423FB6307F12C0357
:1018A00019463D4803F050FAC823FB6201233B630D
:1018B00000237B630023BB6307F12C0319463948DF
:1018C00003F042FA4FF4F863FB6203233B63002307
:1018D0007B6307F12C031946334803F035FA3223B2
:1018E000FB6202233B6300237B630323BB630B2365
:1018F000FB6307F12C0319462C4803F025FA042357
:10190000FB6200233B6300237B6307F12C03194632
:10191000244803F019FA8623FB6202233B63002369
:101920007B630323BB630B23FB6307F12C03194683
:101930001F4803F009FA0123FB6203233B630023E2
:101940007B6307F12C031946194803F0FDF9402386
:10195000FB6202233B6300237B630023BB630923F9
:10196000FB6307F12C0319460B4803F0EDF94FF424
:101970004043FB6202233B6300237B630023BB6382
:101980000523FB6307F12C0319460A4803F0DCF931
:1019900000BF4037BD4680BD001C02400020024011
:1019A000000012100018024000140240000802401B
:1019B000000002400004024080B5AAB000AF786089
:1019C00007F1940300221A605A609A60DA601A6183
:1019D00007F1100384220021184682F0FBFB7B688C
:1019E0001B68264A934244D14FF480333B61002365
:1019F000FB6707F11003184606F016FC0346002BA0
:101A000001D000F0F9F91E4B1B6B1D4A43F0800317
:101A100013631B4B1B6B03F08003FB60FB684FF4ED
:101A2000C073C7F894301223C7F898300023C7F862
:101A30009C300323C7F8A0300423C7F8A43007F173
:101A4000940319460F4803F07FF90D4B1B6C0C4AA9
:101A500043F4000313640A4B1B6C03F40003BB60E4
:101A6000BB6800220521482002F0ACFB482002F0B0
:101A7000C5FB00BFA837BD4680BD00BF005C00406D
:101A800000380240001C024080B582B000AF786090
:101A90007B681B680C4A934211D10C4B1B6C0B4AA0
:101AA00023F4000313648021094803F0F9FA4FF48A
:101AB0008071074803F0F4FA482002F0ADFB00BF44
:101AC0000837BD4680BD00BF005C004000380240C2
:101AD000001C024080B58EB000AF786007F124038F
:101AE00000221A605A609A60DA601A617B681B688B
:101AF000554A934240F0A380544B5B6C534A43F0E9
:101B000080635364514B5B6C03F080633B623B6AC0
:101B10004E4B1B6B4D4A43F0100313634B4B1B6B37
:101B200003F01003FB61FB69484B1B6B474A43F40E
:101B300000731363454B1B6B03F40073BB61BB69FC
:101B4000424B1B6B414A43F4806313633F4B1B6B57
:101B500003F480637B617B693C4B1B6B3B4A43F026
:101B600040031363394B1B6B03F040033B613B693C
:101B7000364B1B6B354A43F480731363334B1B6B3B
:101B800003F48073FB60FB6810237B620223BB625B
:101B90000023FB6200233B630E237B6307F12403D6
:101BA00019462B4803F0D0F84EF6FF737B620223F0
:101BB000BB620023FB6200233B630E237B6307F1C0
:101BC00024031946234803F0BFF8F7237B6202235E
:101BD000BB620023FB6200233B630E237B6307F1A0
:101BE000240319461C4803F0AFF84FF480537B627E
:101BF0000223BB620023FB6200233B6309237B6358
:101C000007F124031946154803F09EF84FF44643A4
:101C10007B620223BB620023FB6200233B630E2333
:101C20007B6307F1240319460D4803F08DF8002269
:101C30000521582002F0C6FA582002F0DFFA00BF52
:101C40003837BD4680BD00BF006801400038024003
:101C50000010024000240240002802400018024008
:101C6000002002400000000080B584B000AF786022
:101C700039604FF000024FF00003C7E90223D7E9B3
:101C8000020111A3D3E90023FFF786F902460B46B0
:101C90007968C1E90023D7E902010BA3D3E9002346
:101CA000FFF77AF9104619464FF47A724FF00003A5
:101CB000FFF772F902460B467B689A6000231846CC
:101CC0001037BD4680BD00BF00CA9A3B000000002F
:101CD00080B500AF02F048F900F00CF8FFF726FCE1
:101CE00000F090F80AF0FEF9FFF702FC0AF02EFA75
:101CF000FEE7000080B594B000AF07F1200330226A
:101D00000021184682F066FA07F10C0300221A60DF
:101D10005A609A60DA601A6105F07EFD2B4B1B6CED
:101D20002A4A43F080531364284B1B6C03F0805302
:101D3000BB60BB68264B1B68254A43F440431360D5
:101D4000234B1B6803F440437B607B6801233B62A9
:101D50004FF480337B620223BB634FF48003FB6349
:101D600019233B644FF4C8737B640223BB640923CB
:101D7000FB6407F12003184605F0AEFD0346002B77
:101D800001D000F039F805F057FD0346002B01D0D3
:101D900000F032F80F23FB6002233B6100237B61DC
:101DA0004FF4A053BB614FF48053FB6107F10C0368
:101DB0000621184606F034F80346002B01D000F047
:101DC0001BF800BF5037BD4680BD00BF0038024041
:101DD0000070004080B582B000AF78607B681B68FF
:101DE000044A934201D102F0CDF800BF0837BD4646
:101DF00080BD00BF0010004080B400AF72B600BFCD
:101E0000FEE7000080B584B002AF0023FB7100F054
:101E100075FF0346FB71FB79002B14BF01230023E0
:101E2000DBB2184600F026F84FF04041002000F0E9
:101E3000FDFF002001F05AF800210C4804F04EF993
:101E400000F026F84FF040431846094B19464FF46E
:101E5000887301934FF4F07300930023002200F085
:101E600037F800BF0837BD4680BD00BF6C150020A5
:101E700000B80BC080B483B000AF78607B68002BE3
:101E800000D0FEE700BF0C37BD465DF8047B70470D
:101E900080B500AF4FF0FF3001F09AF8094801F02B
:101EA0004DF84FF0FF3001F031F8074801F060F8CD
:101EB0000649012001F0C2F94FF4FA6002F082F8FD
:101EC00000BF80BD0000FFFF3C0000201CC30808CD
:101ED00080B588B002AFF860B96011461A460B466B
:101EE000FB801346BB80BB884FF4487203FB02F2B1
:101EF000FB8813445B001A46BB6813447B61FB6894
:101F00003B611F4B00225A601D4B02229A603B8CA2
:101F1000C3F548731A461A4BDA60194B00221A614E
:101F2000174B00221A63164BFF225A63144B0222EE
:101F3000DA62134B00229A62114B124A1A6010485F
:101F400002F036FB0346002B16D101210C4802F0AB
:101F5000CDFD0346002B0FD13A8CBB8C009313466A
:101F60007A693969064802F06DFB0346002B03D1FC
:101F70006421034802F0C0FB00BF1837BD4680BD96
:101F8000FC13002000B0024080B582B000AF114BBE
:101F90001B6C104A43F0805313640E4B1B6C03F010
:101FA00080537B607B680B4B5B6C0A4A43F4804335
:101FB0005364084B5B6C03F480433B603B68002236
:101FC0000F216FF0010002F0FDF800BF0837BD4699
:101FD00080BD00BF0038024080B58EB000AF786091
:101FE0000023FB620023BB62334B1B6C324A43F07D
:101FF00010031364304B1B6C03F01003FB60FB6891
:1020000007F1100207F114031146184606F0DAF83A
:102010003B6AFB62FB6A002B03D106F0BFF87863D2
:1020200004E006F0BBF803465B007B637B6B234A4E
:10203000A2FB03239B0C013BBB62214B214A1A608C
:102040001F4B40F2E732DA601D4ABB6A53601C4BFB
:1020500000221A611A4B00229A60194B00229A61E1
:10206000174806F050FD034687F8333097F83330B1
:10207000002B1BD1124806F071FD034687F8333060
:1020800097F83330002B11D1362002F0B7F87B6877
:102090000F2B08D800227968362002F093F80A4AFC
:1020A0007B68136002E0012387F8333097F8333000
:1020B00018463837BD4680BD0038024083DE1B43DA
:1020C00090140020001000404800002080B400AFB1
:1020D000FEE780B400AFFEE780B400AFFEE780B457
:1020E00000AFFEE780B400AFFEE780B400AF00BFF2
:1020F000BD465DF8047B704780B500AF024806F02E
:1021000057FD00BF80BD00BFD814002080B500AFD0
:10211000024806F04DFD00BF80BD00BF90140020B6
:1021200080B500AF024804F0FFFA00BF80BD00BFD9
:10213000E48A022080B500AF024803F0C5FB00BF6F
:1021400080BD00BF4414002080B500AF024803F0FA
:10215000CFFE00BF80BD00BF6C15002080B500AF72
:10216000024802F0B2FB00BF80BD00BFFC1300209C
:1021700080B400AF01231846BD465DF8047B70476C
:1021800080B582B000AF7860396081F0CFF9034646
:1021900016221A604FF0FF3318460837BD4680BD3F
:1021A00080B582B000AF78604FF0FF317868FFF7FC
:1021B000E7FFFEE780B586B000AFF860B9607A60EF
:1021C00000237B610AE0AFF300800146BB685A1C24
:1021D000BA60CAB21A707B6901337B617A697B6825
:1021E0009A42F0DB7B6818461837BD4680BD80B543
:1021F00086B000AFF860B9607A6000237B6109E0C7
:10220000BB685A1CBA601B781846AFF300807B6924
:1022100001337B617A697B689A42F1DB7B681846FF
:102220001837BD4680BD80B483B000AF78604FF0F2
:10223000FF3318460C37BD465DF8047B704780B409
:1022400083B000AF786039603B684FF400525A6049
:10225000002318460C37BD465DF8047B704780B4F8
:1022600083B000AF7860012318460C37BD465DF897
:10227000047B704780B485B000AFF860B9607A60C5
:10228000002318461437BD465DF8047B70470000F4
:1022900080B586B000AF7860144A154BD31A7B61C5
:1022A0007B693B61134B1B68002B02D1114B124A17
:1022B0001A60104B1A687B6813443A699A4207D235
:1022C00081F034F903460C221A604FF0FF3309E025
:1022D000084B1B68FB60074B1A687B681344054A70
:1022E0001360FB6818461837BD4680BD0000052006
:1022F00000040000D414002060A5022080B400AFC8
:10230000064BD3F88830054A43F47003C2F888308E
:1023100000BFBD465DF8047B704700BF00ED00E0E4
:1023200080B58CB000AF786007F11C0300221A6002
:102330005A609A60DA601A617B681B68324A93427D
:1023400029D1324B5B6C314A43F0010353642F4B6C
:102350005B6C03F00103BB61BB692C4B1B6B2B4A0D
:1023600043F001031363294B1B6B03F001037B61F3
:102370007B694FF48073FB6102233B6200237B6225
:102380000023BB620123FB6207F11C0319462048AE
:1023900002F0DAFC34E07B681B681E4A93422FD1BE
:1023A0001A4B1B6C194A43F002031364174B1B6C46
:1023B00003F002033B613B69144B1B6B134A43F070
:1023C00002031363114B1B6B03F00203FB60FB68FA
:1023D0001023FB6102233B6200237B620023BB626C
:1023E0000223FB6207F11C0319460B4802F0ACFC08
:1023F000002205211D2001F0E5FE1D2001F0FEFE5A
:1024000000BF3037BD4680BD0000014000380240AB
:10241000000002400004004000040240DFF834D015
:102420000D480E490E4A002302E0D458C45004332C
:10243000C4188C42F9D30B4A0B4C002301E0136003
:102440000432A242FBD3FFF759FF81F0DDFCFFF716
:102450003FFC70470000052000000020DC13002036
:10246000244A0A08E01300205CA50220FEE780B59C
:1024700082B000AF0346FB80C82000F033FC00F0C0
:102480007BFA00BF0837BD4680BD80B483B000AF83
:102490000346FB8000BF0C37BD465DF8047B7047E8
:1024A00080B584B000AF0346FB8000237B7300231C
:1024B000FB730023BB7300F05FFA0023FB7310E093
:1024C000FB88DBB2A821184600F0EEFB03467B73C5
:1024D0007B7BDBB2512B01D10123BB73FB7B01332F
:1024E000FB73FB7B022B02D8BB7B002BE8D07B7BF2
:1024F000DBB29BB218461037BD4680BD80B582B0B6
:1025000000AF0346FB80FB88184600F045FAFB88C5
:10251000184600F033F900BF0837BD4680BD000003
:1025200080B584B000AF0346FB800023FB73FB88BB
:10253000DBB20221184600F0B7FB0346FB73FB7BBE
:10254000DBB203F00F03DBB2FB73FB7BDBB2052BCB
:1025500001D90023FB73FB7BDAB2054B5A70044BA5
:1025600000229A70FB7BDBB218461037BD4680BD57
:102570001815002080B586B000AF0346B9607A60B8
:10258000FB810023FB740023FB750023BB75002334
:102590007B7500233B756D4B9A786C4B5B789A4248
:1025A00080F0CF80694B9B78092B71D801A252F83B
:1025B00023F000BFDD250008EF25000801260008F4
:1025C000132600082526000837260008492600089B
:1025D0005B2600086D2600087F2600080423FB7593
:1025E0000323BB7506237B7505233B7551E00A2346
:1025F000FB750923BB750C237B750B233B7548E0EA
:102600001023FB750F23BB7512237B7511233B75BC
:102610003FE01623FB751523BB7518237B75172325
:102620003B7536E01C23FB751B23BB751E237B7596
:102630001D233B752DE02223FB752123BB7524232D
:102640007B7523233B7524E02823FB752723BB756B
:102650002A237B7529233B751BE02E23FB752D2335
:10266000BB7530237B752F233B7512E03423FB753C
:102670003323BB7536237B7535233B7509E03A233D
:10268000FB753923BB753C237B753B233B7500E011
:1026900000BFFB89DBB2FA7D1146184600F004FB4F
:1026A0000346FB74FB7CDBB29AB2294B1A80FB8990
:1026B000DBB2BA7D1146184600F0F6FA0346FB7409
:1026C000FB7CDBB21B0203F470631AB2204B1B8845
:1026D0001BB213431BB29AB21D4B1A801C4B1A88B3
:1026E000BB681A80FB89DBB27A7D1146184600F080
:1026F000DBFA0346FB74FB7CDBB29AB2144B1A8004
:10270000FB89DBB23A7D1146184600F0CDFA03464C
:10271000FB74FB7CDBB21B0203F470631AB20C4B3C
:102720001B881BB213431BB29AB2094B1A80084B89
:102730001A887B681A80054B9B780133DAB2034B09
:102740009A7000BF1837BD4680BD00BF1815002025
:102750001C15002080B584B000AF0346FB80002329
:10276000FB730123FB73FB88DBB2FA7BA4211846C1
:1027700000F080FA00BF1037BD4680BD80B584B040
:1027800000AF0346FB800023FB730023FB73FB8831
:10279000DBB2FA7BA421184600F06CFA00BF1037B8
:1027A000BD4680BD80B483B000AF0346FB800023EC
:1027B00018460C37BD465DF8047B704780B483B083
:1027C00000AF0346FB8000BF0C37BD465DF8047BBD
:1027D000704780B584B000AF03463960FB800023AA
:1027E000FB73FB88DBB20121184600F05DFA03465B
:1027F000FB73FB7BDBB21A463B681A6000BF1037E5
:10280000BD4680BD80B586B000AFB9607A603B60E0
:102810000346FB8100233B750023FB750023BB753A
:1028200000237B754D4B5B781A46BB68934280F062
:102830009080BB68092B5DD801A252F823F000BF3D
:1028400069280008772800088528000893280008D0
:10285000A1280008AF280008BD280008CB280008E0
:10286000D9280008E72800080323FB750723BB7558
:1028700008237B753FE00923FB750D23BB750E23F1
:102880007B7538E00F23FB751323BB7514237B7511
:1028900031E01523FB751923BB751A237B752AE0DC
:1028A0001B23FB751F23BB7520237B7523E021238E
:1028B000FB752523BB7526237B751CE02723FB7541
:1028C0002B23BB752C237B7515E02D23FB75312342
:1028D000BB7532237B750EE03323FB753723BB7545
:1028E00038237B7507E03923FB753D23BB753E23F9
:1028F0007B7500E000BFFB89DBB2FA7D114618460C
:1029000000F0D2F903463B753B7DDBB29B1103F02F
:1029100003023B6A1A60FB89DBB2BA7D1146184696
:1029200000F0C2F903463B753B7DDBB21A467B687B
:102930001A60FB89DBB27A7D1146184600F0B4F9C3
:1029400003463B753B7DDBB21B1103F004023B6881
:102950001A6000BF1837BD4680BD00BF18150020A3
:1029600080B400AF034B1B781846BD465DF8047B6E
:10297000704700BF1815002080B500AFFFF7F0FFCB
:102980000346002B04D100F06BF9024B01221A70B0
:1029900000BF80BD1815002080B485B000AF03468D
:1029A000FB800023FB60FB6818461437BD465DF8CA
:1029B000047B704780B58CB000AF78607B68514A6B
:1029C00093424DD1504B1B6B4F4A43F0800313632E
:1029D0004D4B1B6B03F08003BB61BB698023FB6124
:1029E00012233B6200237B620223BB620423FB624F
:1029F00007F11C031946454802F0A6F94FF480730D
:102A0000FB6107F11C031946404802F09DF93E4B5B
:102A10001B6C3D4A43F4000313643B4B1B6C03F4F3
:102A200000037B617B69384B1B6A374A43F4000320
:102A30001362354B1B6A344A23F4000313620022ED
:102A40000F21482001F0BEFB482001F0D7FB0022F7
:102A50000F21492001F0B6FB492001F0CFFB4DE0EA
:102A6000294B1B6B284A43F002031363264B1B6B55
:102A700003F002033B613B694FF48073FB61122357
:102A80003B6200237B620223BB620423FB6207F1EB
:102A90001C0319461E4802F057F94FF40073FB61FE
:102AA00007F11C0319461A4802F04EF9164B1B6C2D
:102AB000154A43F400131364134B1B6C03F4001307
:102AC000FB60FB68104B1B6A0F4A43F40013136250
:102AD0000D4B1B6A0C4A23F40013136200220F21D2
:102AE0001F2001F06FFB1F2001F088FB00220F2147
:102AF000202001F067FB202001F080FB00BF303771
:102B0000BD4680BD2015002000380240001C024058
:102B10000004024080B582B000AF7860786802F0AF
:102B2000EDFE0346002B25D17B68144A934203D166
:102B30007B68134A1A6002E07B68124A1A607B685D
:102B4000114A5A607B6800229A607B680122DA6031
:102B50007B6800221A617B6800225A617B68002230
:102B6000DA617B6800221A627868FFF723FF7868D1
:102B700002F0BCFB00BF0837BD4680BD2015002019
:102B8000005C0040005400403227914080B58AB07C
:102B900004AFF860084611461A460346FB720B461E
:102BA0003B811346FB800023FB75FB7A99B2F888C2
:102BB0003A894FF47A730293BB8C01933B6A00937A
:102BC0000346F86802F066FD0346FB75FB7D002BAB
:102BD00004D0FB7A1946F86800F032F8FB7D1846FD
:102BE0001837BD4680BD80B58AB004AFF86008468E
:102BF00011461A460346FB720B463B811346FB8087
:102C00000023FB75FB7A99B2F8883A894FF47A73FE
:102C10000293BB8C01933B6A00930346F86802F071
:102C200025FC0346FB75FB7D002B04D0FB7A19467F
:102C3000F86800F005F8FB7D18461837BD4680BDE2
:102C400080B582B000AF78600B46FB70786802F008
:102C5000DDFB7868FFF75EFF00BF0837BD4680BD2B
:102C600080B500AF0248FFF755FF00BF80BD00BF31
:102C70002015002080B584B002AF0346FB710B46DF
:102C8000BB7113467B71BB799AB2F9790123019329
:102C90007B1D009301230348FFF7A5FF00BF083702
:102CA000BD4680BD2015002080B586B002AF03462A
:102CB0000A46FB711346BB710023FB73BB799AB2C2
:102CC000F9790123019307F10F03009301230448CD
:102CD000FFF75CFFFB7B18461037BD4680BD00BF89
:102CE0002015002080B582B000AF7860786801F0D0
:102CF00069F900BF0837BD4680BD000080B500AF50
:102D0000314B28225A61304B09229A612E4B3522D1
:102D1000DA612D4B0B221A622B4B40F21B129A6286
:102D2000294B40F215225A62274B40F21D121A63BA
:102D3000254B40F23522DA620021234800F0B8FB2F
:102D4000214B4FF4F0721A661F4B4FF488725A668B
:102D50001D4B002283F834201B4B002283F83520C2
:102D6000194B002283F83620174B00225A60164B6D
:102D700000229A60144B0022DA60134B00221A6181
:102D8000114B124A1A60104803F0E0F90346002B79
:102D900003D100210C4800F0B1FA0B4802F0D8FF33
:102DA00001224FF480510A4802F086FA01220821DC
:102DB000084802F081FA00F09BFC074800F0D8F8C0
:102DC0000023184680BD00BF6C150020006801403C
:102DD00000200240002802403400002080B400AFF0
:102DE000064B1B68064A342101FB03F3134460338E
:102DF0001B681846BD465DF8047B704754160020DA
:102E00006C15002080B400AF064B1B68064A3421C5
:102E100001FB03F3134464331B681846BD465DF899
:102E2000047B7047541600206C15002080B590B0CC
:102E300000AF03463960FB800023FB60FFF7CEFF45
:102E400003463B6100237B61FFF7DCFF0346BB6168
:102E50000223FB613B683B63FF233B6200237B62F1
:102E6000002387F83C30002387F83D30002387F8A3
:102E70003E304FF4C063BB620723FB62FFF7AEFF37
:102E800003467B63FFF7BEFF0346BB63FA8807F187
:102E90000C031946124803F0E3F8FA881149134667
:102EA0005B0013449B000B4404334FF0FF321A6065
:102EB000FA880C4913465B0013449B000B4408330B
:102EC000094A1A60FA88074913465B0013449B00BD
:102ED0000B444FF07F421A6000BF4037BD4680BDB3
:102EE0006C150020581600203400002080B483B0F8
:102EF00000AF7860044A7B68136000BF0C37BD46A2
:102F00005DF8047B704700BF5416002080B483B086
:102F100000AF7860074B1A68074913465B001344FB
:102F20009B000B447A681A6000BF0C37BD465DF801
:102F3000047B7047541600205816002080B483B0DC
:102F400000AF7860084B1A68084913465B001344C9
:102F50009B000B4404337A681A6000BF0C37BD46EF
:102F60005DF8047B704700BF5416002058160020FF
:102F700080B483B000AF7860084B1A6808491346E4
:102F80005B0013449B000B4408337A681A6000BF4F
:102F90000C37BD465DF8047B704700BF5416002017
:102FA0005816002080B400AF074B1A680749134633
:102FB0005B0013449B000B4408331B681846BD4656
:102FC0005DF8047B704700BF54160020581600209F
:102FD000F0B585B002AF7860104B1C680F4B1B68D2
:102FE0000F4A342101FB03F313445C331B681E4674
:102FF000FFF7F4FE0546FFF705FF02467B680193E5
:103000000023009313462A463146204600F024FB55
:1030100000BF00BF0C37BD46F0BD00BF54160020F6
:103020006C15002090B583B000AF0346FB800B46C3
:10303000BB801346FB701B4B1A681B4913465B0091
:1030400013449B000B4408331B681968FB78A3F1F9
:103050002000144B1A68144C13465B0013449B0069
:10306000234408331B68DB8803FB00F00D4B1A6810
:103070000D4C13465B0013449B00234408331B682C
:103080009B880733002B00DA0733DB1000FB03F3C8
:10309000CA18B988FB88184600F026FA00BF0C371A
:1030A000BD4690BD5416002058160020B0B588B01B
:1030B00000AFBA601A460346FB810B46BB8113463C
:1030C000FB710123FB830023BB830023BB6100232F
:1030D0003B61BB687B6102E0BB690133BB617B691B
:1030E0005A1C7A611B78002BF6D1FFF777FE014658
:1030F000504B1A68504813465B0013449B0003442E
:1031000008331B689B88B1FBF3F33B61FB79032B0E
:103110001CD0032B33DC012B02D0022B19D02EE064
:103120003A69BB69D11A434B1A68434813465B009E
:1031300013449B00034408331B689B8801FB03F383
:103140005B089AB2FB891344FB831BE0FB89FB837A
:1031500018E03A69BB69D31A99B2364B1A683648F7
:1031600013465B0013449B00034408331B689B8891
:1031700011FB03F39AB2FB89D31AFB8302E0FB89AC
:10318000FB8300BFFB8B002B03D0B7F91E30002B55
:103190001DDA0123FB831AE0BB681A78B989FB8B1F
:1031A0001846FFF73FFF234B1A68234913465B007D
:1031B00013449B000B4408331B689A88FB8B134411
:1031C000FB83BB680133BB60BB8B0133BB83BB6834
:1031D0001B78002B14BF01230023DCB2FFF7FEFD98
:1031E000B98B144B1A68144D13465B0013449B00B3
:1031F0002B4408331B689B8801FB03F3C31A99B265
:103200000C4B1A680C4813465B0013449B000344A4
:1032100008331B689B8899422CBF01230023DBB233
:103220002340DBB2002BB7D100BF00BF2037BD4623
:10323000B0BD00BF541600205816002080B582B0E3
:1032400000AF03463960FB80FFF7ACFE0346DB8826
:10325000FA8812FB03F399B203233A680020FFF7C0
:1032600025FF00BF0837BD4680BD0000B0B582B065
:1032700000AF03463A60FB800B46BB801D4B1B68CA
:103280001D4A342101FB03F3134448331B68022B0E
:1032900016D1184B1B68184A342101FB03F3134461
:1032A0005C331C68BD88FFF799FD034603FB05F2FC
:1032B000FB8813445B0023443A6892B21A8015E0FD
:1032C0000C4B1B680C4A342101FB03F313445C33A1
:1032D0001C68BD88FFF782FD034603FB05F2FB88EF
:1032E00013449B0023441A463B68136000BF083711
:1032F000BD46B0BD541600206C15002080B590B0BE
:1033000000AF78603960644B5B6C634A43F0806364
:103310005364614B5B6C03F08063BB62BB6A5E4BC2
:103320001B6B5D4A43F4000313635B4B1B6B03F49D
:1033300000037B627B6A584B1B6B574A43F01003B8
:103340001363554B1B6B03F010033B623B6A524BFC
:103350001B6B514A43F0400313634F4B1B6B03F04D
:103360004003FB61FB694C4B1B6B4B4A43F480737E
:103370001363494B1B6B03F48073BB61BB69464B02
:103380001B6B454A43F400731363434B1B6B03F4FD
:1033900000737B617B69404B1B6B3F4A43F4806346
:1033A00013633D4B1B6B03F480633B613B693A4BFA
:1033B0001B6B394A43F480731363374B1B6B03F465
:1033C0008073FB60FB68344B1B6B334A43F48063B0
:1033D0001363314B1B6B03F48063BB60BB6810232A
:1033E000FB6202233B6300237B630223BB630E2348
:1033F000FB6307F12C031946284801F0A5FC4FF4A4
:103400008053FB6202233B630923FB6307F12C0318
:103410001946234801F098FC4FF46643FB620223EF
:103420003B630E23FB6307F12C0319461D4801F093
:103430008BFC4EF6FF73FB6202233B630E23FB63A0
:1034400007F12C031946184801F07EFCF723FB62B4
:1034500002233B630E23FB6307F12C031946134839
:1034600001F072FC4FF48053FB6201233B6307F1D0
:103470002C0319460B4801F067FC0823FB6201236B
:103480003B6307F12C031946084801F05DFC00BFBF
:103490004037BD4680BD00BF0038024000100240EA
:1034A0000018024000200240002402400028024090
:1034B00080B582B000AF786039600A4B08221A608C
:1034C000084BC0225A61074B0522DA61054B4FF4C5
:1034D0000032DA62034804F0A7FE00BF0837BD4699
:1034E00080BD00BF7016002080B588B000AF0346D5
:1034F0003A60FB800B46BB800023FB610023BB616D
:10350000534B1A68534913465B0013449B000B440A
:1035100008331B68DB887B824D4B1A684D49134684
:103520005B0013449B000B4408331B689B883B8261
:103530003B8A0733002B00DA0733DB10DBB2DB00FA
:10354000DAB23B8ADBB2D31AFB730023FB6176E06D
:103550003B8A0733002B00DA0733DB101A46FB697E
:1035600002FB03F33A681344BB603B8A0733002B2A
:1035700000DA0733DB10012B02D0022B04D00CE061
:10358000BB681B787B6116E0BB681B781B02BA68BE
:103590000132127813437B610DE0BB681B781A047B
:1035A000BB6801331B781B021343BA6802321278DE
:1035B00013437B6100BF0023BB6136E03A8ABB69DD
:1035C000D21AFB7B1344013B012202FA03F31A4691
:1035D0007B691340002B12D0BB699AB2FB8813445D
:1035E00098B21B4B1A681B4913465B0013449B009F
:1035F0000B441A68BB881946FFF738FE12E0BB6916
:103600009AB2FB88134498B2114B1A6811491346B9
:103610005B0013449B000B4404331A68BB881946B3
:10362000FFF724FEBB690133BB613B8ABA699A424A
:10363000C4D3BB880133BB80FB690133FB617B8A48
:10364000FA699A4284D300BF00BF2037BD4680BDCF
:10365000541600205816002080B586B002AFF860DE
:10366000B9607A603B601E4B4FF440325A601D4B8C
:103670001B681D4A342101FB03F3134448331B68C4
:10368000022B03D1164B02229A6002E0144B002257
:103690009A60134ABB69D360114B144A1A601048F0
:1036A00000F086FF0346002B15D1F9680C4801F0A5
:1036B0001DFA0346002B0ED1BA683B6800937B6865
:1036C000F969074800F0BEFF0346002B03D10A2129
:1036D000034801F011F800BF1037BD4680BD00BFA0
:1036E00014160020541600206C15002000B0024073
:1036F00080B500AF294B2A4A1A602A4B02221A6071
:10370000284B07225A60274B04229A60254B072238
:10371000DA60244B02221A61224B02225A61214BA9
:1037200002229A611D4B00225A601C4B00229A60B3
:103730001A4B0422DA60194B10221A61174B4022EF
:103740005A61164B4FF480729A61144B0022DA6171
:10375000124B4FF400621A62104B4FF480525A62BF
:103760000E4B00229A6200210C4800F089F80D49A6
:103770000A4805F049F90346002B03D00A4B012201
:103780001A7002E0084B00221A7040F2036000F049
:103790000DF8054B1B78184680BD00BFF4160020BD
:1037A000400100A0281700204400002080B584B00C
:1037B00000AF78600023BB602F4B01221A602E4BB4
:1037C00010225A602C4B01229A602B4B0022DA60A7
:1037D0004FF6FF722849294805F04AF90023FB609B
:1037E00003E000BFFB680133FB60FB6842F20F722D
:1037F0009342F6DD204B02221A601F4B10225A60C2
:103800001D4B01229A601C4B0022DA604FF6FF72BA
:1038100019491A4805F02CF9174B03221A60164B68
:1038200010225A60144B08229A60134B0022DA606F
:103830004FF6FF721049114805F01AF94FF408735A
:10384000BB600D4B04221A600B4B10225A600A4BCE
:1038500001229A60BB68084AD3604FF6FF7206499E
:10386000064805F005F97968044805F02CF900BF11
:103870001037BD4680BD00BF44170020F41600205D
:1038800080B590B000AF78603960704B9B6B6F4A29
:1038900043F0010393636D4B9B6B03F00103BB6229
:1038A000BB6A6A4B1B6B694A43F480031363674B23
:1038B0001B6B03F480037B627B6A644B1B6B634A64
:1038C00043F004031363614B1B6B03F004033B627F
:1038D0003B6A5E4B1B6B5D4A43F0080313635B4B13
:1038E0001B6B03F00803FB61FB69584B1B6B574ACA
:1038F00043F010031363554B1B6B03F01003BB61C4
:10390000BB69524B1B6B514A43F0200313634F4B6F
:103910001B6B03F020037B617B694C4B1B6B4B4A99
:1039200043F040031363494B1B6B03F040033B61BF
:103930003B69464B1B6B454A43F080031363434B83
:103940001B6B03F08003FB60FB6802233B630123D6
:103950007B630223BB630C23FB630823FB6207F139
:103960002C0319463A4801F0EFF94CF20373FB625D
:1039700007F12C031946374801F0E6F94FF6837337
:10398000FB6207F12C031946334801F0DDF94FF6CD
:103990003F03FB6207F12C031946304801F0D4F9CC
:1039A00048F23313FB6207F12C0319462C4801F04F
:1039B000CBF92823FB6207F12C031946294801F0B3
:1039C000C3F9294B00225A60274B80229A60264B6C
:1039D0004FF40072DA60244B4FF480621A61224B7C
:1039E0004FF480525A61204B4FF480429A611E4B33
:1039F0000022DA611C4B4FF400321A621A4B00228B
:103A00005A62194B03229A62174B0022DA62164B54
:103A100000221A63144B154A1A607B68124A1A6313
:103A2000114A7B689363104800F0B2FC0E4800F026
:103A300001FC00220F21382000F0C4FB382000F0E8
:103A4000DDFB00BF4037BD4680BD00BF00380240EF
:103A500000080240000C0240001002400014024026
:103A600000180240001C024054170020106402405D
:103A700080B584B000AF03460A46FB801346BB8086
:103A80000023FB73144AFB881380144ABB881380FD
:103A9000134B1B6870209847114B5B687020984748
:103AA0000346512B11D10F4B0D4A1A600E4B702259
:103AB0001A700E4B08221A700A4B1B68DB680A4A00
:103AC000127892B21046984701E00323FB73FB7B08
:103AD00018461037BD4680BDB8170020BA17002021
:103AE0000C000020B4170020BD170020BC170020D8
:103AF00090B597B002AF7860002387F84F3000236D
:103B00003B610023FB600023BB60B44B1B681B6957
:103B1000B34A127892B21046984703461A467B6819
:103B20001A707B681B78002B00F096810023BB6421
:103B300085E1AA4B1B685B69A94A127890B207F12C
:103B40002001BA6C52008C1807F11401BA6C5200B3
:103B50000A4421469847A34B1B78012B17D1BB6C15
:103B60005B0050333B4433F8302CBB6C5B0050336C
:103B70003B4423F8182CBB6C5B0050333B4433F8B8
:103B80003C2CBB6C5B0050333B4423F8242C954BFE
:103B90001B7803F00203002B0ED0BB6C5B0050338C
:103BA0003B4433F8303CC3F580539AB2BB6C5B00A6
:103BB00050333B4423F8182C8A4B1B7803F0040342
:103BC000002B0ED0BB6C5B0050333B4433F83C3CC5
:103BD000C3F580539AB2BB6C5B0050333B4423F86F
:103BE000242C804B1B7803F00803002B17D0BB6CF0
:103BF0005B0050333B4433F8302CBB6C5B005033DC
:103C00003B4423F8242CBB6C5B0050333B4433F81B
:103C10003C2CBB6C5B0050333B4423F8182CBB6C32
:103C20005B0050333B4433F8183C19466E4ABB6C7A
:103C300052F8233099420DD9BB6C5B0050333B44A2
:103C400033F8182C6849BB6C51F823309BB2D31A57
:103C50009BB20CE0644ABB6C52F823309AB2BB6C46
:103C60005B0050333B4433F8183CD31A9BB2A7F89F
:103C70004630BB6C5B0050333B4433F8243C194660
:103C80005A4ABB6C52F8233099420DD9BB6C5B0089
:103C900050333B4433F8242C5449BB6C51F8233047
:103CA0009BB2D31A9BB20CE0504ABB6C52F8233043
:103CB0009AB2BB6C5B0050333B4433F8243CD31ABC
:103CC0009BB2A7F84430B7F84620B7F84430134405
:103CD000052B15DDBB6C5B0050333B4433F8183CBF
:103CE0001946414ABB6C42F82310BB6C5B00503351
:103CF0003B4433F8243C19463C4ABB6C42F8231041
:103D0000374B1B78702B19D1BB6C5B0050333B4495
:103D100033F8181C7A68BB6C5B0013440A465A805F
:103D2000BB6C5B0050333B4433F8241C7A68BB6C9B
:103D300004335B0013440A469A8022E02C4B1B8814
:103D40001946294ABB6C52F8233001FB03F31B0BC5
:103D500099B27A68BB6C5B0013440A465A80254BC3
:103D60001B881946214ABB6C52F8233001FB03F330
:103D70001B0B99B27A68BB6C04335B0013440A4690
:103D80009A80174B1B7898B207F10C0107F11002CB
:103D900007F1080300930B46B96CFEF733FD3B694E
:103DA000D9B27A68BB6C134416330A461A70FB68A2
:103DB000D9B27A68BB6C134420330A461A70BB68C8
:103DC000032B35D801A252F823F000BFF93D0008BB
:103DD000073E0008153E0008233E0008B4170020E7
:103DE000BD170020BC170020C0170020D4170020EA
:103DF000B8170020BA1700207A68BB6C13441B3335
:103E000001221A7018E07A68BB6C13441B3302223B
:103E10001A7011E07A68BB6C13441B3303221A70CA
:103E20000AE07A68BB6C13441B3300221A7003E06B
:103E3000012387F84F3000BFBB6C0133BB647B6844
:103E40001B781A46BB6C9342FFF473AE786800F09F
:103E500009F8034687F84F3097F84F301846543723
:103E6000BD4690BD80B584B000AF78600023BB60D4
:103E70000023FB733B4B1B789BB207F108021146F2
:103E80001846FEF7A6FCBB68492B5ED0492B60D8CC
:103E90001C2B3FD81C2B5CD801A252F823F000BF8A
:103EA0001B3F0008533F0008533F0008533F0008E2
:103EB000533F0008533F0008533F0008533F00089A
:103EC000533F0008533F0008533F0008533F00088A
:103ED000533F0008533F0008533F0008533F00087A
:103EE000233F0008533F0008533F0008533F00089A
:103EF0002B3F0008533F0008533F0008533F000882
:103F0000333F0008533F0008533F0008533F000869
:103F10003B3F0008402B14D01BE07B6800229A62D4
:103F20001AE07B6801229A6216E07B6802229A629C
:103F300012E07B6803229A620EE07B6804229A6298
:103F40000AE07B6805229A6206E07B6806229A6294
:103F500002E00123FB7300BFFB7B18461037BD4610
:103F600080BD00BFBD17002080B500AF032000F06A
:103F70001EF90020FEF730F8FEF706F80023184679
:103F800080BD000080B400AF064B1B781A46064B7C
:103F90001B681344044A136000BFBD465DF8047BF0
:103FA000704700BF4C000020E817002080B400AF2D
:103FB000034B1B681846BD465DF8047B704700BF85
:103FC000E817002080B584B000AF7860FFF7EEFFFF
:103FD000B8607B68FB60FB68B3F1FF3F05D00A4B1C
:103FE0001B781A46FB681344FB6000BFFFF7DEFF37
:103FF0000246BB68D31AFA689A42F7D800BF00BFDE
:104000001037BD4680BD00BF4C00002080B485B095
:1040100000AF78607B6803F00703FB600B4BDB6845
:10402000BB60BA684FF6FF031340BB60FB681A021F
:10403000BB681A43064B1343BB60044ABB68D3609A
:1040400000BF1437BD465DF8047B704700ED00E00B
:104050000000FA0580B400AF044BDB681B0A03F0D4
:1040600007031846BD465DF8047B704700ED00E08D
:1040700080B483B000AF0346FB7197F90730002B83
:104080000BDBFB7903F01F02074997F907305B0947
:10409000012000FA02F241F8232000BF0C37BD4690
:1040A0005DF8047B704700BF00E100E080B483B09E
:1040B00000AF0346FB7197F90730002B12DBFB7949
:1040C00003F01F020A4997F907305B09012000FA43
:1040D00002F2203341F82320BFF34F8F00BFBFF31C
:1040E0006F8F00BF00BF0C37BD465DF8047B704783
:1040F00000E100E080B483B000AF03463960FB719B
:1041000097F90730002B0ADB3B68DAB20C4997F9C4
:1041100007301201D2B20B4483F800230AE03B6857
:10412000DAB20849FB7903F00F03043B1201D2B263
:104130000B441A7600BF0C37BD465DF8047B704710
:1041400000E100E000ED00E080B489B000AFF8606D
:10415000B9607A60FB6803F00703FB61FB69C3F198
:104160000703042B28BF0423BB61FB690433062B20
:1041700002D9FB69033B00E000237B614FF0FF3273
:10418000BB6902FA03F3DA43BB681A407B699A40C1
:104190004FF0FF317B6901FA03F3D9437B680B4091
:1041A000134318462437BD465DF8047B704780B53D
:1041B00082B000AF78607868FFF728FF00BF08374B
:1041C000BD4680BD80B586B000AF0346B9607A6059
:1041D000FB7300237B61FFF73DFF78617A68B96864
:1041E0007869FFF7B1FF024697F90F30114618467C
:1041F000FFF780FF00BF1837BD4680BD80B582B095
:1042000000AF0346FB7197F907301846FFF730FF00
:1042100000BF0837BD4680BD80B582B000AF034601
:10422000FB7197F907301846FFF740FF00BF0837CA
:10423000BD4680BD80B586B000AF786000237B614D
:10424000FFF7B4FE38617B68002B01D1012399E0B0
:104250007B68002283F834207B68022283F83520B3
:104260007B681B681A687B681B6822F001021A6071
:104270000FE0FFF79BFE02463B69D31A052B08D9D6
:104280007B6820225A657B68032283F8352003234C
:1042900078E07B681B681B6803F00103002BE8D102
:1042A0007B681B681B687B617A69384B13407B61B4
:1042B0007B685A687B689B681A437B68DB681A4393
:1042C0007B681B691A437B685B691A437B689B693F
:1042D0001A437B68DB691A437B681B6A13437A695C
:1042E00013437B617B685B6A042B07D17B68DA6AC6
:1042F0007B681B6B13437A6913437B617B681B6884
:104300007A691A607B681B685B697B617B6923F053
:1043100007037B617B685B6A7A6913437B617B6817
:104320005B6A042B17D17B689B6A7A6913437B61B4
:104330007B68DB6A002B0ED0786800F0BDF803467E
:10434000002B08D07B6840225A657B68012283F8E5
:104350003520012316E07B681B687A695A6178680A
:1043600000F074F80346FB607B68DB6D3F229A40E7
:10437000FB689A607B6800225A657B68012283F89B
:104380003520002318461837BD4680BD3F8010F009
:1043900080B584B000AF78607B68002B01D1012329
:1043A00050E07B6893F83530DBB2022B01D1022359
:1043B00048E07B681B681A687B681B6822F0010272
:1043C0001A607B681B6800221A607B681B680022E9
:1043D0005A607B681B6800229A607B681B68002219
:1043E000DA607B681B6800221A617B681B682122E7
:1043F0005A61786800F02AF80346FB607B68DB6D41
:104400003F229A40FB689A607B680022DA637B68EF
:1044100000221A647B6800225A647B6800229A6436
:104420007B680022DA647B6800221A657B680022C0
:104430005A657B68002283F835207B68002283F868
:104440003420002318461037BD4680BD80B485B0A7
:1044500000AF78607B681B68DBB2103B134AA2FB9D
:1044600003231B09FB60124AFB6813441B781A469E
:104470007B68DA65FB68032B08D97B681B681A46E2
:104480000C4B13401A1D7B689A6506E07B681B681D
:104490001A46084B13407A6893657B689B6D1846F3
:1044A0001437BD465DF8047B704700BFABAAAAAACB
:1044B0006CFE080800FCFFFF80B485B000AF786098
:1044C0000023FB737B689B6ABB607B689B69002B46
:1044D0001FD1BB68032B56D801A252F823F000BFAE
:1044E000F144000803450008F1440008874500082E
:1044F0007B68DB6A03F08073002B46D00123FB73DB
:1045000043E07B68DB6AB3F1C07F40D10123FB73DA
:104510003DE07B689B69B3F5005F21D1BB68032B4D
:1045200037D801A252F823F0394500083F4500086A
:1045300039450008514500080123FB7330E07B68D2
:10454000DB6A03F08073002B25D00123FB7322E08C
:104550007B68DB6AB3F1C07F1FD10123FB731CE0D2
:10456000BB68022B03D9BB68032B03D018E00123DF
:10457000FB7315E07B68DB6A03F08073002B0ED0C1
:104580000123FB730BE000BF0AE000BF08E000BF9F
:1045900006E000BF04E000BF02E000BF00E000BF93
:1045A000FB7B18461437BD465DF8047B704700BF9F
:1045B00080B582B000AF78607B68002B01D1012309
:1045C00039E07B6893F83930DBB2002B06D17B6889
:1045D000002283F838207868FCF7CAFE7B68022244
:1045E00083F839207B681B681B6823F440317B68A3
:1045F0005A687B681B680A431A607B681B685B6BA0
:1046000023F007017B689A687B681B680A435A633A
:104610007B681B681A6C0A4B13407A68D1687A6809
:1046200012680B4313647B680022DA637B68012203
:1046300083F83920002318460837BD4680BD00BFE7
:1046400000C0FFFF80B586B002AFF860B9607A6045
:104650003B60FB6893F83830012B01D1022318E04E
:10466000FB68012283F83820FB68022283F8392096
:10467000BB6900933B687A68B968F86800F0C8FACB
:10468000FB681B681A68FB681B6842F001021A602D
:10469000002318461037BD4680BD80B586B002AFF6
:1046A000F860B9607A603B60FB6893F83830012BA2
:1046B00001D102231CE0FB68012283F83820FB684B
:1046C000022283F83920FB681B687A685A61FB690B
:1046D0000093BB693A68B968F86800F099FAFB681A
:1046E0001B681A68FB681B6842F001021A6000230D
:1046F00018461037BD4680BD80B586B000AF7860E3
:1047000039600023FB607B681B681B6803F00103B2
:10471000002B56D0FFF74AFC78614BE07B681B68A2
:104720005B68FB60FB6803F02103002B23D0FB6870
:1047300003F02003002B05D07B68DB6B43F0020203
:104740007B68DA63FB6803F00103002B05D07B680C
:10475000DB6B43F001027B68DA637B681B68212214
:104760009A607B68042283F839207B68002283F8F2
:1047700038200123A5E03B68B3F1FF3F1AD0FFF7D3
:1047800015FC02467B69D31A3A689A4202D33B6809
:10479000002B0FD17B68DB6B43F020027B68DA6370
:1047A0007B68032283F839207B68002283F8382055
:1047B000032386E07B681B685B6803F00203002B21
:1047C000ACD07B681B68DB6903F020033B617B682E
:1047D0001B685B6A03F020033A6913433B613B6942
:1047E000002B61D0FFF7E2FB786156E07B681B6825
:1047F0005B68FB60FB6803F02903002B2ED0FB688D
:1048000003F00803002B05D07B68DB6B43F0040248
:104810007B68DA63FB6803F02003002B05D07B681C
:10482000DB6B43F002027B68DA63FB6803F0010391
:10483000002B05D07B68DB6B43F001027B68DA63F9
:104840007B681B6829229A607B68042283F83920E0
:104850007B68002283F83820012332E03B68B3F103
:10486000FF3F1AD0FFF7A2FB02467B69D31A3A68D2
:104870009A4202D33B68002B0FD17B68DB6B43F07D
:1048800020027B68DA637B68032283F839207B6827
:10489000002283F83820032313E07B681B685B68E1
:1048A00003F01003002BA1D07B681B6812229A60D2
:1048B0007B68012283F839207B68002283F8382046
:1048C000002318461837BD4680BD80B584B000AFC0
:1048D00078607B681B685B68FB607B681B681B6893
:1048E000BB60FB6803F00103002B26D0BB6803F418
:1048F0008073002B21D07B681B681A687B681B685B
:1049000022F480721A607B68DB6B43F001027B68E3
:10491000DA637B681B6801229A607B68042283F853
:1049200039207B68002283F838207B685B69002B84
:1049300003D07B685B6978689847FB6803F02003C5
:10494000002B26D0BB6803F40053002B21D07B68DA
:104950001B681A687B681B6822F400521A607B6827
:104960001B6820229A607B68DB6B43F002027B6845
:10497000DA637B68042283F839207B68002283F89D
:1049800038207B685B69002B03D07B685B697868A3
:104990009847FB6803F00803002B26D0BB6803F49C
:1049A0000063002B21D07B681B681A687B681B683A
:1049B00022F400621A607B681B6808229A607B6898
:1049C000DB6B43F004027B68DA637B68042283F8C4
:1049D00039207B68002283F838207B685B69002BD4
:1049E00003D07B685B6978689847FB6803F0040331
:1049F000002B13D0BB6803F48063002B0ED07B68C0
:104A00001B681A687B681B6822F480621A607B68E6
:104A10001B6804229A60786800F053F8FB6803F082
:104A20000203002B24D0BB6803F40073002B1FD0BB
:104A30007B681B681A687B681B6822F400721A6026
:104A40007B681B6802229A607B68DA6B7B68DA639A
:104A50007B68012283F839207B68002283F83820A4
:104A60007B681B69002B03D07B681B6978689847BB
:104A7000FB6803F01003002B1FD0BB6803F48053C6
:104A8000002B1AD07B681B681A687B681B6822F4AD
:104A900080521A607B681B6810229A607B68DA6B10
:104AA0007B68DA637B68012283F839207B68002207
:104AB00083F83820786800F00EF800BF1037BD4644
:104AC00080BD80B483B000AF786000BF0C37BD46B6
:104AD0005DF8047B704780B483B000AF786000BF9E
:104AE0000C37BD465DF8047B7047000080B487B08A
:104AF00000AF786039607B685B68B3F5403F7B68E6
:104B000093F83830012B01D1022379E07B68012230
:104B100083F838207B68022283F839203B681B0128
:104B200018337A6813443B613B695A683B699B6858
:104B30001B0413437B61354BFB603B695B680A2BAD
:104B400003D03B695B68092B07D13B69DB6803F045
:104B50007F437A6913437B6105E03B69DB681B0691
:104B60007A6913437B613B68002B20D17B681B680B
:104B70005A6AFB68DB4302EA03017B681B687A69B7
:104B80000A435A627B681B683A6912689A613B69FA
:104B90005B680A2B03D03B695B68092B27D13B6913
:104BA000DA687B681B6822F07F429A621FE07B68AC
:104BB0001B68DA69FB68DB4302EA03017B681B6858
:104BC0007A690A43DA617B681B683A6912681A617C
:104BD0003B695B680A2B03D03B695B68092B06D1F4
:104BE0003B69DA687B681B6822F07F421A627B6847
:104BF000012283F839207B68002283F838200023C3
:104C000018461C37BD465DF8047B70470F0003FF54
:104C100080B48BB000AFF860B9607A603B60FB682D
:104C20001B685B6C03F040413B681A043B6B1A4302
:104C3000FB681B680A435A64FB681B687A68DA637E
:104C4000FB685B68B3F5403F74D1BB6803F07F43FA
:104C50003B62BB6803F47F03FB61BB6803F47F43E3
:104C6000BB61BB68DBB27B61FB689B68002B08D132
:104C7000BA69FB691A433B6A13437A6913437B623F
:104C800053E0FB689B68012B06D1BA69FB691343AB
:104C90007A6913437B6248E0FB689B68022B11D161
:104CA000FB69DB0CFB61BB699B0ABB617B69DB08B1
:104CB0007B61BB695A01FB69DB0213437A691343C9
:104CC0007B6232E0FB689B68032B17D13B6ADB0FEA
:104CD0003B62FB69DB0CFB61BB69DB0ABB617B6987
:104CE000DB087B61BB695A01FB699B021A433B6A83
:104CF000DB0313437A6913437B6216E03B6A1B0FA5
:104D00003B62FB691B0DFB61BB691B0BBB617B69D4
:104D10001B097B61BB691A01FB691B021A433B6AD1
:104D20001B0313437A6913437B62FB681B687A6A2F
:104D30009A6303E0FB681B68BA68DA6000BF2C372F
:104D4000BD465DF8047B704780B489B000AF7860E1
:104D500039600023FB6100237B6100233B6100235A
:104D6000BB610023FB6175E10122FB6902FA03F3D9
:104D70007B613B681B687A6913403B613A697B69D8
:104D80009A4240F064813B685B68012B0BD03B6822
:104D90005B68022B07D03B685B68112B03D03B6834
:104DA0005B68122B30D17B689B68BB61FB695B0041
:104DB000032202FA03F3DB43BA691340BB613B6889
:104DC000DA68FB695B0002FA03F3BA691343BB615B
:104DD0007B68BA699A607B685B68BB610122FB698A
:104DE00002FA03F3DB43BA691340BB613B685B68BB
:104DF0001B0903F00102FB6902FA03F3BA691343CA
:104E0000BB617B68BA695A607B68DB68BB61FB6920
:104E10005B00032202FA03F3DB43BA691340BB6170
:104E20003B689A68FB695B0002FA03F3BA691343B3
:104E3000BB617B68BA69DA603B685B68022B03D0B0
:104E40003B685B68122B23D1FB69DA087B68083268
:104E500053F82230BB61FB6903F007039B000F226C
:104E600002FA03F3DB43BA691340BB613B681A697A
:104E7000FB6903F007039B0002FA03F3BA691343CB
:104E8000BB61FB69DA087B680832B96943F8221014
:104E90007B681B68BB61FB695B00032202FA03F3BA
:104EA000DB43BA691340BB613B685B6803F00302F4
:104EB000FB695B0002FA03F3BA691343BB617B68C9
:104EC000BA691A603B685B6803F08053002B00F0FE
:104ED000BE80664B5B6C654A43F480435364634B0E
:104EE0005B6C03F48043FB60FB68614AFB699B08D1
:104EF000023352F82330BB61FB6903F003039B00CC
:104F00000F2202FA03F3DB43BA691340BB617B68EB
:104F1000584A934237D07B68574A934231D07B68D6
:104F2000564A93422BD07B68554A934225D07B68E2
:104F3000544A93421FD07B68534A934219D07B68EE
:104F4000524A934213D07B68514A93420DD07B68FA
:104F5000504A934207D07B684F4A934201D10923BC
:104F600012E00A2310E008230EE007230CE00623DA
:104F70000AE0052308E0042306E0032304E00223FB
:104F800002E0012300E00023FA6902F0030292002C
:104F90009340BA691343BB613549FB699B080233EF
:104FA000BA6941F823203D4B1B68BB613B69DB4379
:104FB000BA691340BB613B685B6803F48033002B24
:104FC00003D0BA693B691343BB61344ABB691360C0
:104FD000324B5B68BB613B69DB43BA691340BB6121
:104FE0003B685B6803F40033002B03D0BA693B696C
:104FF0001343BB61294ABB695360284B9B68BB6163
:105000003B69DB43BA691340BB613B685B6803F4EF
:105010008013002B03D0BA693B691343BB611F4A5D
:10502000BB6993601D4BDB68BB613B69DB43BA69BD
:105030001340BB613B685B6803F40013002B03D093
:10504000BA693B691343BB61144ABB69D360FB690E
:105050000133FB61FB690F2B7FF686AE00BF00BFFB
:105060002437BD465DF8047B704700BF003802401E
:1050700000380140000002400004024000080240E5
:10508000000C0240001002400014024000180240D0
:10509000001C02400020024000240240003C01406D
:1050A00080B487B000AF7860396000233B61002393
:1050B000FB600023BB6000237B61D9E001227B6998
:1050C00002FA03F33B613A683B691340FB60FA68FC
:1050D0003B699A4240F0C9806B4A7B699B08023366
:1050E00052F82330BB607B6903F003039B000F225F
:1050F00002FA03F3BA681340BB607B68634A9342C9
:1051000037D07B68624A934231D07B68614A9342D0
:105110002BD07B68604A934225D07B685F4A9342DC
:105120001FD07B685E4A934219D07B685D4A9342E8
:1051300013D07B685C4A93420DD07B685B4A9342F4
:1051400007D07B685A4A934201D1092312E00A230F
:1051500010E008230EE007230CE006230AE00523F5
:1051600008E0042306E0032304E0022302E0012315
:1051700000E000237A6902F0030292009340BA68CB
:105180009A4232D14B4B1A68FB68DB4349491340C2
:105190000B60484B5A68FB68DB43464913404B6041
:1051A000444B9A68FB68DB43424913408B60414B98
:1051B000DA68FB68DB433F491340CB607B6903F04F
:1051C00003039B000F2202FA03F3BB602E4A7B69A4
:1051D0009B08023352F82310BB68DA432A487B69E4
:1051E0009B080A40023340F823207B681A687B69D9
:1051F0005B00032101FA03F3DB431A407B681A606A
:105200007B69DA087B68083253F822107B6903F067
:1052100007039B000F2202FA03F3DB437A69D208EB
:1052200019407B68083243F822107B68DA687B6992
:105230005B00032101FA03F3DB431A407B68DA6069
:105240007B685A6801217B6901FA03F3DB431A404A
:105250007B685A607B689A687B695B00032101FA6E
:1052600003F3DB431A407B689A607B6901337B61FF
:105270007B690F2B7FF622AF00BF00BF1C37BD46F6
:105280005DF8047B704700BF003801400000024019
:105290000004024000080240000C024000100240DE
:1052A0000014024000180240001C0240002002408E
:1052B00000240240003C014080B483B000AF78601D
:1052C0000B467B8013467B707B78002B03D07A885B
:1052D0007B689A6103E07B881A047B689A6100BF4F
:1052E0000C37BD465DF8047B7047000080B582B086
:1052F00000AF78607B68002B01D101237FE07B68E1
:1053000093F84130DBB2002B06D17B68002283F892
:1053100040207868FCF750FB7B68242283F841200A
:105320007B681B681A687B681B6822F001021A60A0
:105330007B685A687B681B6822F070621A617B6820
:105340001B689A687B681B6822F400429A607B683D
:10535000DB68012B07D17B689A687B681B6842F485
:1053600000429A6006E07B689A687B681B6842F49A
:1053700004429A607B68DB68022B04D17B681B685F
:105380004FF400625A607B681B6859687B681A6832
:105390001D4B0B4353607B681B68DA687B681B6896
:1053A00022F40042DA607B681A697B685B6942EA32
:1053B00003017B689B691A027B681B680A43DA60F9
:1053C0007B68D9697B681A6A7B681B680A431A6024
:1053D0007B681B681A687B681B6842F001021A60D0
:1053E0007B6800225A647B68202283F841207B6816
:1053F00000221A637B68002283F8422000231846AB
:105400000837BD4680BD00BF0080000280B582B075
:1054100000AF78607B68002B01D1012321E07B681D
:10542000242283F841207B681B681A687B681B680C
:1054300022F001021A607868FCF726FB7B680022E4
:105440005A647B68002283F841207B6800221A633B
:105450007B68002283F842207B68002283F840208A
:10546000002318460837BD4680BD000080B588B0CF
:1054700002AFF860084611461A4603467B810B4688
:105480003B811346FB80FB6893F84130DBB2202B55
:1054900040F0F9803B6A002B02D0BB8C002B05D179
:1054A000FB684FF400725A640123EDE0FB6893F847
:1054B0004030012B01D10223E6E0FB68012283F892
:1054C0004020FEF773FD78617B6900931923012268
:1054D0004FF40041F86800F0EBFA0346002B01D0CE
:1054E0000123D1E0FB68212283F84120FB684022A0
:1054F00083F84220FB6800225A64FB683A6A5A62C9
:10550000FB68BA8C5A85FB6800225A63F8883A898E
:1055100079897B690193BB6A00930346F86800F0C0
:10552000FBF90346002B05D0FB68002283F84020DE
:105530000123A9E0FB685B8D9BB2FF2B0ED9FB68B2
:10554000FF221A85FB681B8DDAB27989002300934C
:105550004FF08073F86800F0CDFB0FE0FB685B8DC7
:105560009AB2FB681A85FB681B8DDAB27989002331
:1055700000934FF00073F86800F0BCFB7A69B96AD9
:10558000F86800F0D5FA0346002B01D001237BE038
:10559000FB685B6A1A78FB681B689A62FB685B6A47
:1055A0005A1CFB685A62FB685B8D9BB2013B9AB246
:1055B000FB685A85FB681B8D013B9AB2FB681A8514
:1055C000FB685B8D9BB2002B34D0FB681B8D002BDE
:1055D00030D17B690093BB6A00228021F86800F01B
:1055E00067FA0346002B01D001234DE0FB685B8D79
:1055F0009BB2FF2B0ED9FB68FF221A85FB681B8D1F
:10560000DAB27989002300934FF08073F86800F0D4
:1056100071FB0FE0FB685B8D9AB2FB681A85FB6833
:105620001B8DDAB27989002300934FF00073F8687C
:1056300000F060FBFB685B8D9BB2002B9ED17A690A
:10564000B96AF86800F0B4FA0346002B01D00123D0
:105650001AE0FB681B682022DA61FB681B68596846
:10566000FB681A680A4B0B405360FB68202283F8E2
:105670004120FB68002283F84220FB68002283F867
:105680004020002300E0022318461837BD4680BDA5
:1056900000E800FE80B588B002AFF8600846114609
:1056A0001A4603467B810B463B811346FB80FB6811
:1056B00093F84130DBB2202B40F0FD803B6A002B99
:1056C00002D0BB8C002B05D1FB684FF400725A64EA
:1056D0000123F1E0FB6893F84030012B01D1022354
:1056E000EAE0FB68012283F84020FEF75FFC786166
:1056F0007B690093192301224FF40041F86800F000
:10570000D7F90346002B01D00123D5E0FB68222204
:1057100083F84120FB68402283F84220FB68002286
:105720005A64FB683A6A5A62FB68BA8C5A85FB680D
:1057300000225A63F8883A8979897B690193BB6AA8
:1057400000930346F86800F03BF90346002B05D0B0
:10575000FB68002283F840200123ADE0FB685B8DED
:105760009BB2FF2B0ED9FB68FF221A85FB681B8DAD
:10577000DAB27989524B00934FF08073F86800F0E9
:10578000B9FA0FE0FB685B8D9AB2FB681A85FB687B
:105790001B8DDAB279894A4B00934FF00073F86899
:1057A00000F0A8FA7B690093BB6A00220421F86824
:1057B00000F07EF90346002B01D001237CE0FB685A
:1057C0001B685A6AFB685B6AD2B21A70FB685B6A34
:1057D0005A1CFB685A62FB681B8D013B9AB2FB683E
:1057E0001A85FB685B8D9BB2013B9AB2FB685A85B8
:1057F000FB685B8D9BB2002B34D0FB681B8D002BAC
:1058000030D17B690093BB6A00228021F86800F0E8
:105810004FF90346002B01D001234DE0FB685B8D5F
:105820009BB2FF2B0ED9FB68FF221A85FB681B8DEC
:10583000DAB27989002300934FF08073F86800F0A2
:1058400059FA0FE0FB685B8D9AB2FB681A85FB681A
:105850001B8DDAB27989002300934FF00073F8684A
:1058600000F048FAFB685B8D9BB2002B9AD17A69F5
:10587000B96AF86800F09CF90346002B01D00123B7
:105880001AE0FB681B682022DA61FB681B68596814
:10589000FB681A680B4B0B405360FB68202283F8AF
:1058A0004120FB68002283F84220FB68002283F835
:1058B0004020002300E0022318461837BD4680BD73
:1058C0000024008000E800FE80B584B000AF78605E
:1058D0007B681B689B69FB607B681B681B68BB60FF
:1058E0007B685B6B002B05D07B685B6BBA68F968E3
:1058F0007868984700BF1037BD4680BD80B483B03C
:1059000000AF78607B6893F84130DBB218460C3703
:10591000BD465DF8047B704780B586B002AFF86085
:10592000084611461A4603467B810B463B811346C7
:10593000FB80FB88DAB27989204B00934FF08073AB
:10594000F86800F0D7F9FA69B969F86800F0F0F87A
:105950000346002B01D001232CE0FB88012B05D14D
:105960003B89DAB2FB681B689A6215E03B891B0A27
:105970009BB2DAB2FB681B689A62FA69B969F86887
:1059800000F0D6F80346002B01D0012312E03B893A
:10599000DAB2FB681B689A62FB690093BB6900225C
:1059A0008021F86800F084F80346002B01D0012321
:1059B00000E0002318461037BD4680BD002000805F
:1059C00080B586B002AFF860084611461A46034615
:1059D0007B810B463B811346FB80FB88DAB27989D9
:1059E000204B00930023F86800F084F9FA69B96944
:1059F000F86800F09DF80346002B01D001232CE04D
:105A0000FB88012B05D13B89DAB2FB681B689A62DF
:105A100015E03B891B0A9BB2DAB2FB681B689A62ED
:105A2000FA69B969F86800F083F80346002B01D0E1
:105A3000012312E03B89DAB2FB681B689A62FB69BA
:105A40000093BB6900224021F86800F031F803465A
:105A5000002B01D0012300E0002318461037BD467B
:105A600080BD00BF0020008080B483B000AF7860AC
:105A70007B681B689B6903F00203022B03D17B68E0
:105A80001B6800229A627B681B689B6903F0010314
:105A9000012B07D07B681B689A697B681B6842F002
:105AA00001029A6100BF0C37BD465DF8047B704768
:105AB00080B584B000AFF860B9603B601346FB71FD
:105AC00022E03B68B3F1FF3F1ED0FEF76FFA0246BB
:105AD000BB69D31A3A689A4202D33B68002B13D1B0
:105AE000FB685B6C43F02002FB685A64FB68202271
:105AF00083F84120FB68002283F84220FB680022E3
:105B000083F8402001230FE0FB681B689A69BB689B
:105B10001340BA689A420CBF01230023DBB21A4635
:105B2000FB799A42CDD0002318461037BD4680BD80
:105B300080B584B000AFF860B9607A602CE07A6814
:105B4000B968F86800F070F80346002B01D0012313
:105B50002AE0BB68B3F1FF3F1ED0FEF727FA0246EA
:105B60007B68D31ABA689A4202D3BB68002B13D160
:105B7000FB685B6C43F02002FB685A64FB682022E0
:105B800083F84120FB68002283F84220FB68002252
:105B900083F84020012307E0FB681B689B6903F042
:105BA0000203022BCBD1002318461037BD4680BD1F
:105BB00080B584B000AFF860B9607A6028E07A6898
:105BC000B968F86800F030F80346002B01D00123D3
:105BD00026E0FEF7EBF902467B68D31ABA689A42D0
:105BE00002D3BB68002B13D1FB685B6C43F020022F
:105BF000FB685A64FB68202283F84120FB6800227E
:105C000083F84220FB68002283F84020012307E04C
:105C1000FB681B689B6903F02003202BCFD1002376
:105C200018461037BD4680BD80B584B000AFF8601F
:105C3000B9607A60FB681B689B6903F01003102B46
:105C400051D122E0BB68B3F1FF3F1ED0FEF7AEF9A1
:105C500002467B68D31ABA689A4202D3BB68002B0B
:105C600013D1FB685B6C43F02002FB685A64FB684D
:105C7000202283F84120FB68002283F84220FB6841
:105C8000002283F8402001232EE0FB681B689B69FB
:105C900003F02003202BD5D1FB681B681022DA61AA
:105CA000FB681B682022DA61F868FFF7DDFEFB68FD
:105CB0001B685968FB681A680D4B0B405360FB6802
:105CC0005B6C43F00402FB685A64FB68202283F893
:105CD0004120FB68002283F84220FB68002283F801
:105CE0004020012300E0002318461037BD4680BD48
:105CF00000E800FE80B485B000AFF8607B600B4622
:105D00007B8113467B72FB681B685A68BB695B0D1D
:105D100003F480610D4B0B43DB4302EA03017B89F3
:105D2000C3F309027B7A1B0403F47F031A437B68E5
:105D30001A43BB691A43FB681B680A435A6000BFD9
:105D40001437BD465DF8047B704700BFFF63FF0357
:105D500080B584B000AF78607B68002B01D101234F
:105D6000BFE07B6893F8A130DBB2002B06D17B68E3
:105D7000002283F8A0207868FBF7ACFE7B68022243
:105D800083F8A1207B681B689A697B681B6822F0F6
:105D900070429A617B681B6899697B685A687B6866
:105DA0009B681A437B68DB681A437B681B691A434C
:105DB0007B681B680A439A617B681B6899687B68EB
:105DC0001A684A4B0B4093607B685B691B04FB605D
:105DD0007B681B6899687B689A69FB681A437B68D3
:105DE0001B680A439A607B681B68D9687B681A68DD
:105DF0003E4B0B40D3607B68DB691B04FB607B6818
:105E00001B68D9687B681A6AFB681A437B681B6841
:105E10000A43DA607B681B6819697B681A68334B30
:105E20000B4013617B685B6A1B04FB607B681B682B
:105E300019697B689A6AFB681A437B681B680A4386
:105E40001A617B681B6859697B681A68274B0B408D
:105E500053617B68DB6A1B04FB607B681B685969C4
:105E60007B681A6BFB681A437B681B680A435A619C
:105E70007B6893F835301B02FB607B6893F8363003
:105E80001B04BB607B681B68DA6A7B681B6802F0D6
:105E90007F42DA627B681B68D96ABA68FB68134381
:105EA0007A6892F834201A437B681B680A43DA62E6
:105EB0007B681B685A6B7B681B6842F006025A635A
:105EC0007B681B689A697B681B6842F001029A61D3
:105ED0007B680022C3F8A4207B68012283F8A120FC
:105EE000002318461037BD4680BD00BF00F800F003
:105EF00080B584B000AF78607B681B689B6BFB60EB
:105F00007B681B685B6BBB60FB6803F00403002BC2
:105F100023D0BB6803F00403002B1ED07B681B68F2
:105F20005A6B7B681B6822F004025A637B681B680B
:105F30000422DA637B68D3F8A43043F001027B6863
:105F4000C3F8A4207B68042283F8A1207B68002288
:105F500083F8A020786800F06FF8FB6803F0020374
:105F6000002B23D0BB6803F00203002B1ED07B68FC
:105F70001B685A6B7B681B6822F002025A637B68BD
:105F80001B680222DA637B68D3F8A43043F0020274
:105F90007B68C3F8A4207B68042283F8A1207B6877
:105FA000002283F8A020786800F046F8FB6803F030
:105FB0000103002B1BD0BB6803F00103002B16D09C
:105FC0007B681B685A6B7B681B6822F001025A636E
:105FD0007B681B680122DA637B68012283F8A120B9
:105FE0007B68002283F8A02078685BF00DFFFB68D7
:105FF00003F00803002B1BD0BB6803F00803002B41
:1060000016D07B681B685A6B7B681B6822F00802FD
:106010005A637B681B680822DA637B68012283F875
:10602000A1207B68002283F8A020786800F00EF899
:1060300000BF1037BD4680BD80B483B000AF78602C
:1060400000BF0C37BD465DF8047B704780B483B059
:1060500000AF786000BF0C37BD465DF8047B704729
:10606000B0B584B000AFF860B9607A60FB6893F8AF
:10607000A030012B01D102232CE0FB68012283F820
:10608000A020FB68022283F8A120FA687B683421F3
:1060900001FB03F3134403F13802BB6814461D46A9
:1060A0000FCD0FC40FCD0FC40FCD0FC42B682360CD
:1060B0007A68B968F86800F057F8FB681B68012235
:1060C0005A62FB68012283F8A120FB68002283F852
:1060D000A020002318461037BD46B0BD80B483B061
:1060E00000AF786039607B6893F8A030012B01D154
:1060F000022323E07B68012283F8A0207B68022230
:1061000083F8A1207B681B685A6B7B681B6822F0B0
:1061100001025A630C4A3B6813647B681B685A6B24
:106120007B681B6842F001025A637B68012283F896
:10613000A1207B68002283F8A020002318460C379A
:10614000BD465DF8047B70470068014080B483B0B1
:1061500000AF78607B6893F8A130DBB218460C374B
:10616000BD465DF8047B704780B489B000AFF8602D
:10617000B9607A60BB685A68FB681B68DB681B0CF7
:10618000C3F30B0313441B04FB61FB681B681A4633
:106190007B68DB01134484335B68FA68126811463C
:1061A0007A68D2010A44843203F470435360BB68B6
:1061B0001A68FB681B68DB681B0CC3F30B031344F2
:1061C0005A1CFB681B6819467B68DB010B4484334F
:1061D0001946FB6913434B60BB68DA68FB681B68B0
:1061E000DB68C3F30A0313441B04FB61FB681B68F1
:1061F0001A467B68DB01134484339B68FA68126893
:1062000011467A68D2010A44843203F470439360E1
:10621000BB689A68FB681B68DB68C3F30A03134416
:106220005A1CFB681B6819467B68DB010B448433EE
:106230001946FB6913438B60FB681B681A467B6831
:10624000DB01134484331B69FA68126811467A68CB
:10625000D2010A44843223F007031361FB681B68F0
:106260001A467B68DB01134484331A46BB681B69FA
:106270001361BB6893F831301B02FB61BB6893F874
:1062800032301B04BB61BB689B691B067B61FB68EA
:106290001B681A467B68DB01134484339B69FB68E7
:1062A0001B681A467B68DB01134484331A460023BB
:1062B0009361BB6893F830301A46FB691A43BB6997
:1062C0001A43FB681B6819467B68DB010B44843367
:1062D00019467B6913438B61FB681B681A467B6810
:1062E000DB01134484335B69FA68126811467A68EB
:1062F000D2010A44843223F0FF035361FB681B6818
:106300001A467B68DB01134484331A46BB685B6919
:106310005361FB681B681A467B68DB0113448433B6
:10632000DA69FB681B6819467B68DB010B44843320
:106330001946584B1340CB61BB68DA69BB681B6ACE
:10634000F968096808467968C90101448431134332
:10635000CB61FB681B681A467B68DB0113448433FE
:106360009B6AFB681B681A467B68DB011344843315
:106370001A4600239362FB681B681A467B68DB01A0
:10638000134484331A46BB685B6A9362BB681B691B
:10639000002B02D10423FB611BE0BB681B69012BAE
:1063A00002D10323FB6114E0BB681B69042B0BD0F3
:1063B000BB681B69022B07D0BB681B69032B03D08A
:1063C000BB681B69072B02D10223FB6101E001239B
:1063D000FB61FB681B681A467B68DB01134484334E
:1063E000DB6AFA68126811467A68D2010A4484327C
:1063F00003F0E023D362BB689B6AFA6902FB03F3F4
:106400001A04BB685968BB681B68CB1AF96901FBA1
:1064100003F30333F968096808467968C901014440
:1064200084311343CB62FB681B681A467B68DB012F
:10643000134484331A6BFB681B6819467B68DB01C5
:106440000B4484331946144B13400B63FB681B68E1
:106450001A467B68DB01134484331A46BB68DB6A47
:106460001363FB681B681A467B68DB0113448433A3
:106470001B68FA68126811467A68D2010A448432AD
:1064800043F00103136000BF2437BD465DF8047B71
:10649000704700BFF8F8FFFF00F8FFFFF0B58FB0BE
:1064A0000AAF78607B68002B01D1012316E17B687D
:1064B0001B68BB607B6893F8BD33DBB2002B06D151
:1064C0007B68002283F8BC2378685DF0E1FC7B6880
:1064D000032283F8BD23BB68DB6B03F48073002BBE
:1064E00002D17B6800221A617B681B68184602F0A3
:1064F00096FF7B681B683B607E686D4606F1100462
:106500000FCC0FC50FCC0FC594E8030085E803003E
:10651000331D0ECB386802F077FE0346002B05D002
:106520007B68022283F8BD230123D7E07B681B68C8
:106530000021184602F084FF0023FB734AE0FA7B37
:1065400079681346DB009B1A9B000B443D33012204
:106550001A70FA7B79681346DB009B1A9B000B4488
:106560003C33FA7B1A70FA7BFB7B98B2796813464E
:10657000DB009B1A9B000B44423302461A80FA7BD5
:1065800079681346DB009B1A9B000B443F330022C3
:106590001A70FA7B79681346DB009B1A9B000B4448
:1065A000443300221A60FA7B79681346DB009B1A99
:1065B0009B000B44483300221A60FA7B796813462B
:1065C000DB009B1A9B000B44503300221A60FB7BBC
:1065D0000133FB73FA7B7B685B689A42AFD300237D
:1065E000FB7344E0FA7B79681346DB009B1A9B003F
:1065F0000B4403F2FD1300221A70FA7B79681346EC
:10660000DB009B1A9B000B4403F5FE73FA7B1A70A8
:10661000FA7B79681346DB009B1A9B000B4403F25C
:10662000FF1300221A70FA7B79681346DB009B1A6D
:106630009B000B4403F5017300221A60FA7B796812
:106640001346DB009B1A9B000B4403F502730022E8
:106650001A60FA7B79681346DB009B1A9B000B4497
:1066600003F5047300221A60FB7B0133FB73FA7B92
:106670007B685B689A42B5D37B681B683B607E6829
:106680006D4606F110040FCC0FC50FCC0FC594E872
:10669000030085E80300331D0ECB386802F0FAFED4
:1066A0000346002B05D07B68022283F8BD2301231B
:1066B00014E07B68002283F838207B68012283F88D
:1066C000BD237B685B6A012B02D1786801F080F8FA
:1066D0007B681B68184603F049FF002318461437EF
:1066E000BD46F0BD80B582B000AF78607B6893F89E
:1066F000BC33012B01D1022312E07B68012283F815
:10670000BC237B681B68184603F018FF7B681B6876
:10671000184602F073FE7B68002283F8BC23002336
:1067200018460837BD4680BD90B58DB000AF786083
:106730007B681B683B623B6AFB617B681B68184691
:1067400003F0BFFF0346002B40F0CA837B681B6841
:10675000184603F023FF0346002B00F0C0837B683C
:106760001B68184603F01AFF034603F00203022BCE
:1067700007D17B681B685A697B681B6802F00202BC
:106780005A617B681B68184603F008FF034603F054
:106790001003102B61D17B681B689A697B681B68AA
:1067A00022F010029A613B6A1B6ABB61BB6903F06D
:1067B0000F021346DB009B1A9B0003F5FC737A68FB
:1067C000134404337B61BB695B0C03F00F03022BA2
:1067D00024D1BA6947F6F0731340002B35D07B699A
:1067E000D968BB691B099BB2C3F30A039BB21A4663
:1067F000386A03F080FD7B69DA68BB691B09C3F363
:106800000A031A447B69DA607B699A69BB691B09D0
:10681000C3F30A031A447B699A6116E0BB695B0CF7
:1068200003F00F03062B10D17B6803F57173082268
:106830001946386A03F05FFD7B699A69BB691B09D9
:10684000C3F30A031A447B699A617B681B689A69DF
:106850007B681B6842F010029A617B681B681846CF
:1068600003F09CFE034603F40023B3F5002F6ED122
:1068700000237B627B681B68184603F0A2FEB862A7
:1068800062E0BB6A03F00103002B57D07B681B68F2
:106890007A6AD2B21146184603F0C7FE38613B69E6
:1068A00003F00103002B0CD07B6A5A01FB691344EF
:1068B00003F530631A4601239360796A786800F023
:1068C000DDFD3B6903F00803002B0CD07B6A5A0105
:1068D000FB69134403F530631A4608239360796A11
:1068E000786800F0D7FE3B6903F01003002B08D056
:1068F0007B6A5A01FB69134403F530631A4610237F
:1069000093603B6903F02003002B08D07B6A5A0197
:10691000FB69134403F530631A46202393603B69F7
:1069200003F40053002B09D07B6A5A01FB6913441E
:1069300003F530631A464FF4005393607B6A0133CA
:106940007B62BB6A5B08BB62BB6A002B99D17B6828
:106950001B68184603F022FE034603F48023B3F5B8
:10696000802F40F0C0807B681B68184603F043FE10
:10697000B86200237B62B2E0BB6A03F00103002B24
:1069800000F0A7807B681B687A6AD2B2114618466D
:1069900003F069FE38613B6903F00103002B57D017
:1069A0007B6A03F00F03012202FA03F3FB60FB6929
:1069B00003F500635A6BFB68DB43F96901F500617D
:1069C00013404B637B6A5A01FB69134403F5106360
:1069D0001A46012393607B681B69012B32D17968C9
:1069E0007A6A1346DB009B1A9B000B4448331968F4
:1069F00078687A6A1346DB009B1A9B000344443391
:106A00001B68194478687A6A1346DB009B1A9B005E
:106A10000344483319607B6A002B13D179687A6A82
:106A20001346DB009B1A9B000B4450331B68002B62
:106A300008D17B6818687B6803F571731A460121D9
:106A400003F072FE7B6ADBB2194678685DF0B1FA3A
:106A50003B6903F00803002B08D07B6A5A01FB69ED
:106A6000134403F510631A46082393603B6903F04F
:106A70001003002B08D07B6A5A01FB69134403F50D
:106A800010631A46102393603B6903F04003002B08
:106A900008D07B6A5A01FB69134403F510631A4658
:106AA000402393603B6903F00203002B08D07B6A0C
:106AB0005A01FB69134403F510631A4602239360DD
:106AC0003B6903F08003002B03D0796A786800F0FB
:106AD00048FC7B6A01337B62BB6A5B08BB62BB6AB2
:106AE000002B7FF449AF7B681B68184603F056FD06
:106AF000034603F00043B3F1004F22D1FB6903F5D5
:106B000000635B68FA6902F5006223F001035360D9
:106B10007B6893F8F433012B08D17B68002283F85B
:106B2000F423002178685DF093FC02E078685DF062
:106B3000B7FA7B681B685A697B681B6802F00042E1
:106B40005A617B681B68184603F028FD034603F46E
:106B50000063B3F5006F12D1FB6903F500639B6816
:106B600003F00103012B02D178685DF073FA7B68B2
:106B70001B685A697B681B6802F400625A617B6873
:106B80001B68184603F00AFD034603F00063B3F1E7
:106B9000006F21D17B681B685A697B681B6802F013
:106BA00000625A617B6893F8F433002B11D17B6843
:106BB000012283F8F4237B681B685B6D9B0803F05C
:106BC0000F027B68C3F8F823012178685DF040FC70
:106BD00002E078685DF03EFA7B681B68184603F0B7
:106BE000DDFC034603F48053B3F5805F40F0C780BB
:106BF000FB6903F500635B68FA6902F5006223F044
:106C0000010353607B681B681021184602F0B0FD39
:106C10000023FB6256E0FB6A5A01FB69134403F54B
:106C200010631A464FF67F339360FB6A5A01FB6983
:106C3000134403F510631B68FA6A5101FA690A44A8
:106C400002F5106223F400131360FB6A5A01FB691A
:106C5000134403F510631B68FA6A5101FA690A4488
:106C600002F5106243F000631360FB6A5A01FB698E
:106C7000134403F530631A464FF67F339360FB6A83
:106C80005A01FB69134403F530631B68FA6A51012A
:106C9000FA690A4402F5306223F400131360FB6AB8
:106CA0005A01FB69134403F530631B68FA6A51010A
:106CB000FA690A4402F5306243F000631360FB6A2C
:106CC0000133FB627B685B68FA6A9A42A3D3FB6973
:106CD00003F50063DB69FA6902F5006243F0011312
:106CE000D3617B681B6B002B16D0FB6903F5006337
:106CF000D3F88430FA6902F5006243F00B03C2F85E
:106D00008430FB6903F500635B6CFA6902F500628D
:106D100043F00B03536415E0FB6903F500635A6904
:106D2000FB6903F50063194642F22B0313434B61E1
:106D3000FB6903F500631B69FA6902F5006243F021
:106D40000B031361FB6903F500631B68FA6902F525
:106D5000006223F4FE6313607B6818687B681B691C
:106D6000D9B27B6803F571731A4603F0DDFC7B68CA
:106D70001B685A697B681B6802F480525A617B6801
:106D80001B68184603F00AFC034603F40053B3F5EE
:106D9000005F24D17B681B68184603F0A1FC7B6868
:106DA0001B68184602F045FD03461A467B68DA6008
:106DB0007B681C6801F0E6F901467B68DB68DBB2A2
:106DC0001A46204602F078FA78685DF01AF97B6876
:106DD0001B685A697B681B6802F400525A617B6821
:106DE0001B68184603F0DAFB034603F00803082B80
:106DF0000AD178685DF0F7F87B681B685A697B6890
:106E00001B6802F008025A617B681B68184603F091
:106E1000C5FB034603F48013B3F5801F0FD1002395
:106E20007B627B6ADBB2194678685DF059F97B6852
:106E30001B685A697B681B6802F480125A617B6880
:106E40001B68184603F0AAFB034603F40013B3F5CE
:106E5000001F0FD100237B627B6ADBB21946786882
:106E60005DF02CF97B681B685A697B681B6802F42B
:106E700000125A617B681B68184603F08FFB0346BB
:106E800003F08043B3F1804F0AD178685DF03AF99E
:106E90007B681B685A697B681B6802F080425A61F4
:106EA0007B681B68184603F079FB034603F0040374
:106EB000042B15D17B681B685B68BB61BB6903F061
:106EC0000403002B02D078685DF02AF97B681B6808
:106ED00059687B681B68BA690A435A6000E000BFC2
:106EE0003437BD4690BD80B582B000AF78600B46A8
:106EF000FB707B6893F8BC33012B01D1022313E0B4
:106F00007B68012283F8BC237B68FA7883F83820F9
:106F10007B681B68FA781146184603F0E9FA7B682B
:106F2000002283F8BC23002318460837BD4680BDE5
:106F300080B584B000AF7860084611461A46034613
:106F4000FB700B463B801346BB700023FB7297F926
:106F50000330002B0FDAFB7803F00F021346DB003F
:106F60009B1A9B0038337A6813440433FB60FB6838
:106F700001225A700FE0FB7803F00F021346DB008A
:106F80009B1A9B0003F5FC737A6813440433FB607F
:106F9000FB6800225A70FB7803F00F03DAB2FB683B
:106FA0001A703A88FB689A60FB68BA78DA70FB68F6
:106FB0005B78002B04D0FB681B789AB2FB68DA8000
:106FC000BB78022B02D1FB6800221A717B6893F810
:106FD000BC33012B01D102230EE07B68012283F830
:106FE000BC237B681B68F968184602F047FC7B6885
:106FF000002283F8BC23FB7A18461037BD4680BDBB
:1070000080B584B000AF78600B46FB7097F9033011
:10701000002B0FDAFB7803F00F021346DB009B1AFC
:107020009B0038337A6813440433FB60FB68012209
:107030005A700FE0FB7803F00F021346DB009B1A37
:107040009B0003F5FC737A6813440433FB60FB6810
:1070500000225A70FB7803F00F03DAB2FB681A7053
:107060007B6893F8BC33012B01D102230EE07B68CF
:10707000012283F8BC237B681B68F968184602F07C
:1070800085FC7B68002283F8BC2300231846103758
:10709000BD4680BD80B586B000AFF8607A603B60C9
:1070A0000B46FB72FB7A03F00F021346DB009B1AC0
:1070B0009B0003F5FC73FA68134404337B617B691E
:1070C0007A68DA607B693A685A617B6900229A6162
:1070D0007B6900225A70FB7A03F00F03DAB27B69F6
:1070E0001A70FB681B69012B02D17A687B691A61EF
:1070F000FB7A03F00F03002B09D1FB681868FB68CB
:107100001B69DBB21A46796902F068FF08E0FB6888
:107110001868FB681B69DBB21A46796902F012FD38
:10712000002318461837BD4680BD80B483B000AF39
:1071300078600B46FB70FB7803F00F02796813460A
:10714000DB009B1A9B000B4403F505731B68184674
:107150000C37BD465DF8047B704780B586B000AF44
:10716000F8607A603B600B46FB72FB7A03F00F021B
:107170001346DB009B1A9B003833FA681344043330
:107180007B617B697A68DA607B693A685A617B69FE
:1071900000229A617B6901225A70FB7A03F00F0387
:1071A000DAB27B691A70FB681B69012B02D17A681D
:1071B0007B691A61FB7A03F00F03002B09D1FB688E
:1071C0001868FB681B69DBB21A46796902F006FF92
:1071D00008E0FB681868FB681B69DBB21A4679692E
:1071E00002F0B0FC002318461837BD4680BD80B5BC
:1071F00084B000AF78600B46FB70FB7803F00F02A1
:107200007B685B689A4201D9012350E097F903300B
:10721000002B0FDAFB7803F00F021346DB009B1AFA
:107220009B0038337A6813440433FB60FB68012207
:107230005A700DE0FA781346DB009B1A9B0003F5A9
:10724000FC737A6813440433FB60FB6800225A70B5
:10725000FB6801229A70FB7803F00F03DAB2FB6837
:107260001A707B6893F8BC33012B01D102231EE016
:107270007B68012283F8BC237B681B68F968184689
:1072800003F062F8FB7803F00F03002B0AD17B6850
:1072900018687B681B69D9B27B6803F571731A465D
:1072A00003F042FA7B68002283F8BC2300231846CF
:1072B0001037BD4680BD80B584B000AF78600B4606
:1072C000FB70FB7803F00F027B685B689A4201D980
:1072D000012342E097F90330002B0FDAFB7803F02B
:1072E0000F021346DB009B1A9B0038337A68134465
:1072F0000433FB60FB6801225A700FE0FB7803F057
:107300000F021346DB009B1A9B0003F5FC737A689F
:1073100013440433FB60FB6800225A70FB680022B0
:107320009A70FB7803F00F03DAB2FB681A707B687F
:1073300093F8BC33012B01D102230EE07B680122BC
:1073400083F8BC237B681B68F968184603F06AF869
:107350007B68002283F8BC23002318461037BD4603
:1073600080BD80B58AB002AF786039607B681B68E9
:107370007B617B693B613A681346DB009B1A9B008B
:1073800038337A6813440433FB60FB689A69FB68FE
:107390005B699A4201D901236CE0FB685A69FB687A
:1073A0009B69D31AFB61FB689B68FA699A4202D910
:1073B000FB689B68FB61FB6903339B08BB612BE0A7
:1073C000FB685A69FB689B69D31AFB61FB689B6881
:1073D000FA699A4202D9FB689B68FB61FB69033337
:1073E0009B08BB61FB68D9683B68DAB2FB6998B25D
:1073F0007B681B69DBB200930346786902F046FFA5
:10740000FB68DA68FB691A44FB68DA60FB689A6912
:10741000FB691A44FB689A613B685A013B69134453
:1074200003F510639B699BB2BA699A4209D8FB685D
:107430009A69FB685B699A4203D2FB685B69002B1F
:10744000BED1FB685A69FB689B699A4211D83B68B8
:1074500003F00F03012202FA03F3BB603B6903F55B
:1074600000635A6BBB68DB43396901F50061134067
:107470004B63002318462037BD4680BD80B586B0DB
:1074800000AF786039607B681B687B617B693B611A
:107490007B693C3304331B68FB603B685A013B69E2
:1074A000134403F530639B68BB607B681B69012B49
:1074B00040F0A080BB6803F00803002B15D0FB68E8
:1074C000724A934240F2DD80BB6803F40043002B14
:1074D00000F0D7803B685A013B69134403F53063E1
:1074E0001A464FF400439360CBE0BB6803F02003DF
:1074F000002B09D03B685A013B69134403F5306304
:107500001A4620239360BCE0BB6803F02803002BDD
:1075100040F0B780FB685D4A93420FD9BB6803F423
:107520000043002B0AD03B685A013B69134403F522
:1075300030631A464FF400439360A2E079683A68DA
:107540001346DB009B1A9B000B4403F501731A687A
:107550003B6859013B690B4403F530631B69C3F376
:107560001203D11A78683A681346DB009B1A9B0015
:10757000034403F50573196079683A681346DB0024
:107580009B1A9B000B4403F50273196878683A68EC
:107590001346DB009B1A9B00034403F501731B6831
:1075A000194478683A681346DB009B1A9B00034431
:1075B00003F5027319603B68002B14D179683A68AF
:1075C0001346DB009B1A9B000B4403F504731B68F6
:1075D000002B08D17B6818687B6803F571731A4625
:1075E000012103F0A1F83B68DBB2194678685CF032
:1075F000C5FC46E0FB68264A934224D1BB6803F4ED
:107600000043002B0AD03B685A013B69134403F541
:1076100030631A464FF40043936032E0BB6803F0D6
:107620002003002B08D03B685A013B69134403F543
:1076300030631A46202393603B68DBB219467868B2
:107640005CF09CFC1DE03B68002B14D179683A6823
:107650001346DB009B1A9B000B4403F504731B6865
:10766000002B08D17B6818687B6803F571731A4694
:10767000002103F059F83B68DBB2194678685CF0EA
:107680007DFC002318461837BD4680BD0A30544F94
:107690000A31544F80B586B000AF786039607B689E
:1076A0001B687B617B693B617B693C3304331B68EE
:1076B000FB603B685A013B69134403F530639B68E8
:1076C000BB60FB68154A93420ED9BB6803F40043C4
:1076D000002B09D03B685A013B69134403F5306322
:1076E0001A464FF40043936078685CF035FCFB6801
:1076F0000A4A93420CD97B681B69012B08D17B682D
:1077000018687B6803F571731A46012103F00CF8C1
:10771000002318461837BD4680BD00BF0A30544FBD
:1077200080B485B000AF78600B46FB7013463B8099
:107730007B681B685B6ABB60FB78002B07D13B88CA
:1077400019047B681B68BA680A439A6228E07B6860
:107750001B689B6A1B0CBA681344BB600023FB7355
:107760000DE07B681A68FB7B40339B0013445B6829
:107770001B0CBA681344BB60FB7B0133FB73FA7BC1
:10778000FB78013B9A42ECD33B8818047B6819686C
:10779000FB78013BBA68024340339B000B445A60BC
:1077A000002318461437BD465DF8047B704780B44B
:1077B00083B000AF78600B467B807B681B687A885B
:1077C0005A62002318460C37BD465DF8047B7047AB
:1077D00080B485B000AF78607B681B68FB607B6815
:1077E0000122C3F8FC237B68002283F8F423FB68A2
:1077F0009B6943F00062FB689A61FB685A6D054B18
:107800001343FA685365002318461437BD465DF8E4
:10781000047B70470300001080B400AF054B1B6869
:10782000044A43F48073136000BFBD465DF8047BD7
:10783000704700BF0070004080B582B000AF0023E9
:107840007B60234B1B6C224A43F080531364204B14
:107850001B6C03F080533B603B681E4B1B681D4A4A
:1078600043F480331360FCF7A1FB786009E0FCF778
:107870009DFB02467B68D31AB3F57A7F01D90323B7
:1078800022E0144B5B6803F48033B3F5803FEED104
:10789000104B1B680F4A43F400331360FCF786FB60
:1078A000786009E0FCF782FB02467B68D31AB3F5E7
:1078B0007A7F01D9032307E0064B5B6803F40033AA
:1078C000B3F5003FEED1002318460837BD4680BD12
:1078D000003802400070004080B586B000AF78608C
:1078E0000023FB757B68002B01D1012391E27B68AB
:1078F0001B6803F00103002B00F08780964B9B6808
:1079000003F00C03042B0CD0934B9B6803F00C0387
:10791000082B12D1904B5B6803F48003B3F5800F02
:107920000BD18D4B1B6803F40033002B6CD07B68AC
:107930005B68002B68D101236BE27B685B68B3F561
:10794000803F06D1844B1B68834A43F48033136025
:107950002EE07B685B68002B0CD17F4B1B687E4A56
:1079600023F4803313607C4B1B687B4A23F4802311
:1079700013601DE07B685B68B3F5A02F0CD1764BDC
:107980001B68754A43F480231360734B1B68724A6B
:1079900043F4803313600BE06F4B1B686E4A23F493
:1079A000803313606C4B1B686B4A23F48023136095
:1079B0007B685B68002B13D0FCF7F8FA386108E0AD
:1079C000FCF7F4FA02463B69D31A642B01D903236E
:1079D0001FE2614B1B6803F40033002BF0D014E06E
:1079E000FCF7E4FA386108E0FCF7E0FA02463B698C
:1079F000D31A642B01D903230BE2574B1B6803F402
:107A00000033002BF0D100E000BF7B681B6803F05F
:107A10000203002B69D0504B9B6803F00C03002B32
:107A20000BD04D4B9B6803F00C03082B1CD14A4B29
:107A30005B6803F48003002B16D1474B1B6803F0EF
:107A40000203002B05D07B68DB68012B01D00123EA
:107A5000DFE1414B1B6823F0F8027B681B69DB0008
:107A60003D4913430B6040E07B68DB68002B23D06B
:107A7000394B1B68384A43F001031360FCF796FA50
:107A8000386108E0FCF792FA02463B69D31A022BF0
:107A900001D90323BDE1304B1B6803F00203002B27
:107AA000F0D02D4B1B6823F0F8027B681B69DB00CC
:107AB000294913430B6018E0274B1B68264A23F023
:107AC00001031360FCF772FA386108E0FCF76EFA04
:107AD00002463B69D31A022B01D9032399E11E4BBD
:107AE0001B6803F00203002BF0D17B681B6803F0D6
:107AF0000803002B38D07B685B69002B19D0164B2C
:107B00005B6F154A43F001035367FCF74FFA386186
:107B100008E0FCF74BFA02463B69D31A022B01D965
:107B2000032376E10C4B5B6F03F00203002BF0D0D4
:107B30001AE0094B5B6F084A23F001035367FCF717
:107B400035FA38610AE0FCF731FA02463B69D31A8C
:107B5000022B03D903235CE100380240914B5B6F99
:107B600003F00203002BEED17B681B6803F00403D3
:107B7000002B00F0A4808B4B1B6C03F08053002B78
:107B80000DD1884B1B6C874A43F080531364854B9F
:107B90001B6C03F08053BB60BB680123FB75824BF9
:107BA0001B6803F48073002B18D17F4B1B687E4A3F
:107BB00043F480731360FCF7F9F9386108E0FCF7CF
:107BC000F5F902463B69D31A642B01D9032320E15E
:107BD000754B1B6803F48073002BF0D07B689B68A7
:107BE000012B06D16F4B1B6F6E4A43F001031367E5
:107BF0002DE07B689B68002B0CD16A4B1B6F694A98
:107C000023F001031367674B1B6F664A23F00403DD
:107C100013671CE07B689B68052B0CD1614B1B6FC5
:107C2000604A43F0040313675E4B1B6F5D4A43F0E9
:107C3000010313670BE05B4B1B6F5A4A23F00103F0
:107C40001367584B1B6F574A23F0040313677B6875
:107C50009B68002B15D0FCF7A9F938610AE0FCF706
:107C6000A5F902463B69D31A41F28832934201D901
:107C70000323CEE04B4B1B6F03F00203002BEED02F
:107C800014E0FCF793F938610AE0FCF78FF902463B
:107C90003B69D31A41F28832934201D90323B8E0F9
:107CA000404B1B6F03F00203002BEED1FB7D012B39
:107CB00005D13C4B1B6C3B4A23F0805313647B681B
:107CC0009B69002B00F0A480364B9B6803F00C03EB
:107CD000082B6BD07B689B69022B49D1314B1B6809
:107CE000304A23F080731360FCF760F9386108E0D4
:107CF000FCF75CF902463B69D31A022B01D9032336
:107D000087E0284B1B6803F00073002BF0D17B68E1
:107D1000DA697B681B6A1A437B685B6A9B011A43BA
:107D20007B689B6A5B08013B1B041A437B68DB6A28
:107D30001B0613431B4A43F000535360194B1B6847
:107D4000184A43F080731360FCF730F9386108E09B
:107D5000FCF72CF902463B69D31A022B01D9032305
:107D600057E0104B1B6803F00073002BF0D04FE07E
:107D70000C4B1B680B4A23F080731360FCF716F959
:107D8000386108E0FCF712F902463B69D31A022B6E
:107D900001D903233DE0034B1B6803F00073002B64
:107DA000F0D135E000380240007000401B4B5B68AA
:107DB000FB607B689B69012B28D0FB6803F4800281
:107DC0007B68DB699A4221D1FB6803F03F027B6844
:107DD0001B6A9A421AD1FA6847F6C07313407A6850
:107DE000526A9201934211D1FB6803F440327B68DE
:107DF0009B6A5B08013B1B049A4207D1FB6803F0B6
:107E000070627B68DB6A1B069A4201D0012300E0A6
:107E1000002318461837BD4680BD00BF0038024019
:107E200080B584B000AF786039600023FB607B6868
:107E3000002B01D10123D0E06A4B1B6803F00F0334
:107E40003A689A4210D9674B1B6823F00F026549C4
:107E50003B6813430B60634B1B6803F00F033A68E6
:107E60009A4201D00123B8E07B681B6803F002034B
:107E7000002B20D07B681B6803F00403002B05D087
:107E8000594B9B68584A43F4E05393607B681B68E6
:107E900003F00803002B05D0534B9B68524A43F470
:107EA00060439360504B9B6823F0F0027B689B68B3
:107EB0004D4913438B607B681B6803F00103002B63
:107EC00040D07B685B68012B07D1474B1B6803F4EC
:107ED0000033002B15D101237FE07B685B68022B08
:107EE00007D1414B1B6803F00073002B09D101231C
:107EF00073E03D4B1B6803F00203002B01D101230B
:107F00006BE0394B9B6823F003027B685B68364962
:107F100013438B60FCF74AF8F8600AE0FCF746F878
:107F20000246FB68D31A41F28832934201D90323F7
:107F300053E02D4B9B6803F00C027B685B689B0051
:107F40009A42EBD1274B1B6803F00F033A689A4221
:107F500010D2244B1B6823F00F0222493B681343C5
:107F60000B60204B1B6803F00F033A689A4201D064
:107F7000012332E07B681B6803F00403002B08D068
:107F8000194B9B6823F4E0527B68DB681649134366
:107F90008B607B681B6803F00803002B09D0124B31
:107FA0009B6823F460427B681B69DB000E49134326
:107FB0008B6000F021F802460B4B9B681B0903F015
:107FC0000F030A49CB5C22FA03F3094A1360094BF9
:107FD0001B681846FAF700F8002318461037BD460C
:107FE00080BD00BF003C024000380240BCD70808FA
:107FF00008000020480000202DE9B04F90B000AFED
:1080000000237B630023FB6300233B630023BB63EC
:10801000594B9B6803F00C03082B0DD0082B00F282
:10802000A180002B02D0042B03D09BE0534BBB63F9
:108030009BE0534BBB6398E04F4B5B6803F03F03FF
:108040007B634D4B5B6803F48003002B28D04A4BC5
:108050005B689B0900223B627A623B6AC3F30800BB
:108060000021474B03FB01F2002300FB03F3134401
:10807000434AA0FB0212FA620A46BA62FA6A134441
:10808000FB627B6B0022BB61FA61D7E90623D7E96B
:108090000A01F8F781FF02460B461346FB6353E0E3
:1080A000354B5B689B0900223B617A613B69C3F3F6
:1080B000080A4FF0000B52465B464FF000004FF0AD
:1080C0000001590141EAD261500102460B46B2EB70
:1080D0000A0863EB0B094FF000024FF000034FEA70
:1080E000891343EA98634FEA8812B2EB080463EB02
:1080F00009054FF000024FF00003EB0043EA547310
:10810000E20014461D4614EB0A033B6045EB0B03EB
:108110007B604FF000024FF00003D7E9004529468D
:108120008B02214643EA915321468A0210461946A2
:108130007B6B0022BB60FA60D7E90223F8F72CFFC3
:1081400002460B461346FB630B4B5B681B0C03F0AC
:10815000030301335B003B63FA6B3B6BB2FBF3F34E
:10816000BB6302E0054BBB6300BFBB6B18464037E7
:10817000BD46BDE8B08F00BF003802400024F400C7
:1081800040787D0180B400AF034B1B681846BD46A4
:108190005DF8047B704700BF0800002080B500AF89
:1081A000FFF7F0FF0246054B9B689B0A03F00703AD
:1081B0000349CB5C22FA03F3184680BD0038024025
:1081C000CCD7080880B483B000AF786039607B6892
:1081D0000F221A60124B9B6803F003027B685A60FF
:1081E0000F4B9B6803F0F0027B689A600C4B9B6816
:1081F00003F4E0527B68DA60094B9B68DB0803F408
:10820000E0527B681A61074B1B6803F00F023B6862
:108210001A6000BF0C37BD465DF8047B704700BF95
:1082200000380240003C024080B588B000AF786062
:1082300000237B6100233B610023FB600023FB6183
:108240000023BB617B681B6803F00103002B12D085
:10825000694B9B68684A23F400039360664B9A68F5
:108260007B685B6B644913438B607B685B6B002BA3
:1082700001D10123FB617B681B6803F40023002B01
:1082800017D05D4BD3F88C3023F440127B68DB6B46
:1082900059491343C1F88C307B68DB6BB3F5801F01
:1082A00001D10123FB617B68DB6B002B01D1012332
:1082B000BB617B681B6803F48013002B17D04E4B07
:1082C000D3F88C3023F440027B681B6C4A4913437B
:1082D000C1F88C307B681B6CB3F5800F01D1012392
:1082E000FB617B681B6C002B01D10123BB617B68A8
:1082F0001B6803F08073002B01D00123FB617B68B6
:108300001B6803F02003002B00F08B803A4B1B6CA2
:10831000394A43F080531364374B1B6C03F080538E
:10832000BB60BB68354B1B68344A43F480731360F1
:10833000FBF73CFE786108E0FBF738FE02467B69FC
:10834000D31A642B01D9032357E32C4B1B6803F486
:108350008073002BF0D0284B1B6F03F440733B61FC
:108360003B69002B35D07B681B6B03F440733A6983
:108370009A422ED0204B1B6F23F440733B611E4B5F
:108380001B6F1D4A43F4803313671B4B1B6F1A4A44
:1083900023F480331367184A3B691367164B1B6F2E
:1083A00003F00103012B14D1FBF700FE78610AE012
:1083B000FBF7FCFD02467B69D31A41F288329342F7
:1083C00001D9032319E30C4B1B6F03F00203002BAD
:1083D000EED07B681B6B03F44073B3F5407F11D183
:1083E000054B9B6823F4F8127B68196B044B0B4018
:1083F000014913438B600BE00038024000700040DD
:10840000FFFCFF0FAA4B9B68A94A23F4F813936063
:10841000A74B1A6F7B681B6BC3F30B03A449134371
:108420000B677B681B6803F01003002B10D0A04B78
:10843000D3F88C309E4A23F08073C2F88C309C4B6A
:10844000D3F88C207B689B6B99491343C1F88C301F
:108450007B681B6803F48043002B0AD0944BD3F84D
:10846000903023F440327B685B6E91491343C1F82E
:1084700090307B681B6803F40043002B0AD08C4BC0
:10848000D3F8903023F440227B689B6E88491343D5
:10849000C1F890307B681B6803F48033002B0AD04E
:1084A000834BD3F8903023F440127B68DB6E804915
:1084B0001343C1F890307B681B6803F40033002B32
:1084C0000AD07B4BD3F8903023F440027B681B6FBB
:1084D00077491343C1F890307B681B6803F0400371
:1084E000002B0AD0724BD3F8903023F003027B6844
:1084F0005B6C6F491343C1F890307B681B6803F0D5
:108500008003002B0AD06A4BD3F8903023F00C0282
:108510007B689B6C66491343C1F890307B681B688D
:1085200003F48073002B0AD0614BD3F8903023F012
:1085300030027B68DB6C5E491343C1F890307B6886
:108540001B6803F40073002B0AD0594BD3F890300A
:1085500023F0C0027B681B6D55491343C1F890306E
:108560007B681B6803F48063002B0AD0504BD3F860
:10857000903023F440727B685B6D4D491343C1F822
:1085800090307B681B6803F40063002B0AD0484BD3
:10859000D3F8903023F440627B689B6D44491343C9
:1085A000C1F890307B681B6803F48053002B0AD01D
:1085B0003F4BD3F8903023F440527B68DB6D3C494D
:1085C0001343C1F890307B681B6803F40053002B01
:1085D0000AD0374BD3F8903023F440427B681B6EAF
:1085E00033491343C1F890307B681B6803F4800360
:1085F000002B0AD02E4BD3F8903023F080627B689A
:108600009B6F2B491343C1F890307B681B6803F4C0
:108610000013002B11D0264BD3F8903023F00062CA
:108620007B68DB6F22491343C1F890307B68DB6FB6
:10863000B3F1006F01D10123BB617B681B6803F0BC
:108640000803002B01D00123BB617B681B6803F486
:108650008023002B0AD0164BD3F8903023F04072C1
:108660007B685B6F12491343C1F890307B681B68CD
:1086700003F40003002B0BD00D4BD3F8903023F004
:1086800080527B68D3F8803009491343C1F8903099
:10869000FB69012B05D07B681B68B3F1007F40F0BC
:1086A000D980034B1B68024A23F08063136001E00A
:1086B00000380240FBF77AFC786108E0FBF776FCB3
:1086C00002467B69D31A642B01D9032395E16D4BD4
:1086D0001B6803F00063002BF0D17B681B6803F07C
:1086E0000103002B21D07B685B6B002B1DD1654BF8
:1086F000D3F884301B0C03F003033B61614BD3F8C8
:1087000084301B0E03F00F03FB607B685B689A01EB
:108710003B691B041A43FB681B061A437B689B6872
:108720001B0758491343C1F884307B681B6803F466
:108730000023002B04D07B68DB6BB3F5801F0AD0CD
:108740007B681B6803F48013002B2ED07B681B6CA6
:10875000B3F5800F29D14B4BD3F884301B0C03F0B9
:1087600003033B61474BD3F884301B0F03F007032F
:10877000FB607B685B689A013B691B041A437B685A
:10878000DB681B061A43FB681B073E491343C1F80D
:1087900084303C4BD3F88C3023F01F027B685B6A3B
:1087A000013B38491343C1F88C307B681B6803F0E8
:1087B0008073002B1DD0334BD3F884301B0E03F095
:1087C0000F033B612F4BD3F884301B0F03F00703DB
:1087D000FB607B685B689A017B681B691B041A431A
:1087E0003B691B061A43FB681B0726491343C1F864
:1087F00084307B681B6803F00073002B11D07B680A
:108800005B689A017B681B691B041A437B68DB6801
:108810001B061A437B689B681B071A491343C1F860
:108820008430184B1B68174A43F080631360FBF7D2
:10883000BDFB786108E0FBF7B9FB02467B69D31A00
:10884000642B01D90323D8E00E4B1B6803F00063AF
:10885000002BF0D0BB69012B40F0CE80094B1B6888
:10886000084A23F080531360FBF7A0FB78610BE00C
:10887000FBF79CFB02467B69D31A642B04D90323C4
:10888000BBE000BF003802405E4B1B6803F00053A2
:10889000B3F1005FECD07B681B6803F40023002B6E
:1088A00003D07B68DB6B002B09D07B681B6803F46B
:1088B0008013002B2ED07B681B6C002B2AD1514BD0
:1088C000D3F888301B0C03F003033B614D4BD3F806
:1088D00088301B0F03F00703FB607B685B699A011C
:1088E0003B691B041A437B689B691B061A43FB68A0
:1088F0001B0744491343C1F88830424BD3F88C30EE
:1089000023F4F8527B689B6A013B1B023D491343E9
:10891000C1F88C307B681B6803F40013002B22D055
:108920007B68DB6FB3F1006F1DD1364BD3F8883015
:108930001B0E03F00F033B61324BD3F888301B0F43
:1089400003F00703FB607B685B699A017B681B6A25
:108950001B041A433B691B061A43FB681B07294982
:108960001343C1F888307B681B6803F00803002BB1
:1089700028D0244BD3F888301B0E03F00F033B6143
:10898000204BD3F888301B0C03F00303FB607B689B
:108990005B699A01FB681B041A433B691B061A4377
:1089A0007B68DB691B0717491343C1F88830154BF7
:1089B000D3F88C3023F440327B68DB6A11491343CF
:1089C000C1F88C300F4B1B680E4A43F08053136084
:1089D000FBF7ECFA786108E0FBF7E8FA02467B69FE
:1089E000D31A642B01D9032307E0064B1B6803F05D
:1089F0000053B3F1005FEFD1002318462037BD4686
:108A000080BD00BF0038024080B582B000AF786002
:108A100039607B68002B01D1012325E07B6893F846
:108A20002C30DBB2002B06D17B68002283F82D208E
:108A30007868F8F753FD7B68022283F82C207B6866
:108A40001A687B6804331946104600F0B7FA7B6851
:108A500018687B685B681A46396800F021FB7B6800
:108A6000012283F82C20002318460837BD4680BD1C
:108A700080B584B000AFF860B9607A60FB6893F8A5
:108A80002C30DBB2022B01D1022318E0FB6802225A
:108A900083F82C20FB681B687A68B968184600F0D8
:108AA0007FFBBB681B68022B04D1FB68052283F89F
:108AB0002C2003E0FB68012283F82C2000231846B9
:108AC0001037BD4680BD80B582B000AF7860396098
:108AD0007B6893F82C30DBB2022B01D102230EE02D
:108AE0007B68022283F82C207B681B683968184653
:108AF00000F077FB7B68012283F82C2000231846C6
:108B00000837BD4680BD80B582B000AF78607B6815
:108B1000002B01D101231DE07B6893F83D30DBB2CF
:108B2000002B06D17B68002283F83C207868F9F797
:108B3000F7FB7B68022283F83D207B681A687B681C
:108B400004331946104600F07BF97B68012283F854
:108B50003D20002318460837BD4680BD80B485B04F
:108B600000AF78607B681B68DA687B681B6842F03E
:108B70000102DA607B681B689A680C4B1340FB604B
:108B8000FB68062B0BD0FB68B3F5803F07D07B68F2
:108B90001B681A687B681B6842F001021A60002398
:108BA00018461437BD465DF8047B70470700010086
:108BB00080B582B000AF78607B681B681B6903F0EA
:108BC0000203022B22D17B681B68DB6803F00203DF
:108BD000022B1BD17B681B686FF002021A617B6855
:108BE00001221A777B681B689B6903F00303002B43
:108BF00003D0786800F005F905E0786800F0F7F830
:108C0000786800F008F97B6800221A777B681B6897
:108C10001B6903F00403042B22D17B681B68DB680B
:108C200003F00403042B1BD17B681B686FF0040264
:108C30001A617B6802221A777B681B689B6903F4C0
:108C40004073002B03D0786800F0DBF805E078680B
:108C500000F0CDF8786800F0DEF87B6800221A7723
:108C60007B681B681B6903F00803082B22D17B6813
:108C70001B68DB6803F00803082B1BD17B681B68AB
:108C80006FF008021A617B6804221A777B681B6800
:108C9000DB6903F00303002B03D0786800F0B1F820
:108CA00005E0786800F0A3F8786800F0B4F87B6815
:108CB00000221A777B681B681B6903F01003102BD6
:108CC00022D17B681B68DB6803F01003102B1BD1DB
:108CD0007B681B686FF010021A617B6808221A77A4
:108CE0007B681B68DB6903F44073002B03D0786852
:108CF00000F087F805E0786800F079F8786800F00F
:108D00008AF87B6800221A777B681B681B6903F06E
:108D10000103012B0ED17B681B68DB6803F00103A4
:108D2000012B07D17B681B686FF001021A6178681C
:108D3000F9F750F87B681B681B6903F08003802BF0
:108D40000ED17B681B68DB6803F08003802B07D1A2
:108D50007B681B686FF080021A61786800F01AF96E
:108D60007B681B681B6903F48073B3F5807F0ED1A9
:108D70007B681B68DB6803F08003802B07D17B686E
:108D80001B686FF480721A61786800F00DF97B68D7
:108D90001B681B6903F04003402B0ED17B681B68E6
:108DA000DB6803F04003402B07D17B681B686FF042
:108DB00040021A61786800F038F87B681B681B690C
:108DC00003F02003202B0ED17B681B68DB6803F0C7
:108DD0002003202B07D17B681B686FF020021A61EB
:108DE000786800F0CDF800BF0837BD4680BD80B47C
:108DF00083B000AF786000BF0C37BD465DF8047BE0
:108E0000704780B483B000AF786000BF0C37BD46B8
:108E10005DF8047B704780B483B000AF786000BF1A
:108E20000C37BD465DF8047B704780B483B000AF5B
:108E3000786000BF0C37BD465DF8047B70470000CA
:108E400080B485B000AF786039607B681B68FB60D8
:108E50007B68404A934213D07B68B3F1804F0FD0B8
:108E60007B683D4A93420BD07B683C4A934207D0D3
:108E70007B683B4A934203D07B683A4A934208D1CD
:108E8000FB6823F07003FB603B685B68FA68134380
:108E9000FB607B682F4A93422BD07B68B3F1804FF5
:108EA00027D07B682C4A934223D07B682B4A93427D
:108EB0001FD07B682A4A93421BD07B68294A934281
:108EC00017D07B68284A934213D07B68274A934285
:108ED0000FD07B68264A93420BD07B68254A934289
:108EE00007D07B68244A934203D07B68234A93428D
:108EF00008D1FB6823F44073FB603B68DB68FA68C9
:108F00001343FB60FB6823F080023B685B691343FB
:108F1000FB607B68FA681A603B689A687B68DA6273
:108F20003B681A687B689A627B680A4A934203D05E
:108F30007B680C4A934203D13B681A697B681A63C9
:108F40007B6801225A6100BF1437BD465DF8047B7F
:108F5000704700BF000001400004004000080040CE
:108F6000000C00400004014000400140004401406A
:108F70000048014000180040001C00400020004054
:108F800080B483B000AF786000BF0C37BD465DF899
:108F9000047B704780B483B000AF786000BF0C37AB
:108FA000BD465DF8047B704780B483B000AF786045
:108FB00000BF0C37BD465DF8047B704780B485B0B8
:108FC00000AF786039600023FB600023BB603B6822
:108FD0001B68012B27D07B681B68FB60FA682F4B4E
:108FE0001340FB603B685A683B689B681A433B68C8
:108FF000DB681A433B681B691A433B685B691A4389
:109000003B689B691A433B68DB691A433B681B6AF0
:109010001A433B685B6A1343FA681343FB607B683F
:10902000FA681A6032E07B681B68FB60FB6823F417
:10903000F843FB603B68DA693B681B6A1A433B688C
:109040005B6A1343FA681343FB607B685B68BB6031
:10905000BA68124B1340BB603B685A683B689B6818
:109060001A433B68DB681A433B681B691A433B6839
:109070005B691A433B689B691343BA681343BB603F
:109080007B68FA681A607B68BA685A6000231846E1
:109090001437BD465DF8047B704700BF0080FFFFBA
:1090A00080B487B000AFF860B9607A6000237B615C
:1090B00000233B617B68012B2ED0FB689B687B61A2
:1090C0007B6903F070437B61BB681B685A1EBB68F9
:1090D0005B68013B1B011A43BB689B68013B1B0299
:1090E0001A43BB68DB68013B1B031A43BB681B695F
:1090F000013B1B041A43BB685B69013B1B051A4318
:10910000BB689B69013B1B0613437A6913437B6170
:10911000FB687A699A6039E0FB689B687B617A69D1
:109120001E4B13407B61BB68DB68013B1A03BB68C5
:109130005B69013B1B0513437A6913437B61FB6841
:10914000DB683B613B6903F070433B61BB681B68B4
:109150005A1EBB685B68013B1B011A43BB689B68D6
:10916000013B1B021A43BB681B69013B1B041A43EA
:10917000BB689B69013B1B0613433A6913433B6180
:10918000FB687A699A60FB683A69DA6000231846DE
:109190001C37BD465DF8047B704700BFFF0F0FFF13
:1091A00080B487B000AFF860B9607A6000237B615B
:1091B000BB681A68BB685B681A43BB689B68013B65
:1091C0005B011A43BB68DB685B0213437B617A690E
:1091D000FB681A61002318461C37BD465DF8047B06
:1091E000704780B483B000AF786039607B685A699B
:1091F0003B685B001A437B685A61002318460C37B2
:10920000BD465DF8047B704784B080B584B000AF84
:10921000786007F11C0080E80E003B6B012B20D129
:109220007B689B6B23F480327B689A637B68DA6887
:10923000204B13407A68D3607B68DB6823F44012CC
:109240007B68DA60FB6C012B05D17B68DB6843F43B
:1092500080127B68DA60786801F0C4FA0346FB7319
:1092600010E07B68DB6843F040027B68DA60786876
:1092700001F0B8FA0346FB737B689B6B43F48032C2
:109280007B689A63BB6A012B0BD17B689B6843F0B8
:1092900006027B689A607B689B6843F020027B68CB
:1092A0009A60FB7B18461037BD46BDE8804004B08D
:1092B000704700BFBFFFBDFF80B487B000AFF8604C
:1092C000B9601346FB71FB79022B65D1BB68414A3B
:1092D000934206D9BB68404A934202D20F237B6176
:1092E00062E0BB683C4A934206D3BB683B4A934268
:1092F00002D20E237B6157E0BB68384A934206D303
:10930000BB68374A934202D20D237B614CE0BB68B5
:10931000334A934206D3BB68324A934202D80C23A5
:109320007B6141E0BB682F4A934206D9BB682E4A55
:10933000934202D80B237B6136E0BB682A4A9342F2
:1093400006D9BB68294A934202D80A237B612BE0E5
:10935000BB68264A934206D9BB68254A934202D28B
:1093600009237B6120E0BB68214A934206D3BB6896
:10937000204A934202D808237B6115E0BB681D4A4E
:10938000934206D9BB681C4A934202D207237B61F1
:109390000AE006237B6107E0FB79002B02D1092359
:1093A0007B6101E009237B61FB68DB6823F4705279
:1093B000FB68DA60FB68DA687B699B0203F4705330
:1093C0001A43FB68DA60002318461C37BD465DF877
:1093D000047B7047BFACD800C0E1E4000024F40077
:1093E000807306019F491A01FF2C31013FA44C01F3
:1093F00000366E011FABA6010048E80180B483B0BF
:1094000000AF78607B689B6843F001027B689A60DC
:10941000002318460C37BD465DF8047B704780B4C6
:1094200083B000AF78607B689B6823F001027B68A3
:109430009A60002318460C37BD465DF8047B7047E0
:1094400080B582B000AF78600B46FB707B68DB684C
:1094500023F0C0427B68DA60FB78012B06D17B6881
:10946000DB6843F000527B68DA600BE0FB78002B8E
:1094700006D17B68DB6843F080427B68DA6001E0FC
:10948000012303E03220FAF79DFD00231846083738
:10949000BD4680BD84B080B586B000AF786007F16E
:1094A000240080E80E000023FB757B68FB6000232E
:1094B0003B6109E07A683B6940339B00134400221A
:1094C0005A603B6901333B613B690E2BF2D9FB6C5F
:1094D000002B1CD1FB6803F500635B68FA6802F59A
:1094E000006243F0020353607B689B6B23F400121D
:1094F0007B689A637B681B6843F040027B681A6054
:109500007B681B6843F080027B681A6005E07B681B
:109510009B6B43F400127B689A63FB6803F56063FE
:109520001A4600231360FB6803F500631946FB68C5
:1095300003F500631A460B681360BB6B012B0CD15B
:10954000FB6A002B04D10021786800F059F918E07B
:109550000121786800F054F913E0BB6B032B0CD1A8
:10956000FB6A002B04D10021786800F049F908E07B
:109570000121786800F044F903E00321786800F0E5
:109580003FF91021786800F0F3F80346002B01D072
:109590000123FB75786800F011F90346002B01D018
:1095A0000123FB75FB6803F500631A460023136172
:1095B000FB6803F500631A4600235361FB6803F55B
:1095C00000631A460023D36100233B6143E03B69FB
:1095D0005A01FB68134403F510631B6803F0004352
:1095E000B3F1004F18D13B69002B0AD13B695A01F6
:1095F000FB68134403F510631A464FF000631360D1
:1096000013E03B695A01FB68134403F510631A46E3
:109610004FF09043136008E03B695A01FB68134424
:1096200003F510631A46002313603B695A01FB6877
:10963000134403F510631A46002313613B695A0172
:10964000FB68134403F510631A464FF67F339360AB
:109650003B6901333B617B6A3A699A42B7D3002385
:109660003B6143E03B695A01FB68134403F53063F7
:109670001B6803F00043B3F1004F18D13B69002B86
:109680000AD13B695A01FB68134403F530631A465B
:109690004FF00063136013E03B695A01FB68134409
:1096A00003F530631A464FF09043136008E03B69BE
:1096B0005A01FB68134403F530631A460023136014
:1096C0003B695A01FB68134403F530631A460023D3
:1096D00013613B695A01FB68134403F530631A4672
:1096E0004FF67F3393603B6901333B617B6A3A6994
:1096F0009A42B7D3FB6803F500631B69FA6802F569
:10970000006223F4807313617B6800229A617B6896
:109710006FF080425A613B6B002B05D17B689B69DF
:1097200043F010027B689A617B689A690E4B134381
:109730007A689361FB6B002B05D07B689B6943F0D3
:1097400008027B689A61FB6C012B05D17B689A69E2
:10975000064B13437A689361FB7D18461837BD4664
:10976000BDE8804004B0704700383C8004000040F1
:1097700080B485B000AF786039600023FB603B683F
:109780009B0143F020027B681A61FB680133FB6098
:10979000FB68094A934201D9032306E07B681B69F1
:1097A00003F02003202BF0D0002318461437BD46C9
:1097B0005DF8047B704700BF400D030080B485B0A6
:1097C00000AF78600023FB607B6810221A61FB68A1
:1097D0000133FB60FB68094A934201D9032306E089
:1097E0007B681B6903F01003102BF0D00023184690
:1097F0001437BD465DF8047B704700BF400D030081
:1098000080B485B000AF78600B46FB707B68FB606E
:10981000FB6803F500631A68FB78F96801F50061DD
:1098200013430B60002318461437BD465DF8047BD4
:10983000704780B487B000AF78607B683B613B695C
:1098400003F500639B6803F00603FB60FB68002BD5
:1098500002D10023FB750AE0FB68022B02D0FB68F3
:10986000062B02D10223FB7501E00F23FB75FB7D64
:1098700018461C37BD465DF8047B704780B485B040
:1098800000AF786039607B68FB603B681B78BB6029
:109890003B685B78012B39D1FB6803F50063DA691B
:1098A0003B681B7803F00F03012101FA03F39BB21D
:1098B000F96801F500611343CB61BB685A01FB688D
:1098C000134403F510631B6803F40043002B53D1CA
:1098D000BB685A01FB68134403F510631A683B68C0
:1098E0009B68C3F30A013B68DB789B041943BB68A0
:1098F0009B050B431A43BB685901FB680B4403F5F6
:1099000010631946204B13430B6035E0FB6803F5E9
:109910000063DA693B681B7803F00F03012101FA49
:1099200003F31B04F96801F500611343CB61BB68C5
:109930005A01FB68134403F530631B6803F40043CA
:10994000002B19D1BB685A01FB68134403F530633F
:109950001A683B689B68C3F30A013B68DB789B0489
:109960000B431A43BB685901FB680B4403F5306392
:109970001946054B13430B60002318461437BD46A8
:109980005DF8047B704700BF0080001080B485B094
:1099900000AF786039607B68FB603B681B78BB6018
:1099A0003B685B78012B61D1BB685A01FB681344AB
:1099B00003F510631B6803F00043B3F1004F1FD1A0
:1099C000BB685A01FB68134403F510631B68BA684F
:1099D0005101FA680A4402F5106243F00063136013
:1099E000BB685A01FB68134403F510631B68BA682F
:1099F0005101FA680A4402F5106243F08043136093
:109A0000FB6803F50063DA6B3B681B7803F00F0318
:109A1000012101FA03F39BB2DB43F96801F5006110
:109A20001340CB63FB6803F50063DA693B681B787E
:109A300003F00F03012101FA03F39BB2DB43F96842
:109A400001F500611340CB61BB685A01FB68134408
:109A500003F510631A68BB685901FB680B4403F5F2
:109A600010631946354B13400B6060E0BB685A0128
:109A7000FB68134403F530631B6803F00043B3F144
:109A8000004F1FD1BB685A01FB68134403F53063D4
:109A90001B68BA685101FA680A4402F5306243F063
:109AA00000631360BB685A01FB68134403F530631D
:109AB0001B68BA685101FA680A4402F5306243F043
:109AC00080431360FB6803F50063DA6B3B681B7827
:109AD00003F00F03012101FA03F31B04DB43F968D0
:109AE00001F500611340CB63FB6803F50063DA699D
:109AF0003B681B7803F00F03012101FA03F31B04F9
:109B0000DB43F96801F500611340CB61BB685A0182
:109B1000FB68134403F530631A68BB685901FB689E
:109B20000B4403F530631946054B13400B600023CB
:109B300018461437BD465DF8047B7047007833EC57
:109B40000078F3EF80B58AB002AFF860B9601346D1
:109B5000FB71FB68FB61BB681B78BB61BB685B7812
:109B6000012B40F06381BB685B69002B32D1BB697C
:109B70005A01FB69134403F510631A69BB69590163
:109B8000FB690B4403F510631946A54B13400B61A9
:109B9000BB695A01FB69134403F510631B69BA6979
:109BA0005101FA690A4402F5106243F4002313617B
:109BB000BB695A01FB69134403F510631A69BB6959
:109BC0005901FB690B4403F510631946954B13408B
:109BD0000B6174E0BB695A01FB69134403F5106320
:109BE0001A69BB695901FB690B4403F510631946F7
:109BF0008C4B13400B61BB695A01FB69134403F59D
:109C000010631A69BB695901FB690B4403F51063C2
:109C10001946834B13400B61BB695A01FB6913441E
:109C200003F510631A69BB685969BB689B680B44EC
:109C3000591EBB689B68B1FBF3F3D9047A4B0B4008
:109C4000B9694801F969014401F5106113430B61D9
:109C5000BB695A01FB69134403F510631A69BB68B9
:109C60005B69C3F31203B9694801F969014401F55D
:109C7000106113430B61BB68DB78012B1FD1BB69FB
:109C80005A01FB69134403F510631B69BA6951015A
:109C9000FA690A4402F5106223F0C0431361BB69FC
:109CA0005A01FB69134403F510631B69BA6951013A
:109CB000FA690A4402F5106243F000531361FB791C
:109CC000012B4BD1BB681B69002B09D0BB695A0122
:109CD000FB69134403F510631A46BB681B695361A3
:109CE000BB68DB78012B28D1FB6903F500639B6817
:109CF00003F48073002B10D1BB695A01FB69134434
:109D000003F510631B68BA695101FA690A4402F548
:109D1000106243F0005313600FE0BB695A01FB6906
:109D2000134403F510631B68BA695101FA690A44C8
:109D300002F5106243F080531360BB695A01FB695E
:109D4000134403F510631B68BA695101FA690A44A8
:109D500002F5106243F00443136033E1BB695A011A
:109D6000FB69134403F510631B68BA695101FA6972
:109D70000A4402F5106243F004431360BB68DB78C9
:109D8000012B15D0BB685B69002B00F01B81FB69C0
:109D900003F500635A6BBB681B7803F00F030121C6
:109DA00001FA03F3F96901F5006113434B6309E11B
:109DB000FB6903F500639B6803F48073002B10D1EB
:109DC000BB695A01FB69134403F510631B68BA6948
:109DD0005101FA690A4402F5106243F0005313601E
:109DE0000FE0BB695A01FB69134403F510631B685C
:109DF000BA695101FA690A4402F5106243F08053CE
:109E00001360BB68D968BB681A78BB685B6998B295
:109E1000FB7900930346F86800F038FAD2E000BFFF
:109E2000FFFF07E00000F8FF0000F81FBB695A01C0
:109E3000FB69134403F530631A69BB695901FB6977
:109E40000B4403F530631946614B13400B61BB694A
:109E50005A01FB69134403F530631A69BB69590160
:109E6000FB690B4403F5306319465A4B13400B61F1
:109E7000BB685B69002B23D1BB695A01FB691344A2
:109E800003F530631A69BB689B68C3F31203B969B1
:109E90004801F969014401F5306113430B61BB6965
:109EA0005A01FB69134403F530631B69BA69510118
:109EB000FA690A4402F5306243F40023136133E087
:109EC000BB685A69BB689B6813445A1EBB689B6891
:109ED000B2FBF3F3FB82BB695A01FB69134403F540
:109EE00030631A69FB8AD9043B4B0B40B9694801BE
:109EF000F969014401F5306113430B61BB695A01F3
:109F0000FB69134403F530631A69BB689B68F98ADF
:109F100001FB03F3C3F31203B9694801F969014472
:109F200001F5306113430B61FB79012B0DD1BB6847
:109F3000DB68002B09D0BB68D968BB695A01FB6993
:109F4000134403F530630A465A61BB68DB78012B82
:109F500028D1FB6903F500639B6803F48073002B31
:109F600010D1BB695A01FB69134403F530631B68C8
:109F7000BA695101FA690A4402F5306243F00053AC
:109F800013600FE0BB695A01FB69134403F53063AA
:109F90001B68BA695101FA690A4402F5306243F05C
:109FA00080531360BB695A01FB69134403F53063A6
:109FB0001B68BA695101FA690A4402F5306243F03C
:109FC00004431360002318462037BD4680BD00BF00
:109FD0000000F8FFFFFF07E00000F81F80B487B023
:109FE00000AFF860B9601346FB71FB687B61BB682A
:109FF0001B783B61BB685B78012B40F0CD80BB6870
:10A000005B69002B32D13B695A017B69134403F52C
:10A0100010631A693B6959017B690B4403F51063AE
:10A020001946984B13400B613B695A017B691344F5
:10A0300003F510631B693A6951017A690A4402F514
:10A04000106243F4002313613B695A017B69134496
:10A0500003F510631A693B6959017B690B4403F5E9
:10A0600010631946884B13400B614EE03B695A015F
:10A070007B69134403F510631A693B6959017B69D5
:10A080000B4403F5106319467F4B13400B613B698A
:10A090005A017B69134403F510631A693B6959013E
:10A0A0007B690B4403F510631946764B13400B6133
:10A0B000BB685A69BB689B689A4203D9BB689A68B7
:10A0C000BB685A613B695A017B69134403F510630D
:10A0D0001B693A6951017A690A4402F5106243F436
:10A0E000002313613B695A017B69134403F5106334
:10A0F0001A69BB685B69C3F312033969480179695E
:10A10000014401F5106113430B61FB79012B1ED152
:10A11000BB681B69002B09D03B695A017B6913445A
:10A1200003F510631A46BB681B6953613B695A010A
:10A130007B69134403F510631B683A6951017A691E
:10A140000A4402F5106243F00443136092E03B6955
:10A150005A017B69134403F510631B683A69510186
:10A160007A690A4402F5106243F004431360BB6845
:10A170005B69002B7ED07B6903F500635A6BBB687B
:10A180001B7803F00F03012101FA03F3796901F54C
:10A19000006113434B636DE03B695A017B691344D3
:10A1A00003F530631A693B6959017B690B4403F578
:10A1B00030631946344B13400B613B695A017B698C
:10A1C000134403F530631A693B6959017B690B44F9
:10A1D00003F5306319462B4B13400B61BB685B6979
:10A1E000002B03D0BB689A68BB685A613B695A016F
:10A1F0007B69134403F530631B693A6951017A693D
:10A200000A4402F5306243F4002313613B695A01AA
:10A210007B69134403F530631A69BB689B68C3F319
:10A220001203396948017969014401F5306113432A
:10A230000B61FB79012B0DD1BB68DB68002B09D0CA
:10A24000BB68D9683B695A017B69134403F53063E5
:10A250000A465A613B695A017B69134403F530632E
:10A260001B683A6951017A690A4402F5306243F089
:10A2700004431360002318461C37BD465DF8047B79
:10A28000704700BFFFFF07E00000F8FF80B489B00F
:10A2900000AFF860B96011461A460B46FB711346D1
:10A2A000BB80FB687B61BB68FB6197F82830002BA3
:10A2B0001AD1BB8803339B083B610023BB610FE0CD
:10A2C000FB791A037B69134403F580531A46FB6933
:10A2D0001B681360FB690433FB61BB690133BB611D
:10A2E000BA693B699A42EBD3002318462437BD462E
:10A2F0005DF8047B704780B489B000AFF860B96046
:10A300001346FB80FB687B61BB68FB61FB88033302
:10A310009B083B610023BB610BE07B6903F5805325
:10A320001A68FB691A60FB690433FB61BB6901337E
:10A33000BB61BA693B699A42EFD3FB69184624377F
:10A34000BD465DF8047B704780B485B000AF78608F
:10A3500039607B68FB603B681B78BB603B685B785F
:10A36000012B2CD1BB685A01FB68134403F5106321
:10A370001B68002B12DBBB68002B0FD0BB685A0197
:10A38000FB68134403F510631B68BA685101FA684F
:10A390000A4402F5106223F080431360BB685A013F
:10A3A000FB68134403F510631B68BA685101FA682F
:10A3B0000A4402F5106243F4001313602BE0BB68FB
:10A3C0005A01FB68134403F530631B68002B12DB52
:10A3D000BB68002B0FD0BB685A01FB68134403F520
:10A3E00030631B68BA685101FA680A4402F53062AA
:10A3F00023F080431360BB685A01FB68134403F5E4
:10A4000030631B68BA685101FA680A4402F5306289
:10A4100043F400131360002318461437BD465DF85B
:10A42000047B704780B485B000AF786039607B688A
:10A43000FB603B681B78BB603B685B78012B28D1D5
:10A44000BB685A01FB68134403F510631B68BA68C4
:10A450005101FA680A4402F5106223F400131360F4
:10A460003B68DB78032B03D03B68DB78022B38D1C9
:10A47000BB685A01FB68134403F510631B68BA6894
:10A480005101FA680A4402F5106243F080531360E8
:10A4900027E0BB685A01FB68134403F530631B686F
:10A4A000BA685101FA680A4402F5306223F40013D5
:10A4B00013603B68DB78032B03D03B68DB78022B0F
:10A4C0000FD1BB685A01FB68134403F530631B6866
:10A4D000BA685101FA680A4402F5306243F08053C9
:10A4E0001360002318461437BD465DF8047B70479F
:10A4F00080B485B000AF78600B46FB707B68FB6072
:10A50000FB6803F500631B68FA6802F5006223F438
:10A51000FE631360FB6803F500631A68FB781B0198
:10A5200003F4FE63F96801F5006113430B60002337
:10A5300018461437BD465DF8047B704780B584B07B
:10A5400000AF78607B68FB60FB6803F500635B68C5
:10A55000FA6802F5006223F0020353600320F9F762
:10A5600031FD002318461037BD4680BD80B584B04C
:10A5700000AF78607B68FB60FB6803F500635B6895
:10A58000FA6802F5006243F0020353600320F9F712
:10A5900019FD002318461037BD4680BD80B485B034
:10A5A00000AF78607B685B69FB607B689B69FA68D9
:10A5B0001340FB60FB6818461437BD465DF8047B0A
:10A5C000704780B485B000AF78607B68FB60FB6843
:10A5D00003F500639B69BB60FB6803F50063DB69FF
:10A5E000BA681340BB60BB681B0C18461437BD46E5
:10A5F0005DF8047B704780B485B000AF78607B68FD
:10A60000FB60FB6803F500639B69BB60FB6803F5B7
:10A610000063DB69BA681340BB60BB689BB2184635
:10A620001437BD465DF8047B704780B485B000AF39
:10A6300078600B46FB707B68FB60FB785A01FB6817
:10A64000134403F530639B68BB60FB6803F500634C
:10A650005B69BA681340BB60BB6818461437BD46D7
:10A660005DF8047B704780B487B000AF78600B461C
:10A67000FB707B687B617B6903F500631B693B6151
:10A680007B6903F500635B6BFB60FB7803F00F03F2
:10A69000FA6822FA03F3DB01DBB23A6913433B6148
:10A6A000FB785A017B69134403F510639B683A6990
:10A6B0001340BB60BB6818461C37BD465DF8047B81
:10A6C000704780B483B000AF78607B685B6903F04B
:10A6D000010318460C37BD465DF8047B7047000047
:10A6E00080B485B000AF78607B68FB60FB6803F5E1
:10A6F00010631A68FB6803F510631946094B134091
:10A700000B60FB6803F500635B68FA6802F50062A2
:10A7100043F480735360002318461437BD465DF838
:10A72000047B704700F8FFFF80B487B000AFF8608B
:10A730000B467A60FB72FB687B61FB683C33043339
:10A740001B683B613B69264A93420AD97B6903F542
:10A7500030631B6803F00043B3F1004F01D10023C5
:10A7600037E07B6903F530631A46002313617B6988
:10A7700003F530631B697A6902F5306243F4002304
:10A7800013617B6903F530631B697A6902F53062F6
:10A7900043F0180313617B6903F530631B697A6921
:10A7A00002F5306243F0C0431361FB7A012B0FD1F5
:10A7B0007B6903F530631A467B6853617B6903F557
:10A7C00030631B687A6902F5306243F080231360BE
:10A7D000002318461C37BD465DF8047B704700BF58
:10A7E0000A30544F80B485B000AF78600023FB601E
:10A7F000FB680133FB60FB68134A934201D90323D2
:10A800001BE07B681B69002BF2DA0023FB607B688E
:10A810001B6943F001027B681A61FB680133FB602E
:10A82000FB68094A934201D9032306E07B681B6950
:10A8300003F00103012BF0D0002318461437BD4666
:10A840005DF8047B704700BF400D030080B584B005
:10A8500000AF78600B46FB704FF4077079F038FC5E
:10A860000346FB60FB68002B05D17B680022C3F820
:10A87000BC22022366E07B68FA68C3F8BC227B68CE
:10A880001B7C002B19D14FF40073022281217868C0
:10A8900059F0BBFC7B6801221A874FF40073022237
:10A8A0000121786859F0B1FC7B680122A3F8782176
:10A8B0007B681022A3F84E2016E04023022281215B
:10A8C000786859F0A2FC7B6801221A874023022293
:10A8D0000121786859F099FC7B680122A3F878215E
:10A8E0007B681022A3F84E20082303228221786877
:10A8F00059F08BFC7B680122A3F84C207B68D3F8CD
:10A90000C0321B689847FB680022C3F81422FB681A
:10A910000022C3F818227B681B7C002B09D1FB683E
:10A92000D3F804224FF400730121786859F05CFDDC
:10A9300007E0FB68D3F8042240230121786859F02E
:10A9400053FD002318461037BD4680BD80B584B046
:10A9500000AF78600B46FB700023FB7381217868A1
:10A9600059F079FC7B6800221A870121786859F038
:10A9700072FC7B680022A3F878218221786859F064
:10A980006AFC7B680022A3F84C207B680022A3F8B5
:10A990004E207B68D3F8BC32002B0ED07B68D3F8F6
:10A9A000C0325B6898477B68D3F8BC32184679F0B0
:10A9B00097FB7B680022C3F8BC22FB7B184610374C
:10A9C000BD4680BD80B586B000AF786039607B68D9
:10A9D000D3F8BC323B610023FB730023BB8100230F
:10A9E000FB753B681B7803F06003002B3AD0202BEB
:10A9F00040F097803B68DB88002B29D03B681B78B0
:10AA00005BB2002B11DA7B68D3F8C0329B683A68DE
:10AA1000507839693A68D288984739693B68DB8849
:10AA20001A46786801F0D6FA82E03B685A783B69AA
:10AA300083F800223B68DB88DAB23B6983F80122A5
:10AA400039693B68DB881A46786801F0EFFA6FE0F5
:10AA50007B68D3F8C0329B683A6850780022396826
:10AA6000984765E03B685B780B2B4FD801A252F802
:10AA700023F000BFA5AA00081BAB00080DAB00081F
:10AA80000DAB00080DAB00080DAB00080DAB0008C6
:10AA90000DAB00080DAB00080DAB0008CDAA0008F7
:10AAA000F5AA00087B6893F89C32032B07D107F1C5
:10AAB0000C0302221946786801F08CFA30E03968FC
:10AAC000786801F016FA0323FB7529E07B6893F898
:10AAD0009C32032B07D107F10F0301221946786836
:10AAE00001F078FA1CE03968786801F002FA032373
:10AAF000FB7515E07B6893F89C32032B0FD0396807
:10AB0000786801F0F6F90323FB7508E03968786886
:10AB100001F0EFF90323FB7502E000BF08E000BF7E
:10AB200006E03968786801F0E4F90323FB7500BF9B
:10AB3000FB7D18461837BD4680BD00BF80B584B088
:10AB400000AF78600B46FB707B68D3F8C432FB60C3
:10AB50007B68D3F8BC32002B01D1032349E07B682A
:10AB6000D3F8BC32BB60FA78796813469B00134473
:10AB70009B000B4418331B68002B29D0FA787968A6
:10AB800013469B0013449B000B4418331A68F97852
:10AB9000F8680B46DB005B1A9B00034444331B68D8
:10ABA000B2FBF3F101FB03F3D31A002B10D1FA78B7
:10ABB000796813469B0013449B000B441833002212
:10ABC0001A60F97800230022786859F0ECFB0FE056
:10ABD000BB680022C3F814227B68D3F8C0321B691B
:10ABE000BA68D2F80802BA6802F50471FA78984790
:10ABF000002318461037BD4680BD80B584B000AF35
:10AC000078600B46FB707B68D3F8BC32FB607B68D6
:10AC1000D3F8BC32002B01D1032315E0FB78194691
:10AC2000786859F002FC0246FB68C3F80C227B6886
:10AC3000D3F8C032DB68FA68D2F80402FA6802F589
:10AC4000037211469847002318461037BD4680BD51
:10AC500080B584B000AF78607B68D3F8BC32FB600D
:10AC60007B68D3F8C032002B15D0FB6893F8003214
:10AC7000FF2B10D07B68D3F8C0329B68FA6892F83B
:10AC80000002F968FA6892F8012292B29847FB68CC
:10AC9000FF2283F80022002318461037BD4680BDEE
:10ACA00080B483B000AF78607B6843221A80034B86
:10ACB00018460C37BD465DF8047B7047D80000206D
:10ACC00080B483B000AF78607B6843221A80034B66
:10ACD00018460C37BD465DF8047B70479400002091
:10ACE00080B483B000AF78607B6843221A80034B46
:10ACF00018460C37BD465DF8047B70471C010020E8
:10AD000080B483B000AF78607B680A221A80034B5E
:10AD100018460C37BD465DF8047B70475000002094
:10AD200080B483B000AF786039603B68002B01D1FC
:10AD3000032304E07B683A68C3F8C0220023184666
:10AD40000C37BD465DF8047B704780B487B000AF18
:10AD5000F860B9607A60FB68D3F8BC327B617B69CC
:10AD6000BA68C3F808227B697A68C3F81022002306
:10AD700018461C37BD465DF8047B704780B485B02B
:10AD800000AF786039607B68D3F8BC32FB60FB6849
:10AD90003A68C3F80422002318461437BD465DF80C
:10ADA000047B704780B584B000AF78607B68D3F8CF
:10ADB000BC32BB600123FB737B68D3F8BC32002B31
:10ADC00001D103231AE0BB68D3F81432002B14D14D
:10ADD000BB680122C3F81422BB68D3F810227B6839
:10ADE000DA62BB68D3F80822BB68D3F8103281213D
:10ADF000786859F0D8FA0023FB73FB7B18461037AC
:10AE0000BD4680BD80B584B000AF78607B68D3F864
:10AE1000BC32FB607B68D3F8BC32002B01D103232A
:10AE200016E07B681B7C002B09D1FB68D3F8042259
:10AE30004FF400730121786859F0D6FA07E0FB68F7
:10AE4000D3F8042240230121786859F0CDFA002379
:10AE500018461037BD4680BD80B586B000AFF8609B
:10AE6000B9601346FB71FB68002B01D1032325E079
:10AE7000FB68D3F8B832002B03D0FB680022C3F87C
:10AE8000B822FB68D3F8CC32002B03D0FB68002239
:10AE9000C3F8CC22BB68002B03D0FB68BA68C3F8A8
:10AEA000B422FB68012283F89C22FB68FA791A70AD
:10AEB000F86859F043F90346FB75FB7D18461837CF
:10AEC000BD4680BD80B584B000AF78603960002396
:10AED000FB813B68002B01D1032310E07B683A68BB
:10AEE000C3F8B8227B68D3F8B8329B6A07F10E0228
:10AEF0001046984702467B68C3F8CC2200231846C8
:10AF00001037BD4680BD80B582B000AF78607868EC
:10AF100059F060F9034618460837BD4680BD80B435
:10AF200083B000AF7860002318460C37BD465DF84B
:10AF3000047B704780B584B000AF78600B46FB702F
:10AF40000323FB737B68D3F8B832002B09D07B68EE
:10AF5000D3F8B8321B68FA781146786898470346E8
:10AF6000FB73FB7B18461037BD4680BD80B582B0B1
:10AF700000AF78600B46FB707B68D3F8B832002BCB
:10AF800007D07B68D3F8B8325B68FA7811467868E6
:10AF90009847002318460837BD4680BD80B584B069
:10AFA00000AF786039607B6803F2AA2339681846DD
:10AFB00000F065FF7B680122C3F894227B68B3F838
:10AFC000B0321A467B68C3F898227B6893F8AA329D
:10AFD00003F01F03022B1AD0022B22D8002B02D021
:10AFE000012B0AD01DE07B6803F2AA23194678687A
:10AFF00000F018FA0346FB7320E07B6803F2AA23F3
:10B000001946786800F07CFA0346FB7316E07B680B
:10B0100003F2AA231946786800F0BAFA0346FB73D4
:10B020000CE07B6893F8AA3223F07F03DBB2194669
:10B03000786859F02FF90346FB7300BFFB7B184675
:10B040001037BD4680BD80B586B000AFF8600B46B6
:10B050007A60FB72FB7A002B37D1FB6803F5AA7389
:10B060003B61FB68D3F89432032B4AD13B699A6861
:10B070003B69DB689A4213D93B699A683B69DB6894
:10B08000D21A3B699A603B69DA683B699B689342D4
:10B0900028BF13461A467968F86800F0E4FF30E0EC
:10B0A000FB68D3F8B8321B69002B0AD0FB6893F811
:10B0B0009C32032B05D1FB68D3F8B8321B69F868C2
:10B0C0009847F86800F0E0FF1BE0FB68D3F8B8325F
:10B0D0009B69002B13D0FB6893F89C32032B0ED195
:10B0E000FB68D3F8B8329B69FA7A1146F86898473A
:10B0F0000346FB75FB7D002B03D0FB7D02E00323A1
:10B1000000E0002318461837BD4680BD80B586B0E4
:10B1100000AFF8600B467A60FB72FB7A002B6AD1B5
:10B12000FB6814333B61FB68D3F89432022B55D192
:10B130003B699A683B69DB689A4214D93B699A6813
:10B140003B69DB68D21A3B699A603B699B681A4687
:10B150007968F86800F059FF002300220021F868A0
:10B1600059F042F93AE03B69DA683B699B689A42D8
:10B170001CD13B695A683B69DB689A4216D33B692C
:10B180005A68FB68D3F898329A420FD20022002105
:10B19000F86800F03AFFFB680022C3F89822002309
:10B1A00000220021F86859F01FF917E0FB68D3F876
:10B1B000B832DB68002B0AD0FB6893F89C32032B73
:10B1C00005D1FB68D3F8B832DB68F868984780216E
:10B1D000F86859F05FF8F86800F069FFFB6893F8C9
:10B1E000A032012B23D1F868FFF799FEFB680022FB
:10B1F00083F8A0221BE0FB68D3F8B8325B69002B10
:10B2000013D0FB6893F89C32032B0ED1FB68D3F864
:10B21000B8325B69FA7A1146F86898470346FB75BD
:10B22000FB7D002B03D0FB7D02E0032300E0002325
:10B2300018461837BD4680BD80B582B000AF786033
:10B240007B68012283F89C227B680022C3F8942249
:10B250007B6800225A607B680022C3F8A4227B68C6
:10B26000D3F8BC32002B09D07B68D3F8B8325B68C6
:10B270007A685268D2B21146786898474023002213
:10B280000021786858F0C1FF7B680122A3F864218F
:10B290007B684022C3F86021402300228021786827
:10B2A00058F0B3FF7B6801229A847B6840221A62BF
:10B2B000002318460837BD4680BD80B483B000AF78
:10B2C00078600B46FB707B68FA781A740023184686
:10B2D0000C37BD465DF8047B704780B483B000AF87
:10B2E00078607B6893F89C227B6883F89D227B685A
:10B2F000042283F89C22002318460C37BD465DF8D3
:10B30000047B704780B483B000AF78607B6893F8AB
:10B310009C32042B05D17B6893F89D227B6883F8CF
:10B320009C22002318460C37BD465DF8047B70470D
:10B3300080B582B000AF78607B6893F89C32032BB5
:10B340000BD17B68D3F8B832DB69002B05D07B6862
:10B35000D3F8B832DB697868984700231846083775
:10B36000BD4680BD80B483B000AF78600B46FB70F3
:10B37000002318460C37BD465DF8047B704780B447
:10B3800083B000AF78600B46FB70002318460C3783
:10B39000BD465DF8047B704780B483B000AF786031
:10B3A000002318460C37BD465DF8047B704780B516
:10B3B00082B000AF78607B68012283F89C227B68B2
:10B3C000D3F8B832002B09D07B68D3F8B8325B6869
:10B3D0007A685268D2B211467868984700231846B6
:10B3E0000837BD4680BD80B487B000AF78607B6809
:10B3F0007B617B691B787B827B6901337B617B6925
:10B400001B783B823B8A1B021AB2B7F912301343F6
:10B410001BB2FB81FB8918461C37BD465DF8047BD7
:10B420007047000080B584B000AF786039600023B9
:10B43000FB733B681B7803F06003402B05D0402B67
:10B4400053D8002B0BD0202B4FD17B68D3F8B832C8
:10B450009B683968786898470346FB734AE03B6805
:10B460005B78092B3BD801A252F823F0C1B4000845
:10B47000D5B40008DFB40008CBB40008DFB400087E
:10B480009FB4000895B40008DFB40008B7B4000802
:10B49000A9B400083968786800F0D8F924E0396860
:10B4A000786800F067FB1FE03968786800F0A6FB59
:10B4B0000346FB7318E03968786800F043FC13E03A
:10B4C0003968786800F073FC0EE03968786800F03D
:10B4D000A1FC09E03968786800F0B0FC04E0396844
:10B4E000786800F006FD00BF04E03968786800F075
:10B4F00000FD00BFFB7B18461037BD4680BD00BF76
:10B5000080B584B000AF786039600023FB733B687E
:10B510001B7803F06003402B05D0402B2ED8002B66
:10B5200001D0202B2AD17B6893F89C32013B022B5F
:10B530001DD83B689B88DBB2012B13D87B68D3F8FE
:10B54000B8329B683968786898470346FB733B6854
:10B55000DB88002B10D1FB7B002B0DD1786800F02D
:10B5600093FD09E03968786800F0C3FC04E03968AD
:10B57000786800F0BEFC00E000BF04E0396878683D
:10B5800000F0B7FC00BFFB7B18461037BD4680BDFE
:10B5900080B584B000AF786039600023FB733B68EE
:10B5A0009B88BB733B681B7803F06003402B07D07C
:10B5B000402B00F24081002B0CD0202B40F03B812F
:10B5C0007B68D3F8B8329B68396878689847034637
:10B5D000FB7335E13B685B78032B07D0032B00F34B
:10B5E0002481002B7BD0012B3BD01EE17B6893F89C
:10B5F0009C32022B02D0032B16D02CE0BB7B002BFD
:10B600000DD0BB7B802B0AD0BB7B1946786858F0E5
:10B6100041FE8021786858F03DFE00BF20E0396887
:10B62000786800F066FC1BE03B685B88002B0ED15D
:10B63000BB7B002B0BD0BB7B802B08D03B68DB880F
:10B64000002B04D1BB7B1946786858F023FE78683C
:10B6500000F01AFD04E03968786800F04AFC00BF89
:10B66000E8E07B6893F89C32022B02D0032B16D0C3
:10B670002EE0BB7B002B0DD0BB7B802B0AD0BB7B8D
:10B680001946786858F006FE8021786858F002FE66
:10B6900000BF23E03968786800F02BFC1EE03B68AF
:10B6A0005B88002B19D1BB7B03F07F03002B04D0F8
:10B6B000BB7B1946786858F00CFE786800F0E4FC13
:10B6C0007B68D3F8B8329B6839687868984704E09B
:10B6D0003968786800F00DFC00E000BFAAE07B68E4
:10B6E00093F89C32022B02D0032B32D097E0BB7B25
:10B6F000002B07D0BB7B802B04D03968786800F022
:10B70000F8FB91E097F90E30002B0BDABB7B03F0CE
:10B710007F0213469B0013449B0010337A68134446
:10B7200004330BE0BB7B03F07F0213469B00134402
:10B730009B0003F5A8737A6813440433BB60BB68AD
:10B7400000221A60BB6802221946786800F042FCA9
:10B750006AE097F90E30002B11DABB7B03F00F0281
:10B76000796813469B0013449B000B4424331B88C9
:10B77000002B17D13968786800F0BBFB54E0BB7B25
:10B7800003F00F02796813469B0013449B000B449F
:10B7900003F5B2731B88002B04D13968786800F078
:10B7A000A8FB41E097F90E30002B0BDABB7B03F0CE
:10B7B0007F0213469B0013449B0010337A681344A6
:10B7C00004330BE0BB7B03F07F0213469B00134462
:10B7D0009B0003F5A8737A6813440433BB60BB7BFA
:10B7E000002B02D0BB7B802B03D1BB6800221A60E8
:10B7F0000EE0BB7B1946786858F08AFD0346002BA3
:10B8000003D0BB6801221A6002E0BB6800221A6004
:10B81000BB6802221946786800F0DCFB04E0396856
:10B82000786800F066FB00BF04E03968786800F0D3
:10B8300060FB00BF04E03968786800F05AFB00BF85
:10B84000FB7B18461037BD4680BD000080B584B034
:10B8500000AF7860396000233B810023FB60002348
:10B86000FB723B685B881B0A9BB2013B0E2B00F20C
:10B87000528101A252F823F0E9B8000801B900088A
:10B8800041B9000817BB000817BB0008B7BA000889
:10B89000E3BA000817BB000817BB000817BB000875
:10B8A00017BB000817BB000817BB000817BB000830
:10B8B000B5B800087B68D3F8B432DB69002B0BD035
:10B8C0007B68D3F8B432DB697A68127C07F108012F
:10B8D00010469847F86026E13968786800F009FB5F
:10B8E000FB7A0133FB721EE17B68D3F8B4321B682C
:10B8F0007A68127C07F1080110469847F86012E157
:10B900007B681B7C002B0DD17B68D3F8B8329B6A17
:10B9100007F1080210469847F860FB6801330222DD
:10B920001A7000E17B68D3F8B832DB6A07F10802CD
:10B9300010469847F860FB68013302221A70F2E063
:10B940003B685B88DBB2052B00F2AC8001A252F8A9
:10B9500023F000BF6DB90008A1B90008D5B90008EF
:10B9600009BA00083DBA000871BA00087B68D3F82C
:10B97000B4325B68002B0BD07B68D3F8B4325B68C1
:10B980007A68127C07F1080110469847F86091E048
:10B990003968786800F0ADFAFB7A0133FB7289E010
:10B9A0007B68D3F8B4329B68002B0BD07B68D3F84C
:10B9B000B4329B687A68127C07F1080110469847F8
:10B9C000F86077E03968786800F093FAFB7A013321
:10B9D000FB726FE07B68D3F8B432DB68002B0BD0CE
:10B9E0007B68D3F8B432DB687A68127C07F108010F
:10B9F00010469847F8605DE03968786800F079FA99
:10BA0000FB7A0133FB7255E07B68D3F8B4321B69D3
:10BA1000002B0BD07B68D3F8B4321B697A68127C98
:10BA200007F1080110469847F86043E039687868E4
:10BA300000F05FFAFB7A0133FB723BE07B68D3F8DE
:10BA4000B4325B69002B0BD07B68D3F8B4325B69EE
:10BA50007A68127C07F1080110469847F86029E0DF
:10BA60003968786800F045FAFB7A0133FB7221E00F
:10BA70007B68D3F8B4329B69002B0BD07B68D3F87A
:10BA8000B4329B697A68127C07F108011046984726
:10BA9000F8600FE03968786800F02BFAFB7A013320
:10BAA000FB7207E03968786800F023FAFB7A01330B
:10BAB000FB7200BF37E07B681B7C002B09D17B68E1
:10BAC000D3F8B8325B6B07F1080210469847F8606C
:10BAD00029E03968786800F00CFAFB7A0133FB72D0
:10BAE00021E07B681B7C002B0DD17B68D3F8B8323A
:10BAF0001B6B07F1080210469847F860FB6801339A
:10BB000007221A700FE03968786800F0F2F9FB7AC2
:10BB10000133FB7207E03968786800F0EAF9FB7AD4
:10BB20000133FB7200BFFB7A002B1ED13B68DB8820
:10BB3000002B16D03B89002B0ED03B68DA883B895E
:10BB4000934228BF13469BB23B813B891A46F96852
:10BB5000786800F03FFA09E03968786800F0C9F9C0
:10BB600004E0786800F090FA00E000BF1037BD46AE
:10BB700080BD00BF80B584B000AF786039603B689D
:10BB80009B88002B30D13B68DB88002B2CD13B6895
:10BB90005B887F2B28D83B685B88DBB203F07F0390
:10BBA000FB737B6893F89C32032B04D13968786867
:10BBB00000F09FF91DE07B68FA7B83F89E22FB7BF7
:10BBC0001946786858F0D0FB786800F05DFAFB7B86
:10BBD000002B04D07B68022283F89C2209E07B685A
:10BBE000012283F89C2204E03968786800F081F92A
:10BBF00000BF00BF1037BD4680BD000080B584B0D7
:10BC000000AF786039600023FB733B685B88DAB271
:10BC10004B4B1A704A4B1B78012B05D93968786851
:10BC200000F067F9032387E07B6893F89C32022BCE
:10BC300002D0032B25D071E0414B1B78002B1CD088
:10BC40003F4B1B781A467B685A603D4B1B78194660
:10BC50007868FFF76FF90346FB73FB7B002B04D07A
:10BC60003968786800F045F965E0786800F00CFA0A
:10BC70007B68032283F89C225DE0786800F004FA78
:10BC800059E02F4B1B78002B12D17B68022283F8DE
:10BC90009C222B4B1B781A467B685A60284B1B78DA
:10BCA00019467868FFF762F9786800F0EDF942E02C
:10BCB000234B1B781A467B685B689A422AD07B68C4
:10BCC0005B68DBB219467868FFF750F91C4B1B78AC
:10BCD0001A467B685A601A4B1B7819467868FFF73A
:10BCE00029F90346FB73FB7B002B0FD0396878687A
:10BCF00000F0FFF87B685B68DBB219467868FFF7F5
:10BD000035F97B68022283F89C2214E0786800F001
:10BD1000BBF910E0786800F0B7F90CE03968786892
:10BD200000F0E7F8064B1B7819467868FFF71EF914
:10BD30000323FB7300BFFB7B18461037BD4680BD55
:10BD4000EC17002080B582B000AF786039603B68A6
:10BD5000DB88012B04D03968786800F0CAF822E04B
:10BD60007B6893F89C32022B02DC002B03DC15E08D
:10BD7000032B0BD012E07B6800229A607B680833AB
:10BD800001221946786800F025F90CE07B6804333D
:10BD900001221946786800F01DF904E039687868D6
:10BDA00000F0A7F800BF00BF0837BD4680BD80B5D2
:10BDB00082B000AF786039607B6893F89C32013BB9
:10BDC000022B1ED83B68DB88022B04D039687868C8
:10BDD00000F08FF81AE07B680122DA607B68D3F804
:10BDE000A432002B05D07B68DB6843F002027B683D
:10BDF000DA607B680C3302221946786800F0EAF8B2
:10BE000004E03968786800F074F800BF00BF0837B4
:10BE1000BD4680BD80B582B000AF786039603B68B8
:10BE20005B88012B06D17B680122C3F8A4227868C5
:10BE300000F02AF900BF0837BD4680BD80B582B04A
:10BE400000AF786039607B6893F89C32013B022B2D
:10BE50000BD83B685B88012B0CD17B680022C3F8B0
:10BE6000A422786800F010F904E03968786800F0DE
:10BE700040F800E000BF00BF0837BD4680BD80B578
:10BE800084B000AF786039603B68FB60FB681A786B
:10BE90007B681A70FB680133FB60FB681A787B686B
:10BEA0005A70FB680133FB60F868FFF79CFA0346A1
:10BEB0001A467B685A80FB680133FB60FB680133DC
:10BEC000FB60F868FFF78FFA03461A467B689A8092
:10BED000FB680133FB60FB680133FB60F868FFF728
:10BEE00082FA03461A467B68DA8000BF1037BD46E7
:10BEF00080BD80B582B000AF7860396080217868FD
:10BF000058F0C8F90021786858F0C4F900BF083724
:10BF1000BD4680BD80B586B000AFF860B9607A607C
:10BF20000023FB75FB68002B36D0FB683B6138694A
:10BF300000F036F8034601339BB25B009AB27B688F
:10BF40001A80FB7DBA6813447A6812781A70FB7DF8
:10BF50000133FB75FB7DBA68134403221A70FB7D25
:10BF60000133FB7513E0FB7DBA6813443A6912781C
:10BF70001A703B6901333B61FB7D0133FB75FB7D2F
:10BF8000BA68134400221A70FB7D0133FB753B69CC
:10BF90001B78002BE7D100E000BF1837BD4680BDFD
:10BFA00080B485B000AF78600023FB737B68BB6012
:10BFB00005E0FB7B0133FB73BB680133BB60BB68EF
:10BFC0001B78002BF5D1FB7B18461437BD465DF876
:10BFD000047B704780B584B000AFF860B9607A60C8
:10BFE000FB680222C3F89422FB687A689A61FB68B6
:10BFF0007A68DA617B68BA680021F86858F0D3F98A
:10C00000002318461037BD4680BD80B584B000AF10
:10C01000F860B9607A607B68BA680021F86858F007
:10C02000C2F9002318461037BD4680BD80B584B0E4
:10C0300000AFF860B9607A60FB680322C3F894220D
:10C04000FB687A68C3F85821FB687A68C3F85C21FA
:10C050007B68BA680021F86858F0C6F900231846D2
:10C060001037BD4680BD80B584B000AFF860B960C0
:10C070007A607B68BA680021F86858F0B5F9002347
:10C0800018461037BD4680BD80B582B000AF7860DD
:10C090007B680422C3F894220023002200217868E0
:10C0A00058F081F9002318460837BD4680BD80B599
:10C0B00082B000AF78607B680522C3F89422002329
:10C0C00000220021786858F08FF9002318460837BD
:10C0D000BD4680BD80B400AF00BFBD465DF8047BA7
:10C0E0007047000080B485B000AFEFF30583BB60FC
:10C0F000BB68002B0FD1EFF310837B607B68002BB4
:10C1000005D1EFF311833B603B68002B07D00E4B4A
:10C110001B68022B03D16FF00503FB600CE00A4B98
:10C120001B68002B05D1084B01221A600023FB601D
:10C1300002E04FF0FF33FB60FB6818461437BD4642
:10C140005DF8047B704700BFF017002080B584B015
:10C1500000AFEFF30583BB60BB68002B0FD1EFF39B
:10C1600010837B607B68002B05D1EFF311833B606C
:10C170003B68002B07D00F4B1B68022B03D16FF0DD
:10C180000503FB6010E00B4B1B68012B09D1FFF787
:10C19000A1FF084B02221A6001F03CFE0023FB6065
:10C1A00002E04FF0FF33FB60FB6818461037BD46D6
:10C1B00080BD00BFF017002080B590B004AFF860DC
:10C1C000B9607A6000233B61EFF30583FB61FB6993
:10C1D000002B40F08F80EFF31083BB61BB69002B15
:10C1E00005D1EFF311837B617B69002B03D0444BB6
:10C1F0001B68022B7ED0FB68002B7BD08023BB62A8
:10C2000018237B620023FB624FF0FF333B627B68A5
:10C21000002B45D07B681B68002B02D07B681B6815
:10C22000FB627B689B69002B02D07B689B697B6209
:10C230007B6A002B08D07B6A382B05D87B685B684B
:10C2400003F00103002B01D0002354E07B685B69FD
:10C25000002B03D07B685B699B08BB627B689B6893
:10C26000002B0ED07B68DB68BF2B0AD97B681B696B
:10C27000002B06D07B685B69002B02D001233B6258
:10C2800010E07B689B68002B0CD17B68DB68002B7F
:10C2900008D17B681B69002B04D100233B6201E0BD
:10C2A00000233B623B6A012B10D17B681B697A68D3
:10C2B0009268029201937B6A0093BB68BA6AF96A3A
:10C2C000F86801F0ADFB03463B6113E03B6A002BCD
:10C2D00010D1BB6A9AB207F1100301937B6A0093F5
:10C2E000BB68F96AF86801F0FEFB0346012B01D038
:10C2F00000233B613B6918463037BD4680BD00BF17
:10C30000F017002080B582B000AF02F0F5F9786038
:10C310007B6818460837BD4680BD000080B586B0F2
:10C3200000AF7860EFF305833B613B69002B0FD1D1
:10C33000EFF31083FB60FB68002B05D1EFF3118353
:10C34000BB60BB68002B07D00A4B1B68022B03D1D4
:10C350006FF005037B6107E000237B617B68002BA6
:10C3600002D0786801F020FD7B6918461837BD4679
:10C3700080BD00BFF017002080B58AB000AF7860A4
:10C3800000237B62EFF305833B613B69002B40F0A8
:10C390008580EFF31083FB60FB68002B05D1EFF382
:10C3A0001183BB60BB68002B03D03F4B1B68022B83
:10C3B00074D07B68002B03D07B685B683B6201E034
:10C3C00000233B623B6A03F00103002B02D00123F0
:10C3D000FB6101E00023FB613B6A03F00803002BD3
:10C3E0005CD14FF0FF33BB617B68002B15D07B68BD
:10C3F0009B68002B06D07B68DB684F2B02D901239A
:10C40000BB610CE07B689B68002B08D17B68DB6814
:10C41000002B04D10023BB6101E00023BB61BB6999
:10C42000012B12D1FB69002B07D07B689B68194652
:10C43000042000F0C0FC786216E07B689B68194617
:10C44000012000F0B8FC78620EE0BB69002B0BD134
:10C45000FB69002B04D0042000F095FC786203E017
:10C46000012000F090FC78627B6A002B0CD07B6886
:10C47000002B03D07B681B687B6101E000237B619C
:10C480007969786A01F06EFA7B6A002B06D0FB6945
:10C49000002B03D07B6A43F001037B627B6A184662
:10C4A0002837BD4680BD00BFF017002080B588B09A
:10C4B00000AF786039607B6823F00103BB617B6863
:10C4C00003F001037B610023FB61EFF305833B6114
:10C4D0003B69002B0FD1EFF31083FB60FB68002B4F
:10C4E00005D1EFF31183BB60BB68002B07D01D4B58
:10C4F0001B68022B03D16FF00503FB612CE0BB69C5
:10C50000002B03D16FF00303FB6125E07B69002B57
:10C5100011D03968B86900F09FFC0346012B1BD08D
:10C520003B68002B03D06FF00103FB6114E06FF058
:10C530000203FB6110E03968B86900F051FF03465F
:10C54000012B09D03B68002B03D06FF00103FB6186
:10C5500002E06FF00203FB61FB6918462037BD461D
:10C5600080BD00BFF017002080B588B000AF7860B4
:10C570007B6823F00103BB617B6803F001037B61EF
:10C580000023FB61EFF305833B613B69002B0FD177
:10C59000EFF31083FB60FB68002B05D1EFF31183F1
:10C5A000BB60BB68002B07D0164B1B68022B03D166
:10C5B0006FF00503FB611FE0BB69002B03D16FF037
:10C5C0000303FB6118E07B69002B09D0B86900F018
:10C5D0000DFC0346012B0FD06FF00203FB610BE053
:10C5E000002300220021B86900F06EFC0346012BF5
:10C5F00002D06FF00203FB61FB6918462037BD468D
:10C6000080BD00BFF017002080B58CB002AFF8608D
:10C61000B9607A6000237B62EFF30583BB61BB697D
:10C62000002B6FD1EFF310837B617B69002B05D169
:10C63000EFF311833B613B69002B03D0344B1B6844
:10C64000022B5FD0FB68002B5CD0BB68002B59D05D
:10C650004FF0FF333B627B68002B29D07B689B68DF
:10C66000002B12D07B68DB684F2B0ED97B681B69CF
:10C67000002B0AD07B685A69FB68B96801FB03F399
:10C680009A4202D301233B6214E07B689B68002B33
:10C6900010D17B68DB68002B0CD17B681B69002BF9
:10C6A00008D17B685B69002B04D100233B6201E069
:10C6B00000233B623B6A012B0BD17B681A697B68C4
:10C6C0009B6800210091B968F86800F05BFA786215
:10C6D00008E03B6A002B05D10022B968F86800F039
:10C6E000D3FA78627B6A002B0CD07B68002B03D0D6
:10C6F0007B681B68FB6101E00023FB61F969786AD4
:10C7000001F030F97B6A18462837BD4680BD00BF6E
:10C71000F017002080B58AB000AFF860B9603B60C8
:10C720001346FB71FB683B6200237B62EFF30583DA
:10C73000FB61FB69002B0FD1EFF31083BB61BB6979
:10C74000002B05D1EFF311837B617B69002B2CD08B
:10C75000284B1B68022B28D13B6A002B05D0BB68F5
:10C76000002B02D03B68002B03D06FF003037B62E9
:10C7700039E000233B6107F110020023B968386AF1
:10C7800000F0A8FC0346012B03D06FF002037B628C
:10C7900029E03B69002B26D0174B4FF080521A60DE
:10C7A000BFF34F8FBFF36F8F1DE03B6A002B02D0AA
:10C7B000BB68002B03D16FF003037B6214E00023FE
:10C7C0003A68B968386A00F07FFB0346012B0BD04A
:10C7D0003B68002B03D06FF001037B6204E06FF035
:10C7E00002037B6200E000BF7B6A18462837BD4623
:10C7F00080BD00BFF017002004ED00E080B58AB0D6
:10C8000000AFF860B9607A603B60FB683B62002370
:10C810007B62EFF30583FB61FB69002B0FD1EFF324
:10C820001083BB61BB69002B05D1EFF311837B61E2
:10C830007B69002B2CD0284B1B68022B28D13B6A2C
:10C84000002B05D0BB68002B02D03B68002B03D027
:10C850006FF003037B6238E000233B6107F11003B4
:10C860001A46B968386A00F0CFFE0346012B03D0A0
:10C870006FF002037B6228E03B69002B25D0174B49
:10C880004FF080521A60BFF34F8FBFF36F8F1CE0E1
:10C890003B6A002B02D0BB68002B03D16FF003036F
:10C8A0007B6213E03A68B968386A00F0B3FC03466B
:10C8B000012B0BD03B68002B03D06FF001037B6290
:10C8C00004E06FF002037B6200E000BF7B6A184661
:10C8D0002837BD4680BD00BFF017002004ED00E002
:10C8E00080B485B000AFF860B9607A60FB68074A31
:10C8F0001A60BB68064A1A607B6880221A6000BF13
:10C900001437BD465DF8047B704700BFF417002064
:10C91000B418002080B485B000AFF860B9607A60C8
:10C92000FB68074A1A60BB68064A1A607B684FF4C6
:10C9300080721A6000BF1437BD465DF8047B7047F3
:10C94000B41A0020741B002080B483B000AF78605C
:10C950007B6803F108027B685A607B684FF0FF3206
:10C960009A607B6803F108027B68DA607B6803F1F8
:10C9700008027B681A617B6800221A6000BF0C37CE
:10C98000BD465DF8047B704780B483B000AF78602B
:10C990007B6800221A6100BF0C37BD465DF8047B3E
:10C9A000704780B485B000AF786039607B685B68A1
:10C9B000FB603B68FA685A60FB689A683B689A605B
:10C9C000FB689B683A685A60FB683A689A603B6803
:10C9D0007A681A617B681B685A1C7B681A6000BF02
:10C9E0001437BD465DF8047B704780B485B000AF56
:10C9F000786039603B681B68BB60BB68B3F1FF3F80
:10CA000003D17B681B69FB600CE07B680833FB602B
:10CA100002E0FB685B68FB60FB685B681B68BA68E8
:10CA20009A42F6D2FB685A683B685A603B685B687A
:10CA30003A689A603B68FA689A60FB683A685A609C
:10CA40003B687A681A617B681B685A1C7B681A60AD
:10CA500000BF1437BD465DF8047B704780B485B0D5
:10CA600000AF78607B681B69FB607B685B687A68F5
:10CA700092689A607B689B687A6852685A60FB6823
:10CA80005B687A689A4203D17B689A68FB685A604F
:10CA90007B6800221A61FB681B685A1EFB681A60DB
:10CAA000FB681B6818461437BD465DF8047B704769
:10CAB00080B584B000AF786039607B68FB60FB684C
:10CAC000002B0CD14FF0500372B683F31188BFF3E3
:10CAD0006F8FBFF34F8F62B6BB6000BFFEE702F0FF
:10CAE0006DFCFB681A68FB68DB6BF968096C01FB7D
:10CAF00003F31A44FB689A60FB6800229A63FB68A0
:10CB00001A68FB685A60FB681A68FB68DB6B013BBC
:10CB1000F968096C01FB03F31A44FB68DA60FB68EF
:10CB2000FF2283F84420FB68FF2283F845203B68FE
:10CB3000002B14D1FB681B69002B1AD0FB68103343
:10CB4000184601F00FFC0346002B12D00C4B4FF09F
:10CB500080521A60BFF34F8FBFF36F8F09E0FB68FD
:10CB600010331846FFF7F0FEFB6824331846FFF732
:10CB7000EBFE02F057FC012318461037BD4680BD7E
:10CB800004ED00E080B58EB002AFF860B9607A6065
:10CB90003B60FB68002B0CD14FF0500372B683F35F
:10CBA0001188BFF36F8FBFF34F8F62B6BB6200BFB8
:10CBB000FEE73B68002B0CD14FF0500372B683F3B5
:10CBC0001188BFF36F8FBFF34F8F62B67B6200BFD8
:10CBD000FEE77B68002B02D0BB68002B01D001234D
:10CBE00000E00023002B0CD14FF0500372B683F30A
:10CBF0001188BFF36F8FBFF34F8F62B63B6200BFE8
:10CC0000FEE77B68002B02D1BB68002B01D101231A
:10CC100000E00023002B0CD14FF0500372B683F3D9
:10CC20001188BFF36F8FBFF34F8F62B6FB6100BFF8
:10CC3000FEE750237B617B69502B0CD04FF05003F3
:10CC400072B683F31188BFF36F8FBFF34F8F62B655
:10CC5000BB6100BFFEE77B693B68FB62FB6A002BA0
:10CC60000DD0FB6A012283F8462097F83820FB6A32
:10CC7000009313467A68B968F86800F047F8FB6AD1
:10CC800018463037BD4680BD80B58AB002AFF86027
:10CC9000B9601346FB71FB68002B0CD14FF05003B9
:10CCA00072B683F31188BFF36F8FBFF34F8F62B6F5
:10CCB0003B6100BFFEE7BB68002B02D10023FB6194
:10CCC00004E0FB68BA6802FB03F3FB61FB695033C5
:10CCD000184602F09FFCB861BB69002B11D0BB69FC
:10CCE0007B617B6950337B61BB69002283F84620FE
:10CCF000FA79BB69009313467A69B968F86800F05D
:10CD000005F8BB6918462037BD4680BD80B584B0A4
:10CD100000AFF860B9607A60FB70BB68002B03D18C
:10CD2000BB69BA691A6002E0BB697A681A60BB69BC
:10CD3000FA68DA63BB69BA681A640121B869FFF757
:10CD4000B7FEBB69FA7883F84C2000BF1037BD46A8
:10CD500080BD80B582B000AF78607B68002B0ED0BC
:10CD60007B6800229A607B6800221A607B68002240
:10CD7000DA60002300220021786800F0A5F800BFE7
:10CD80000837BD4680BD80B586B000AF0346FB7155
:10CD900001237B6100233B61FB791A46396978697D
:10CDA000FFF772FFF860F868FFF7D3FFFB681846DB
:10CDB0001837BD4680BD80B588B002AF03463960E4
:10CDC000FB7101237B6100233B61FB7900933B688E
:10CDD000002239697869FFF7D5FEF860F868FFF737
:10CDE000B8FFFB6818461837BD4680BD90B587B0C0
:10CDF00000AF78607B683B613B69002B0CD14FF042
:10CE0000500372B683F31188BFF36F8FBFF34F8F58
:10CE100062B6FB6000BFFEE73B699C6801F06CFCFA
:10CE200003469C4211D13B69DB685A1E3B69DA60BC
:10CE30003B69DB68002B05D1002300220021386903
:10CE400000F042F801237B6101E000237B617B69F4
:10CE500018461C37BD4690BD90B587B000AF7860CE
:10CE600039607B683B613B69002B0CD14FF050036C
:10CE700072B683F31188BFF36F8FBFF34F8F62B623
:10CE8000FB6000BFFEE73B699C6801F035FC034690
:10CE90009C4207D13B69DB685A1C3B69DA6001237D
:10CEA0007B610CE03968386900F09AFA78617B6937
:10CEB000002B04D03B69DB685A1C3B69DA607B6954
:10CEC00018461C37BD4690BD80B58EB000AFF860E7
:10CED000B9607A603B6000237B63FB683B633B6B1C
:10CEE000002B0CD14FF0500372B683F31188BFF3BF
:10CEF0006F8FBFF34F8F62B6BB6200BFFEE7BB68A8
:10CF0000002B03D13B6B1B6C002B01D1012300E0F4
:10CF10000023002B0CD14FF0500372B683F311881D
:10CF2000BFF36F8FBFF34F8F62B67B6200BFFEE728
:10CF30003B68022B03D13B6BDB6B012B01D101233F
:10CF400000E00023002B0CD14FF0500372B683F3A6
:10CF50001188BFF36F8FBFF34F8F62B63B6200BF84
:10CF6000FEE701F0D9FB0346002B02D17B68002BC2
:10CF700001D1012300E00023002B0CD14FF050031E
:10CF800072B683F31188BFF36F8FBFF34F8F62B612
:10CF9000FB6100BFFEE702F011FA3B6B9A6B3B6B43
:10CFA000DB6B9A4202D33B68022B29D13A68B968FD
:10CFB000386B00F0C7FBF8623B6B5B6A002B10D04C
:10CFC0003B6B2433184601F0CDF90346002B13D0F8
:10CFD0003F4B4FF080521A60BFF34F8FBFF36F8FFC
:10CFE0000AE0FB6A002B07D0394B4FF080521A60E1
:10CFF000BFF34F8FBFF36F8F02F014FA012363E08A
:10D000007B68002B03D102F00DFA00235CE07B6B00
:10D01000002B06D107F11403184601F009FA012389
:10D020007B6302F0FFF900F069FF02F0C7F93B6B88
:10D0300093F844305BB2B3F1FF3F03D13B6B002266
:10D0400083F844203B6B93F845305BB2B3F1FF3F6C
:10D0500003D13B6B002283F8452002F0E3F93A1D2F
:10D0600007F114031146184601F0F8F90346002BA6
:10D0700024D1386B00F05EFC0346002B18D03B6BCC
:10D0800010337A681146184601F018F9386B00F031
:10D09000E9FB00F041FF0346002B7FF47CAF0C4B13
:10D0A0004FF080521A60BFF34F8FBFF36F8F72E75C
:10D0B000386B00F0D7FB00F02FFF6CE7386B00F007
:10D0C000D1FB00F029FF002318463837BD4680BD4C
:10D0D00004ED00E080B58EB000AFF860B9607A6012
:10D0E0003B60FB683B633B6B002B0CD14FF0500364
:10D0F00072B683F31188BFF36F8FBFF34F8F62B6A1
:10D100007B6200BFFEE7BB68002B03D13B6B1B6C4F
:10D11000002B01D1012300E00023002B0CD14FF0A4
:10D12000500372B683F31188BFF36F8FBFF34F8F35
:10D1300062B63B6200BFFEE73B68022B03D13B6B4C
:10D14000DB6B012B01D1012300E00023002B0CD16C
:10D150004FF0500372B683F31188BFF36F8FBFF3A4
:10D160004F8F62B6FB6100BFFEE702F00FFAEFF3EC
:10D1700011824FF0500372B683F31188BFF36F8FA3
:10D18000BFF34F8F62B6BA617B61BB69FB623B6BD9
:10D190009A6B3B6BDB6B9A4202D33B68022B2CD120
:10D1A0003B6B93F8453087F82B303A68B968386B99
:10D1B00000F0C8FA97F92B30B3F1FF3F12D13B6B67
:10D1C0005B6A002B16D03B6B2433184601F0CAF87B
:10D1D0000346002B0ED07B68002B0BD07B6801220E
:10D1E0001A6007E097F82B300133DBB25AB23B6B81
:10D1F00083F8452001237B6301E000237B63FB6A06
:10D200003B613B6983F3118800BF7B6B184638375D
:10D21000BD4680BD80B58CB000AFF860B9607A6063
:10D220000023FB62FB68BB62BB6A002B0CD14FF092
:10D23000500372B683F31188BFF36F8FBFF34F8F24
:10D2400062B63B6200BFFEE7BB68002B03D1BB6A3E
:10D250001B6C002B01D1012300E00023002B0CD11B
:10D260004FF0500372B683F31188BFF36F8FBFF393
:10D270004F8F62B6FB6100BFFEE701F04DFA034637
:10D28000002B02D17B68002B01D1012300E0002399
:10D29000002B0CD14FF0500372B683F31188BFF30B
:10D2A0006F8FBFF34F8F62B6BB6100BFFEE702F026
:10D2B00085F8BB6A9B6B7B627B6A002B1FD0B968C9
:10D2C000B86A00F0A9FA7B6A5A1EBB6A9A63BB6A05
:10D2D0001B69002B0FD0BB6A1033184601F042F8CF
:10D2E0000346002B07D03D4B4FF080521A60BFF32E
:10D2F0004F8FBFF36F8F02F095F8012369E07B68D1
:10D30000002B03D102F08EF8002362E0FB6A002BB1
:10D3100006D107F11003184601F08AF80123FB62D9
:10D3200002F080F800F0EAFD02F048F8BB6A93F8DA
:10D3300044305BB2B3F1FF3F03D1BB6A002283F8F4
:10D340004420BB6A93F845305BB2B3F1FF3F03D191
:10D35000BB6A002283F8452002F064F83A1D07F109
:10D3600010031146184601F079F80346002B23D12B
:10D37000B86A00F0C9FA0346002B17D0BB6A243301
:10D380007A681146184600F099FFB86A00F06AFA08
:10D3900000F0C2FD0346002B89D1104B4FF08052A4
:10D3A0001A60BFF34F8FBFF36F8F80E7B86A00F04A
:10D3B00059FA00F0B1FD7AE7B86A00F053FA00F0CC
:10D3C000ABFDB86A00F0A0FA0346002B3FF46FAF44
:10D3D000002318463037BD4680BD00BF04ED00E095
:10D3E00080B58EB000AF7860396000237B637B68C6
:10D3F000FB6200233B63FB6A002B0CD14FF0500310
:10D4000072B683F31188BFF36F8FBFF34F8F62B68D
:10D410003B6200BFFEE7FB6A1B6C002B0CD04FF099
:10D42000500372B683F31188BFF36F8FBFF34F8F32
:10D4300062B6FB6100BFFEE701F06EF90346002B08
:10D4400002D13B68002B01D1012300E00023002B17
:10D450000CD14FF0500372B683F31188BFF36F8F76
:10D46000BFF34F8F62B6BB6100BFFEE701F0A6FFBE
:10D47000FB6A9B6BBB62BB6A002B24D0BB6A5A1E43
:10D48000FB6A9A63FB6A1B68002B04D101F0C2FAA5
:10D490000246FB6A9A60FB6A1B69002B0FD0FB6A8D
:10D4A0001033184600F05EFF0346002B07D0554BA3
:10D4B0004FF080521A60BFF34F8FBFF36F8F01F0B0
:10D4C000B1FF012399E03B68002B13D13B6B002B8C
:10D4D0000CD04FF0500372B683F31188BFF36F8FF7
:10D4E000BFF34F8F62B67B6100BFFEE701F09AFF8A
:10D4F000002382E07B6B002B06D107F10C0318465A
:10D5000000F096FF01237B6301F08CFF00F0F6FC36
:10D5100001F054FFFB6A93F844305BB2B3F1FF3F74
:10D5200003D1FB6A002283F84420FB6A93F845305C
:10D530005BB2B3F1FF3F03D1FB6A002283F84520C1
:10D5400001F070FF3A4607F10C031146184600F04F
:10D5500085FF0346002B32D1F86A00F0D5F9034667
:10D56000002B26D0FB6A1B68002B09D101F026FF97
:10D57000FB6A9B68184601F0EDF8386301F052FF32
:10D58000FB6A24333A681146184600F097FEF86AA1
:10D5900000F068F900F0C0FC0346002B7FF466AF92
:10D5A000184B4FF080521A60BFF34F8FBFF36F8F4D
:10D5B0005CE7F86A00F056F900F0AEFC56E7F86A4E
:10D5C00000F050F900F0A8FCF86A00F09DF903465D
:10D5D000002B3FF44BAF3B6B002B0DD001F0EEFE68
:10D5E000F86A00F097F87862FB6A9B68796A1846D7
:10D5F00001F08AF901F016FF002318463837BD46BE
:10D6000080BD00BF04ED00E080B58EB000AFF860D3
:10D61000B9607A60FB683B633B6B002B0CD14FF029
:10D62000500372B683F31188BFF36F8FBFF34F8F30
:10D6300062B63B6200BFFEE7BB68002B03D13B6BC9
:10D640001B6C002B01D1012300E00023002B0CD127
:10D650004FF0500372B683F31188BFF36F8FBFF39F
:10D660004F8F62B6FB6100BFFEE701F08FFFEFF363
:10D6700011824FF0500372B683F31188BFF36F8F9E
:10D68000BFF34F8F62B6BA617B61BB69FB623B6BD4
:10D690009B6BBB62BB6A002B2FD03B6B93F8443073
:10D6A00087F82730B968386B00F0B6F8BB6A5A1EA5
:10D6B0003B6B9A6397F92730B3F1FF3F12D13B6B75
:10D6C0001B69002B16D03B6B1033184600F04AFE46
:10D6D0000346002B0ED07B68002B0BD07B68012209
:10D6E0001A6007E097F827300133DBB25AB23B6B80
:10D6F00083F8442001237B6301E000237B63FB6A02
:10D700003B613B6983F3118800BF7B6B1846383758
:10D71000BD4680BD80B485B000AF78607B685B6A31
:10D72000002B06D07B681B6B1B68C3F13803FB60C2
:10D7300001E00023FB60FB6818461437BD465DF826
:10D74000047B704780B586B000AFF860B9607A603E
:10D7500000237B61FB689B6B3B61FB681B6C002BB0
:10D760000DD1FB681B68002B4DD1FB689B681846E8
:10D7700001F058F87861FB6800229A6043E07B680A
:10D78000002B19D1FB685868FB681B6C1A46B968F6
:10D7900076F0F8FCFB685A68FB681B6C1A44FB685F
:10D7A0005A60FB685A68FB689B689A422BD3FB68F7
:10D7B0001A68FB685A6026E0FB68D868FB681B6C37
:10D7C0001A46B96876F0DEFCFB68DA68FB681B6C09
:10D7D0005B421A44FB68DA60FB68DA68FB681B6826
:10D7E0009A4207D2FB689A68FB681B6C5B421A443A
:10D7F000FB68DA607B68022B05D13B69002B02D005
:10D800003B69013B3B613B695A1CFB689A637B693E
:10D8100018461837BD4680BD80B582B000AF78602D
:10D8200039607B681B6C002B18D07B68DA687B68DA
:10D830001B6C1A447B68DA607B68DA687B689B68DB
:10D840009A4203D37B681A687B68DA607B68D96880
:10D850007B681B6C1A46386876F094FC00BF08376A
:10D86000BD4680BD80B584B000AF786001F0A6FDF4
:10D870007B6893F84530FB7311E07B685B6A002B93
:10D8800012D07B682433184600F06CFD0346002B51
:10D8900001D000F049FEFB7B013BDBB2FB7397F943
:10D8A0000F30002BE9DC00E000BF7B68FF2283F82B
:10D8B000452001F0B7FD01F081FD7B6893F844300D
:10D8C000BB7311E07B681B69002B12D07B6810339F
:10D8D000184600F047FD0346002B01D000F024FE5F
:10D8E000BB7B013BDBB2BB7397F90E30002BE9DC4D
:10D8F00000E000BF7B68FF2283F8442001F092FD26
:10D9000000BF1037BD4680BD80B584B000AF7860E1
:10D9100001F054FD7B689B6B002B02D10123FB605F
:10D9200001E00023FB6001F07DFDFB681846103725
:10D93000BD4680BD80B584B000AF786001F03EFD8B
:10D940007B689A6B7B68DB6B9A4202D10123FB6098
:10D9500001E00023FB6001F065FDFB68184610370D
:10D96000BD4680BD80B485B000AF786039600023CB
:10D97000FB6014E00F4AFB6852F83330002B0BD1E8
:10D980000C49FB683A6841F833200A4AFB68DB001F
:10D9900013447A685A6006E0FB680133FB60FB6859
:10D9A000072BE7D900BF00BF1437BD465DF8047BE5
:10D9B000704700BF741F002080B586B000AFF860CC
:10D9C000B9607A60FB687B6101F0F8FC7B6993F8D1
:10D9D00044305BB2B3F1FF3F03D17B69002283F88F
:10D9E00044207B6993F845305BB2B3F1FF3F03D12C
:10D9F0007B69002283F8452001F014FD7B699B6B55
:10DA0000002B06D17B6924337A68B968184600F088
:10DA10007BFC7869FFF726FF00BF1837BD4680BD45
:10DA200080B58EB004AFF860B9607A603B607B6B04
:10DA3000002B0CD14FF0500372B683F31188BFF363
:10DA40006F8FBFF34F8F62B63B6200BFFEE7BB6BC9
:10DA5000002B0CD14FF0500372B683F31188BFF343
:10DA60006F8FBFF34F8F62B6FB6100BFFEE7C0232D
:10DA70003B613B69C02B0CD04FF0500372B683F36F
:10DA80001188BFF36F8FBFF34F8F62B6BB6100BFCA
:10DA9000FEE73B69BB6B002B1ED07B6B002B1BD0C2
:10DAA000BB6B7B627B6A7A6B1A637B6A022283F8A8
:10DAB000BD20002303937B6A029307F114030193B3
:10DAC0003B6B00933B687A68B968F86800F050F8DF
:10DAD000786A00F0F9F801E000237B617B69184661
:10DAE0002837BD4680BD80B58CB004AFF860B96002
:10DAF0003B601346FB80FB889B00184601F08AFDC3
:10DB000078617B69002B0ED0C02001F083FDF861A5
:10DB1000FB69002B03D0FB697A691A6305E0786919
:10DB200001F042FE01E00023FB61FB69002B17D0EE
:10DB3000FB69002283F8BD20FA8800230393FB6968
:10DB40000293FB6A0193BB6A00933B68B968F8686B
:10DB500000F00EF8F86900F0B7F80123BB6102E0AD
:10DB60004FF0FF33BB61BB6918462037BD4680BD0F
:10DB700080B588B000AFF860B9607A603B603B6BFD
:10DB8000186B7B689B001A46A52176F023FB3B6B44
:10DB90001A6B79686FF040430B449B001344BB61E0
:10DBA000BB6923F00703BB61BB6903F00703002BCC
:10DBB0000CD04FF0500372B683F31188BFF36F8F10
:10DBC000BFF34F8F62B67B6100BFFEE7BB68002BDF
:10DBD0001FD00023FB6112E0BA68FB691344197877
:10DBE0003A6BFB69134434330A461A70BA68FB690E
:10DBF00013441B78002B06D0FB690133FB61FB69E2
:10DC00000F2BE9D900E000BF3B6B002283F84320D3
:10DC100003E03B6B002283F83420BB6A372B01D929
:10DC20003723BB623B6BBA6ADA623B6BBA6ADA646F
:10DC30003B6B00221A653B6B04331846FEF7A4FECB
:10DC40003B6B18331846FEF79FFE3B6B3A6B1A612D
:10DC5000BB6AC3F138023B6B9A613B6B3A6B5A6209
:10DC60003B6B00225A653B6B0022C3F8B8203B6B2C
:10DC7000002283F8BC203B6B5833602200211846F9
:10DC800076F0A8FA3B6B0D4ADA653B6B0C4A1A66D4
:10DC90003B6B0C4A5A663A68F968B86901F07EFA3B
:10DCA00002463B6B1A60FB6A002B02D0FB6A3A6BA0
:10DCB0001A6000BF2037BD4680BD00BF80390A080A
:10DCC000A0390A0860390A0880B582B000AF7860D0
:10DCD00001F074FB2D4B1B6801332C4A13602C4B55
:10DCE0001B68002B09D12A4A7B681360274B1B68ED
:10DCF000012B10D100F03CFC0DE0264B1B68002BE3
:10DD000009D1234B1B68DA6A7B68DB6A9A4202D826
:10DD10001F4A7B681360204B1B6801331E4A136047
:10DD20001D4B1A687B685A647B68DA6A1B4B1B6858
:10DD30009A4203D97B68DB6A184A13607B68DA6A07
:10DD400013469B0013449B00154A1A447B68043316
:10DD500019461046FEF725FE01F064FB0D4B1B68CB
:10DD6000002B0ED00A4B1B68DA6A7B68DB6A9A428A
:10DD700007D20C4B4FF080521A60BFF34F8FBFF3A6
:10DD80006F8F00BF0837BD4680BD00BF88240020CC
:10DD9000B41F002094240020A424002090240020FC
:10DDA000B81F002004ED00E080B584B000AF7860BB
:10DDB0000023FB607B68002B19D0144B1B68002BE1
:10DDC0000CD04FF0500372B683F31188BFF36F8FFE
:10DDD000BFF34F8F62B6BB6000BFFEE700F08EF866
:10DDE0000021786800F02AFE00F096F8F860FB68E1
:10DDF000002B07D1064B4FF080521A60BFF34F8FB4
:10DE0000BFF36F8F00BF1037BD4680BDB024002028
:10DE100004ED00E080B58AB004AF0023BB600023AE
:10DE20007B603A46391D07F108031846FEF758FD96
:10DE300039687B68BA68029201930023009300233B
:10DE40000A4626492648FFF7EBFD0346254A13609C
:10DE5000244B1B68002B02D001237B6101E00023CF
:10DE60007B617B69012B02D100F03CFE78617B690C
:10DE7000012B1DD14FF0500372B683F31188BFF30D
:10DE80006F8FBFF34F8F62B63B6100BF164B1B68AD
:10DE90005833164A1360164B4FF0FF321A60154B79
:10DEA00001221A60144B00221A6001F009FA10E0F6
:10DEB0007B69B3F1FF3F0CD14FF0500372B683F38F
:10DEC0001188BFF36F8FBFF34F8F62B6FB6000BF47
:10DED000FEE700BF1837BD4680BD00BF44C3080839
:10DEE00041E50008AC240020B41F0020A41100204C
:10DEF000A8240020942400208C24002080B400AFAB
:10DF0000044B1B680133034A136000BFBD465DF834
:10DF1000047B7047B024002080B584B000AF00239C
:10DF2000FB600023BB60434B1B68002B0CD14FF000
:10DF3000500372B683F31188BFF36F8FBFF34F8F17
:10DF400062B63B6000BFFEE701F038FA394B1B6850
:10DF5000013B384A1360374B1B68002B62D1364BAC
:10DF60001B68002B5ED02FE0344BDB68DB68FB6066
:10DF7000FB6818331846FEF771FDFB68043318463A
:10DF8000FEF76CFDFB68DA6A2D4B1B689A4203D9D9
:10DF9000FB68DB6A2A4A1360FB68DA6A13469B0057
:10DFA00013449B00274A1A44FB6804331946104661
:10DFB000FEF7F7FCFB68DA6A234B1B68DB6A9A42C0
:10DFC00002D3224B01221A601C4B1B68002BCBD1C1
:10DFD000FB68002B01D000F06FFB1D4B1B687B60C2
:10DFE0007B68002B10D000F047F80346002B02D0CE
:10DFF000164B01221A607B68013B7B607B68002B1B
:10E00000F1D1134B00221A60104B1B68002B09D072
:10E010000123BB600F4B4FF080521A60BFF34F8F4C
:10E02000BFF36F8F01F0FEF9BB6818461037BD468D
:10E0300080BD00BFB0240020882400204824002098
:10E0400090240020B81F0020B41F00209C24002032
:10E050009824002004ED00E080B483B000AF054BAD
:10E060001B687B607B6818460C37BD465DF8047BF7
:10E07000704700BF8C24002080B586B000AF00231D
:10E080007B61504B1B68002B40F08B804E4B1B6814
:10E0900001333B614C4A3B6913603B69002B22D141
:10E0A0004A4B1B681B68002B0CD04FF0500372B614
:10E0B00083F31188BFF36F8FBFF34F8F62B63B605E
:10E0C00000BFFEE7414B1B68FB60414B1B683F4AAA
:10E0D00013603F4AFB6813603E4B1B6801333D4AA7
:10E0E000136000F0E9FA3C4B1B683A699A4249D345
:10E0F000364B1B681B68002B04D1374B4FF0FF32A7
:10E100001A603FE0314B1B68DB68DB68BB60BB68B3
:10E110005B687B603A697B689A4203D22E4A7B68CF
:10E1200013602FE0BB6804331846FEF797FCBB680A
:10E130009B6A002B04D0BB6818331846FEF78EFC90
:10E14000BB68DA6A254B1B689A4203D9BB68DB6A55
:10E15000224A1360BB68DA6A13469B0013449B0093
:10E160001F4A1A44BB68043319461046FEF719FCCF
:10E17000BB68DA6A1B4B1B68DB6A9A42B8D301237F
:10E180007B61B5E7174B1B68DA6A154913469B009C
:10E1900013449B000B441B68012B07D901237B61AF
:10E1A00004E0114B1B6801330F4A13600F4B1B68CF
:10E1B000002B01D001237B617B6918461837BD46CF
:10E1C00080BD00BFB02400208C240020402400200B
:10E1D00044240020A0240020A82400209024002013
:10E1E000B81F0020B41F0020982400209C24002089
:10E1F00080B485B000AF2B4B1B68002B03D02A4B9B
:10E2000001221A6048E0284B00221A60274B1B6845
:10E21000FB6012E0FB68002B0CD14FF0500372B68C
:10E2200083F31188BFF36F8FBFF34F8F62B67B60AC
:10E2300000BFFEE7FB68013BFB601D49FA6813461F
:10E240009B0013449B000B441B68002BE2D0FA6830
:10E2500013469B0013449B00154A1344BB60BB68E4
:10E260005B685A68BB685A60BB685A68BB68083309
:10E270009A4204D1BB685B685A68BB685A60BB6845
:10E280005B68DB680B4A1360084AFB681360094B44
:10E290001B685833084A136000BF1437BD465DF849
:10E2A000047B7047B02400209C2400209024002090
:10E2B000B81F0020B41F0020A411002080B584B036
:10E2C00000AF786039607B68002B0CD14FF05003B1
:10E2D00072B683F31188BFF36F8FBFF34F8F62B6AF
:10E2E000FB6000BFFEE7074B1B68183319467868D0
:10E2F000FEF77BFB0121386800F0A0FB00BF103760
:10E30000BD4680BDB41F002080B586B000AFF86068
:10E31000B9607A60FB68002B0CD14FF0500372B6E5
:10E3200083F31188BFF36F8FBFF34F8F62B67B61AA
:10E3300000BFFEE70A4B1B6818331946F868FEF762
:10E3400030FB7B68002B02D04FF0FF33BB60796855
:10E35000B86800F073FB00BF1837BD4680BD00BF32
:10E36000B41F002080B586B000AF78607B68DB68A2
:10E37000DB683B613B69002B0CD14FF0500372B658
:10E3800083F31188BFF36F8FBFF34F8F62B6FB60CB
:10E3900000BFFEE73B6918331846FEF75FFB1E4BD4
:10E3A0001B68002B1DD13B6904331846FEF756FB52
:10E3B0003B69DA6A194B1B689A4203D93B69DB6AED
:10E3C000164A13603B69DA6A13469B0013449B00AC
:10E3D000134A1A443B69043319461046FEF7E1FA22
:10E3E00005E03B69183319460E48FEF7DAFA3B6937
:10E3F000DA6A0D4B1B68DB6A9A4205D901237B61FF
:10E400000A4B01221A6001E000237B617B691846F8
:10E410001837BD4680BD00BFB024002090240020E6
:10E42000B81F002048240020B41F00209C24002096
:10E4300080B483B000AF7860064B1A687B681A60BE
:10E44000054B1A687B685A6000BF0C37BD465DF803
:10E45000047B7047A02400208C24002080B588B065
:10E4600000AF786039607B68002B0CD14FF050030F
:10E4700072B683F31188BFF36F8FBFF34F8F62B60D
:10E480003B6100BFFEE73B68002B0CD14FF050030F
:10E4900072B683F31188BFF36F8FBFF34F8F62B6ED
:10E4A000FB6000BFFEE700F089FF1D4B1B68BB61EE
:10E4B0007B685B68BA69D31A7B613B681B68B3F100
:10E4C000FF3F02D10023FB6123E07B681A68154BF4
:10E4D0001B689A4207D07B685B68BA699A4202D38C
:10E4E0000123FB6115E03B681B687A699A420BD2F5
:10E4F0003B681A687B69D21A3B681A607868FFF734
:10E5000097FF0023FB6104E03B6800221A600123AF
:10E51000FB6100F087FFFB6918462037BD4680BDD0
:10E520008C240020A024002080B400AF034B0122E3
:10E530001A6000BFBD465DF8047B70479C24002034
:10E5400080B582B000AF786000F052F8064B1B68CF
:10E55000012BF9D9054B4FF080521A60BFF34F8F52
:10E56000BFF36F8FF0E700BFB81F002004ED00E09D
:10E5700080B582B000AF00237B600CE07A68134660
:10E580009B0013449B00124A13441846FEF7DCF923
:10E590007B6801337B607B68372BEFD90D48FEF732
:10E5A000D3F90D48FEF7D0F90C48FEF7CDF90C4829
:10E5B000FEF7CAF90B48FEF7C7F90B4B054A1A607C
:10E5C0000A4B054A1A6000BF0837BD4680BD00BF30
:10E5D000B81F0020182400202C24002048240020EC
:10E5E0005C240020742400204024002044240020C7
:10E5F00080B582B000AF19E000F0E0FE104BDB68A0
:10E60000DB687B607B6804331846FEF727FA0D4B06
:10E610001B68013B0B4A13600B4B1B68013B0A4A0A
:10E62000136000F0FFFE786800F010F8064B1B68DE
:10E63000002BE1D100BF00BF0837BD4680BD00BF41
:10E640005C240020882400207024002080B584B041
:10E6500000AF78607B685833184676F0DDFC7B6845
:10E6600093F8BD30002B08D17B681B6B184601F076
:10E670009BF8786801F098F81AE07B6893F8BD3051
:10E68000012B03D1786801F08FF811E07B6893F8D3
:10E69000BD30022B0CD04FF0500372B683F31188BB
:10E6A000BFF36F8FBFF34F8F62B6FB6000BFFEE713
:10E6B00000BF1037BD4680BD80B483B000AF0C4BA7
:10E6C0001B681B68002B04D10A4B4FF0FF321A6005
:10E6D00008E0074B1B68DB68DB687B607B685B6876
:10E6E000044A136000BF0C37BD465DF8047B7047D9
:10E6F00040240020A824002080B483B000AF054B44
:10E700001B687B607B6818460C37BD465DF8047B50
:10E71000704700BFB41F002080B483B000AF0B4B24
:10E720001B68002B02D101237B6008E0084B1B68AB
:10E73000002B02D102237B6001E000237B607B6819
:10E7400018460C37BD465DF8047B704794240020C2
:10E75000B024002080B584B000AF78607B68BB60D7
:10E760000023FB607B68002B51D0BB68DA6A2A4B20
:10E770001B68DB6A9A4241D2BB689B69002B06DBAF
:10E78000254B1B68DB6AC3F13802BB689A61BB6822
:10E790005969BB68DA6A13469B0013449B001F4A01
:10E7A0001344994222D1BB6804331846FEF756F948
:10E7B000194B1B68DA6ABB68DA62BB68DA6A184B05
:10E7C0001B689A4203D9BB68DB6A154A1360BB68B1
:10E7D000DA6A13469B0013449B00104A1A44BB6834
:10E7E000043319461046FEF7DCF804E00A4B1B68B8
:10E7F000DA6ABB68DA620123FB6008E0BB68DA6CA6
:10E80000054B1B68DB6A9A4201D20123FB60FB685F
:10E8100018461037BD4680BDB41F0020B81F002029
:10E820009024002080B586B000AF78607B683B61A3
:10E8300000237B617B68002B5AD0304B1B683A6900
:10E840009A420CD04FF0500372B683F31188BFF395
:10E850006F8FBFF34F8F62B6FB6000BFFEE73B696F
:10E860001B6D002B0CD14FF0500372B683F311884F
:10E87000BFF36F8FBFF34F8F62B6BB6000BFFEE781
:10E880003B691B6D5A1E3B691A653B69DA6A3B6935
:10E89000DB6C9A422CD03B691B6D002B28D13B6965
:10E8A00004331846FEF7DAF83B69DA6C3B69DA6242
:10E8B0003B69DB6AC3F138023B699A613B69DA6AFA
:10E8C0000F4B1B689A4203D93B69DB6A0C4A136001
:10E8D0003B69DA6A13469B0013449B00094A1A44B9
:10E8E0003B69043319461046FEF75BF801237B6150
:10E8F0007B6918461837BD4680BD00BFB41F002095
:10E9000090240020B81F002080B588B000AF786048
:10E9100039607B68BB6101237B617B68002B6ED013
:10E92000BB691B6D002B0CD14FF0500372B683F303
:10E930001188BFF36F8FBFF34F8F62B6FB6000BFCC
:10E94000FEE7BB69DB6C3A689A4202D93B68FB611F
:10E9500002E0BB69DB6CFB61BB69DB6AFA699A4266
:10E960004DD0BB691B6D7A699A4248D1264B1B6812
:10E97000BA699A420CD14FF0500372B683F31188F2
:10E98000BFF36F8FBFF34F8F62B6BB6000BFFEE770
:10E99000BB69DB6A3B61BB69FA69DA62BB699B6987
:10E9A000002B04DBFB69C3F13802BB699A61BB69C8
:10E9B00059693A6913469B0013449B00134A134458
:10E9C00099421CD1BB6904331846FEF747F8BB696E
:10E9D000DA6A0F4B1B689A4203D9BB69DB6A0C4A9F
:10E9E0001360BB69DA6A13469B0013449B00074A15
:10E9F0001A44BB69043319461046FDF7D2FF00BF25
:10EA00002037BD4680BD00BFB41F0020B81F0020C6
:10EA10009024002080B400AF074B1B68002B04D06B
:10EA2000054B1B681A6D01321A65034B1B681846AB
:10EA3000BD465DF8047B7047B41F002080B584B0EC
:10EA400000AF78603960214B1B68FB60204B1B686E
:10EA500004331846FEF702F87B68B3F1FF3F0AD192
:10EA60003B68002B07D01A4B1B6804331946194822
:10EA7000FDF797FF26E0FA687B681344BB60144BF0
:10EA80001B68BA685A60BA68FB689A4209D2124B8E
:10EA90001A680F4B1B68043319461046FDF7A5FF93
:10EAA00010E00E4B1A680A4B1B68043319461046D7
:10EAB000FDF79BFF0A4B1B68BA689A4202D2084ACC
:10EAC000BB68136000BF1037BD4680BD8C2400209A
:10EAD000B41F00207424002044240020402400207F
:10EAE000A824002080B58AB004AF00237B6100F029
:10EAF00015FB1D4B1B68002B21D00023FB6000235E
:10EB0000BB603A1D07F1080107F10C031846FDF739
:10EB100001FF7968BB68FA680292019302230093AF
:10EB200000230A4611491248FEF77AFF0346114AAC
:10EB30001360104B1B68002B01D001237B617B69A4
:10EB4000002B0CD14FF0500372B683F31188BFF342
:10EB50006F8FBFF34F8F62B63B6100BFFEE77B69EB
:10EB600018461837BD4680BDE42400204CC3080871
:10EB7000B5EC0008E824002080B58AB000AFF8604A
:10EB8000B9607A603B6000237B62FB68002B0CD18C
:10EB90004FF0500372B683F31188BFF36F8FBFF34A
:10EBA0004F8F62B63B6200BFFEE71A4B1B68002B1B
:10EBB0002AD0BB683B617B687B61FB68BB61BB683B
:10EBC000052B18DCFFF7A8FD0346022B09D1114BDA
:10EBD000186807F1100100233A6BFEF775F97862A7
:10EBE00012E00C4B186807F1100100230022FEF719
:10EBF0006BF9786208E0074B186807F110010023F1
:10EC00003A68FEF767FA78627B6A18462837BD468D
:10EC100080BD00BFE424002080B588B002AF7860DA
:10EC20003960234B1B68DB68DB687B617B690433DD
:10EC30001846FDF713FF7B6993F8283003F00403AF
:10EC4000002B24D07B699A697B68D1187B683A686D
:10EC5000786900F0D3F80346002B21D000230093FD
:10EC600000237A6800217869FFF786FF38613B69E5
:10EC7000002B15D14FF0500372B683F31188BFF308
:10EC80006F8FBFF34F8F62B6FB6000BFFEE77B69FB
:10EC900093F8283023F00103DAB27B6983F8282047
:10ECA0007B691B6A7869984700BF1837BD4680BDED
:10ECB000DC24002080B584B000AF786007F1080341
:10ECC000184600F057F8F860BB681946F86800F07D
:10ECD00003F800F0D5F8F1E780B584B000AF7860B4
:10ECE0003960FFF70BF907F10803184600F066F8E2
:10ECF000F860BB68002B30D13B68002B0AD17A68E2
:10ED0000FB689A4206D8FFF707F9F9687868FFF7B9
:10ED100083FF24E03B68002B08D0134B1B681B6863
:10ED2000002B01D1012300E000233B600F4B18684A
:10ED30007A68FB68D31A3A681946FEF73DFEFFF77A
:10ED4000EBF80346002B0AD1094B4FF080521A60B2
:10ED5000BFF34F8FBFF36F8F01E0FFF7DDF800BF08
:10ED60001037BD4680BD00BFE0240020E424002011
:10ED700004ED00E080B485B000AF78600E4B1B68F6
:10ED80001B68002B01D1012200E000227B681A6081
:10ED90007B681B68002B05D1074B1B68DB681B6871
:10EDA000FB6001E00023FB60FB6818461437BD469A
:10EDB0005DF8047B704700BFDC24002080B584B080
:10EDC00000AF7860FFF748F9F8600B4B1B68FA68F2
:10EDD0009A4205D200F03CF97B6801221A6002E0F9
:10EDE0007B6800221A60044AFB681360FB681846BF
:10EDF0001037BD4680BD00BFEC24002080B586B032
:10EE000000AFF860B9607A603B6000237B61FB680B
:10EE1000BA685A60FB68FA681A61BA687B689A42F5
:10EE200012D87A683B68D21AFB689B699A4202D36F
:10EE300001237B611BE0104B1A68FB680433194601
:10EE40001046FDF7D2FD12E07A683B689A4206D27E
:10EE5000BA683B689A4202D301237B6107E0074B03
:10EE60001A68FB68043319461046FDF7BEFD7B693E
:10EE700018461837BD4680BDE0240020DC24002061
:10EE800080B58EB002AFD0E07B68002B1ADA3B1D54
:10EE90000433FB62FB6A002B0CD14FF0500372B6B7
:10EEA00083F31188BFF36F8FBFF34F8F62B6FB619F
:10EEB00000BFFEE7FB6A1B68FA6A5068FA6A92684C
:10EEC000114698477B68002BC0F2AE80FB68BB629E
:10EED000BB6A5B69002B04D0BB6A04331846FDF79C
:10EEE000BDFD3B461846FFF769FF78627B68092B3A
:10EEF00000F29B8001A252F823F000BF25EF00082A
:10EF000025EF000825EF00089DEF0008B1EF00088D
:10EF1000FFEF000825EF000825EF00089DEF00082F
:10EF2000B1EF0008BB6A93F8283043F00103DAB26E
:10EF3000BB6A83F82820BA68BB6A9B69D118BB6892
:10EF40007A6AB86AFFF75AFF0346002B6DD0BB6A96
:10EF50001B6AB86A9847BB6A93F8283003F0040329
:10EF6000002B62D0BA68BB6A9B691A4400230093E5
:10EF700000230021B86AFFF7FFFD38623B6A002BCF
:10EF800053D14FF0500372B683F31188BFF36F8FE4
:10EF9000BFF34F8F62B6BB6100BFFEE7BB6A93F859
:10EFA000283023F00103DAB2BB6A83F828203CE062
:10EFB000BB6A93F8283043F00103DAB2BB6A83F8E6
:10EFC0002820BA68BB6A9A61BB6A9B69002B0CD186
:10EFD0004FF0500372B683F31188BFF36F8FBFF306
:10EFE0004F8F62B67B6100BFFEE7BB6A9A697B6A9E
:10EFF000D1187B6A7A6AB86AFFF700FF15E0BB6A2E
:10F0000093F8283003F00203002B03D1B86A00F014
:10F01000CBFB0AE0BB6A93F8283023F00103DAB295
:10F02000BB6A83F8282000E000BF084B1B68391D2D
:10F0300000221846FEF7EEF80346002B7FF424AFBB
:10F0400000BF00BF3037BD4680BD00BFE4240020B4
:10F0500080B588B002AF4AE02E4B1B68DB681B68A6
:10F060003B612C4B1B68DB68DB68FB60FB6804338F
:10F070001846FDF7F3FCFB681B6AF8689847FB68C5
:10F0800093F8283003F00403002B30D0FB689B6911
:10F090003A691344BB60BA683B699A420ED9FB686F
:10F0A000BA685A60FB68FA681A611A4B1A68FB68FA
:10F0B000043319461046FDF798FC18E0002300932E
:10F0C00000233A690021F868FFF756FD78607B68F5
:10F0D000002B0CD14FF0500372B683F31188BFF3AD
:10F0E0006F8FBFF34F8F62B63B6000BFFEE7094BE7
:10F0F0001B681B68002BAFD1064B1B687B61064B5E
:10F100001B68044A1360044A7B69136000BF183708
:10F11000BD4680BDDC240020E024002080B582B004
:10F1200002AF00F04BF9154B1B68002B20D114489F
:10F13000FDF70AFC1348FDF707FC134B104A1A6051
:10F14000124B104A1A6000230093114B114A1021F0
:10F150000A20FDF717FD0346084A1360074B1B689A
:10F16000002B05D0054B1B680B491846FEF7FAFB30
:10F1700000F058F900BFBD4680BD00BFE424002068
:10F18000B4240020C8240020DC240020E024002037
:10F1900090250020F024002054C3080880B485B0D6
:10F1A00000AFF860B9607A60FB68043BFB60FB6805
:10F1B0004FF080721A60FB68043BFB60BB6823F071
:10F1C0000102FB681A60FB68043BFB600C4AFB68A9
:10F1D0001A60FB68143BFB607A68FB681A60FB6886
:10F1E000043BFB60FB686FF002021A60FB68203B87
:10F1F000FB60FB6818461437BD465DF8047B70471A
:10F2000005F2000880B485B000AF00237B60144B8A
:10F210001B68B3F1FF3F0CD04FF0500372B683F37D
:10F220001188BFF36F8FBFF34F8F62B6FB6000BFD3
:10F23000FEE74FF0500372B683F31188BFF36F8F70
:10F24000BFF34F8F62B6BB6000BF00BF7B68002B6F
:10F25000FCD000BF00BF1437BD465DF8047B70478B
:10F26000600100200000000000000000000000001D
:10F27000074B19680868B0E8F04F80F30988BFF3BE
:10F280006F8F4FF0000080F311887047AFF300805C
:10F29000B41F002000BF00BF08480068006880F36A
:10F2A00008884FF0000080F3148862B661B6BFF39F
:10F2B0004F8FBFF36F8F00DF00BF00BF08ED00E08E
:10F2C00080B584B000AF374BFB60FB681B78DBB2C6
:10F2D0007B60FB68FF221A70FB681B78DBB2FB7057
:10F2E000FB78DBB203F05003DAB22F4B1A702F4BCE
:10F2F00007221A6009E02D4B1B68013B2B4A136063
:10F30000FB78DBB25B00DBB2FB70FB78DBB203F0B7
:10F310008003802BEFD0254B1B68C3F10703042B20
:10F320000CD04FF0500372B683F31188BFF36F8F88
:10F33000BFF34F8F62B6BB6000BFFEE71B4B1B687D
:10F340001B021A4A1360194B1B6803F4E063174A47
:10F3500013607B68DAB2FB681A70154B1B68144A9D
:10F3600043F470031360124B1B68114A43F070435F
:10F37000136000F0DDF80F4B00221A6000F0FCF87B
:10F380000D4B1B680C4A43F040431360FFF784FFAA
:10F39000FEF72EFFFFF736FF002318461037BD4655
:10F3A00080BD00BF00E400E0E0250020E42500204F
:10F3B00020ED00E06001002034EF00E080B483B075
:10F3C00000AF4FF0500372B683F31188BFF36F8F15
:10F3D000BFF34F8F62B67B6000BF104B1B680133D9
:10F3E0000E4A13600D4B1B68012B11D10C4B1B688F
:10F3F000DBB2002B0CD04FF0500372B683F31188B0
:10F40000BFF36F8FBFF34F8F62B63B6000BFFEE765
:10F4100000BF0C37BD465DF8047B704760010020DB
:10F4200004ED00E080B483B000AF134B1B68002BE9
:10F430000CD14FF0500372B683F31188BFF36F8F76
:10F44000BFF34F8F62B67B6000BFFEE70A4B1B68BD
:10F45000013B094A1360084B1B68002B05D10023B0
:10F460003B603B6883F3118800BF00BF0C37BD468B
:10F470005DF8047B704700BF6001002000000000C1
:10F48000EFF30980BFF36F8F154B1A681EF0100F52
:10F4900008BF20ED108A20E9F04F10602DE9090027
:10F4A0004FF0500072B680F31188BFF34F8FBFF357
:10F4B0006F8F62B6FEF79CFE4FF0000080F311885C
:10F4C00009BC19680868B0E8F04F1EF0100F08BFBB
:10F4D000B0EC108A80F30988BFF36F8F704700BFCC
:10F4E000B41F002000BF00BF80B582B000AF4FF056
:10F4F000500372B683F31188BFF36F8FBFF34F8F42
:10F5000062B67B6000BFFEF7B7FD0346002B03D059
:10F51000064B4FF080521A6000233B603B6883F338
:10F52000118800BF00BF0837BD4680BD04ED00E074
:10F5300080B400AF0B4B00221A600B4B00221A6004
:10F540000A4B1B680A4AA2FB03239B09094A013B99
:10F550001360044B07221A6000BFBD465DF8047BB0
:10F56000704700BF10E000E018E000E00800002055
:10F57000D34D621014E000E0DFF80C00016841F4A4
:10F5800070010160704700BF88ED00E080B485B075
:10F5900000AFEFF30583FB60FB680F2B16D9194A08
:10F5A000FB6813441B78FB72174B1B78FA7A9A425C
:10F5B0000CD24FF0500372B683F31188BFF36F8FF4
:10F5C000BFF34F8F62B67B6000BFFEE70F4B1B6837
:10F5D00003F4E0620E4B1B689A420CD94FF05003C3
:10F5E00072B683F31188BFF36F8FBFF34F8F62B68C
:10F5F0003B6000BFFEE700BF1437BD465DF8047BEB
:10F60000704700BFF0E300E0E02500200CED00E0D3
:10F61000E425002080B58AB000AF78600023FB614C
:10F62000FEF76CFC5B4B1B68002B01D100F01AF954
:10F63000594B1A687B681340002B40F092807B681E
:10F64000002B1FD008227B6813447B607B6803F08B
:10F650000703002B16D07B6823F0070308337B6079
:10F660007B6803F00703002B0CD04FF0500372B6F9
:10F6700083F31188BFF36F8FBFF34F8F62B67B6147
:10F6800000BFFEE77B68002B6BD0444B1B687A6899
:10F690009A4266D8424B3B62414B1B687B6204E056
:10F6A0007B6A3B627B6A1B687B627B6A5B687A6809
:10F6B0009A4203D97B6A1B68002BF1D1354B1B683A
:10F6C0007A6A9A424DD03B6A1B6808221344FB6158
:10F6D0007B6A1A683B6A1A607B6A5A687B68D21A2E
:10F6E00008235B009A4221D97A6A7B681344BB6184
:10F6F000BB6903F00703002B0CD04FF0500372B628
:10F7000083F31188BFF36F8FBFF34F8F62B63B61F6
:10F7100000BFFEE77B6A5A687B68D21ABB695A60F1
:10F720007B6A7A685A60B86900F0FEF81B4B1A6869
:10F730007B6A5B68D31A194A1360184B1A68194B15
:10F740001B689A4203D2154B1B68164A13607B6AEA
:10F750005A68114B1B681A437B6A5A607B6A002205
:10F760001A60FEF7D9FBFB6903F00703002B0CD0EE
:10F770004FF0500372B683F31188BFF36F8FBFF35E
:10F780004F8F62B6FB6000BFFEE7FB691846283763
:10F79000BD4680BDF0250220FC250220F425022074
:10F7A000E8250220F825022080B586B000AF7860F9
:10F7B0007B687B617B68002B4CD008235B427A69B5
:10F7C00013447B617B693B613B695A68234B1B682F
:10F7D0001340002B0CD14FF0500372B683F3118805
:10F7E000BFF36F8FBFF34F8F62B6FB6000BFFEE7C2
:10F7F0003B691B68002B0CD04FF0500372B683F3AB
:10F800001188BFF36F8FBFF34F8F62B6BB6000BF2D
:10F81000FEE73B695A68114B1B681340002B19D057
:10F820003B691B68002B15D13B695A680B4B1B6861
:10F83000DB431A403B695A60FEF760FB3B695A683C
:10F84000074B1B681344064A1360386900F06CF8D4
:10F85000FEF762FB00BF1837BD4680BDFC250220C5
:10F86000F425022080B485B000AF4FF40033BB60B4
:10F87000274BFB60FB6803F00703002B0CD0FB68F1
:10F880000733FB60FB6823F00703FB60BA68FB6883
:10F89000D31A1F4A1344BB60FB687B601D4A7B6818
:10F8A00013601C4B00225A607B68BA681344FB60EB
:10F8B0000822FB689B1AFB60FB6823F00703FB60D0
:10F8C000FB68154A1360144B1B6800225A60124BE8
:10F8D0001B6800221A607B683B603B68FA68D21A9A
:10F8E0003B685A600C4B1A683B681A603B685B685F
:10F8F0000A4A13603B685B68094A1360094B4FF082
:10F9000000421A6000BF1437BD465DF8047B7047A3
:10F91000E8250020E8250220F0250220F825022015
:10F92000F4250220FC25022080B485B000AF786069
:10F93000284BFB6002E0FB681B68FB60FB681B68F0
:10F940007A689A42F7D8FB68BB60FB685B68BA6864
:10F9500013447A689A4208D1FB685A687B685B68EE
:10F960001A44FB685A60FB687B607B68BB607B68FD
:10F970005B68BA681A44FB681B689A4218D1FB6836
:10F980001A68154B1B689A420DD07B685A68FB6851
:10F990001B685B681A447B685A60FB681B681A68BE
:10F9A0007B681A6008E00C4B1A687B681A6003E0F9
:10F9B000FB681A687B681A60FA687B689A4202D012
:10F9C000FB687A681A6000BF1437BD465DF8047B97
:10F9D000704700BFE8250220F025022080B584B0E2
:10F9E00000AF786039600D4A7B6813600B4B1B6871
:10F9F000FB60FB6800221A60FB6801225A603B68CA
:10FA0000A3F11002FB689A600548FCF7B5FC0346B9
:10FA1000044A136000BF1037BD4680BD0026022097
:10FA200074FE08080426022080B586B000AF786016
:10FA300039607B68002B01D100235FE0314B1B68EC
:10FA400000211846FCF732FD0346002B0CBF0123B2
:10FA50000023DBB2002B50D02B4B1B683B613B6972
:10FA60007B617B68073323F007037B607B69002B96
:10FA70000DD07B695B68002B04D07B699B687A683A
:10FA80009A4203D97B691B687B61EFE700BF7B6902
:10FA9000002B06D11B4B1B681846FCF765FD0023A5
:10FAA0002CE07B699A687B68D31A103BFB60FB688B
:10FAB000072B14DD7B6810337A691344BB607B69C4
:10FAC0001A68BB681A60BB6801225A60FA68BB6892
:10FAD0009A607B69BA681A607B697A689A607B6908
:10FAE00000225A607B693A68DA60064B1B68184648
:10FAF000FCF73AFD7B69103300E000231846183705
:10FB0000BD4680BD042602200026022080B586B0B6
:10FB100000AF78607B68002B00F08C80474B1B683F
:10FB200000211846FCF7C2FC0346002B0CBF012342
:10FB30000023DBB2002B7ED0414B1B68FB6000230F
:10FB40007B61FB683B613B69002B0AD03B6910334A
:10FB50007A689A4205D93B697B613B691B683B61C6
:10FB6000F1E73B69002B08D03B6910337A689A4271
:10FB700003D13B695B68002B05D0324B324A8121AF
:10FB8000324873F055FC3B699B681A46CC21786873
:10FB900074F020FB3B691B68BB60BB68002B2CD05A
:10FBA000BB685B68002B28D07B69002B14D07B6975
:10FBB0005B68002B10D0BB681A687B691A607B6990
:10FBC0009A683B699968BB689B680B44134403F1CE
:10FBD00020027B699A6027E0BB681A683B691A605B
:10FBE0003B699A68BB689B68134403F110023B6948
:10FBF0009A603B6901225A6016E07B69002B10D0A5
:10FC00007B695B68002B0CD07B69BA681A607B69E2
:10FC10009A683B699B68134403F110027B699A6000
:10FC200002E03B6901225A60044B1B681846FCF74E
:10FC30009BFC00E000BF1837BD4680BD04260220B3
:10FC40000026022064C308086CC3080884C308089F
:10FC500080B584B000AF786039607B6800221A609C
:10FC60003B6800221A601B4B1B6800211846FCF7FA
:10FC70001DFC0346002B0CBF01230023DBB2002B2D
:10FC800023D0154B1B68BB60BB68FB60FB68002B77
:10FC900016D0FB685B68002B07D07B681A68FB688E
:10FCA0009B681A447B681A6006E03B681A68FB6828
:10FCB0009B681A443B681A60FB681B68FB60E5E7B9
:10FCC000044B1B681846FCF74FFC00BF1037BD46BD
:10FCD00080BD00BF04260220002602200EB480B59D
:10FCE000C5B000AF024607F58873A3F209131A7076
:10FCF00007F59073C7F80C3107F10800D7F80C31FD
:10FD0000D7F81C214FF4807177F054FE07F5887303
:10FD1000A3F58473002283F8002107F58873A3F20A
:10FD200009131B78002B0CD107F108031846F0F7D4
:10FD3000C9FA024607F108031146184652F0E6FFD9
:10FD40001FE007F58873A3F209131B78012B0CD170
:10FD500007F108031846F0F7B5FA024607F1080361
:10FD60001146184652F0EAFF0BE007F10803184667
:10FD7000F0F7A8FA024607F108031146184652F0B8
:10FD8000F5FF00BF07F58A77BD46BDE8804003B0A8
:10FD90007047000080B582B000AF0B4B1B7883F03A
:10FDA0000103DBB2002B0AD000F020F878607B68FA
:10FDB0004EF65F22934202D9034B01221A7000BF14
:10FDC0000837BD4680BD00BF6401002080B500AF8C
:10FDD00000F0E4F80346034A1360034B00221A7054
:10FDE00000BF80BD082602206401002080B500AF5E
:10FDF000074B1B78002B02D04EF6602305E000F085
:10FE0000CDF80246034B1B68D31A184680BD00BFCD
:10FE1000640100200826022080B500AF084B4FF097
:10FE200040421A60074B4FF400021A604FF4001072
:10FE300000F07EF80346044A136000BF80BD00BF97
:10FE400044260220482602200C26022080B582B0DB
:10FE500000AF4FF4004000F06BF80346274A1360F0
:10FE60004FF47F337B60786800F062F80346244AE1
:10FE70001360786800F05CF80346224A13607868E3
:10FE800000F056F80346204A1360786800F050F8F6
:10FE900003461E4A1360786800F04AF803461C4A7D
:10FEA0001360786800F044F803461A4A13607868D3
:10FEB00000F03EF80346184A1360786800F038F8FE
:10FEC0000346164A1360786800F032F80346144A75
:10FED0001360786800F02CF80346124A13604FF460
:10FEE000803000F025F803460F4A1360064B1B686C
:10FEF0000E4A136000BF0837BD4680BD10260220A1
:10FF000014260220182602201C2602202026022069
:10FF100024260220282602202C2602203026022019
:10FF20003426022038260220402602203C260220C9
:10FF300080B584B000AF78607B6803F2FF32114B6C
:10FF400013407B60104B1B68FB60104B1B687A688A
:10FF50009A4205D30E4B0F4A5C210F4873F068FAA2
:10FF6000094B1A687B681344074A1360074B1A68E9
:10FF70007B68D31A054A1360FB6818461037BD46E4
:10FF800080BD00BF00FCFFFF44260220482602205F
:10FF9000A8C30808C4C30808E8C3080880B500AFB0
:10FFA000F4F704F80346184680BD000080B584B01D
:10FFB00000AF78607B68002B16D00023FB60FB68E5
:10FFC000222B11D80B4AFB6852F823307968184667
:10FFD000F0F76EF90346002B02D1FB68DBB204E0B8
:10FFE000FB680133FB60EAE7002318461037BD4683
:10FFF00080BD00BF6801002080B483B000AF03461D
:020000040801F1
:10000000FB71FB79FF2B01D1FF2302E0FB79044A4E
:10001000D35C18460C37BD465DF8047B704700BFC3
:1000200084FE080880B483B000AF0346FB71FB79FF
:10003000FF2B02D14FF07E5304E0FB79064A9B0070
:1000400013441B6807EE903AB0EE670A0C37BD46C2
:100050005DF8047B704700BFA8FE080880B485B037
:1000600000AF034687ED000AFB71FB79FF2B01D13E
:10007000FF2322E00023FB60FB68222B1CD8124ADE
:10008000FB6813441A78FB790F49CB5C9A420FD175
:100090000E4AFB689B001344D3ED007A97ED007A7B
:1000A000B4EE677AF1EE10FA02D1FB68DBB204E03D
:1000B000FB680133FB60DFE7FF2318461437BD46BA
:1000C0005DF8047B704700BF84FE0808A8FE08089E
:1000D00080B588B000AF87ED010A0346FB700123AD
:1000E000FB61324AFB699B0013441B687B61D7EDBF
:1000F000057AB7EE007AF4EEC77AF1EE10FA20DC5A
:1001000097ED017AD7ED057AB4EEE77AF1EE10FAC1
:1001100013D5FB69013B254A9B001344D3ED007ABC
:10012000FB78B0EE670A1846FFF798FF0346FB74AA
:10013000FB7CFF2B01D0FB7C34E0FB690133FB61CE
:10014000CFE700BF0823BB61BB69002B29DB174A3F
:10015000BB699B0013441B68FB60D7ED037AB7EEC5
:10016000007AF4EE477AF1EE10FA19D097ED017AA1
:10017000D7ED037AB4EEE77AF1EE10FA0CDBFB78F8
:1001800097ED030A1846FFF769FF0346FB74FB7CF3
:10019000FF2B01D0FB7C05E0BB69013BBB61D3E7D2
:1001A00000BFFB7818462037BD4680BD34FF0808E5
:1001B00080B485B000AF87ED010A0823FB60FB68BF
:1001C000002B14DD0F4AFB689B0013441B68BB60C7
:1001D00097ED027AD7ED017AB4EEE77AF1EE10FAF4
:1001E00001D5BB6804E0FB68013BFB60E7E7064B19
:1001F00007EE903AB0EE670A1437BD465DF8047B0F
:10020000704700BF34FF0808CCBC8C2B80B586B08B
:1002100000AF034687ED020AC7ED010AFB73FB7BC3
:100220001846FFF7FFFE87ED050A97ED017AD7ED37
:10023000057AB4EEE77AF1EE10FA08D997ED027A72
:10024000D7ED057AB4EEE77AF1EE10FA0DD897ED16
:10025000050AFFF7ADFFF0EE407AFB7BB0EE670AD0
:100260001846FFF7FBFE034600E0FF231846183749
:10027000BD4680BD80B586B000AF034687ED000A5D
:10028000FB7108237B617B69002B1FDB124A7B69B2
:100290009B0013441B683B6197ED007AD7ED047A0D
:1002A000B4EEE77AF1EE10FA0CDBFB7997ED040A75
:1002B0001846FFF7D3FE0346FB73FB7BFF2B01D0F1
:1002C000FB7B04E07B69013B7B61DCE7FF23184695
:1002D0001837BD4680BD00BF34FF080880B588B020
:1002E00000AF034687ED020AC7ED010AFB73002346
:1002F000FB61FB69082B28DC164AFB699B00134451
:100300001B68BB6197ED017AD7ED067AB4EEE77A08
:10031000F1EE10FA08D997ED027AD7ED067AB4EE2D
:10032000E77AF1EE10FA0CD8FB7B97ED060A184637
:10033000FFF794FE0346FB75FB7DFF2B01D0FB7D91
:1003400004E0FB690133FB61D3E7FF231846203744
:10035000BD4680BD34FF080880B487B000AF87ED8C
:10036000050AC7ED040A87ED031AC7ED021A87EDE7
:10037000012A97ED057AD7ED047A37EE677AD7ED43
:10038000016AD7ED037A76EEE77A67EE276A97ED92
:10039000027AD7ED047A77EE677A86EEA77AD7ED00
:1003A000037A77EE277AB0EE670A1C37BD465DF810
:1003B000047B704780B485B000AF87ED030AC7EDBA
:1003C000020A87ED011A97ED037AD7ED027AB4EEAF
:1003D000E77AF1EE10FA01D5BB680BE097ED037AEE
:1003E000D7ED017AB4EEE77AF1EE10FA01DD7B6821
:1003F00000E0FB6807EE903AB0EE670A1437BD469E
:100400005DF8047B704780B584B000AFF860B960D8
:100410007A60BA687968F86875F07BFFBB68013B61
:10042000FA68134400221A7000BF1037BD4680BD21
:1004300080B586B000AFF860B9607A603B603A681A
:10044000BB689A4201D23B6800E0BB687B617A6975
:100450007968F86875F05DFFFA687B6913440022DB
:100460001A7000BF1837BD4680BD80B586B000AF9A
:10047000F860B9607A60F868EFF724FF0246BB685D
:100480009B1A013B7B617B69002B05DB7B691A466C
:100490007968F86875F016FF00BF1837BD4680BD53
:1004A00080B586B000AFF860B9607A60F868EFF7A1
:1004B00009FF7861FA687B69D018BA687B69D11A3C
:1004C0007B68034A74F018FF00BF1837BD4680BD33
:1004D000D0C4080880B586B000AFF860B9607A6013
:1004E000F868EFF7EFFE7861FA687B69D018BA68B0
:1004F0007B69D11A7B68034A74F0FEFE00BF18378F
:10050000BD4680BDD4C4080880B588B002AFF8608D
:10051000B960C7E90023F868EFF7D4FE7861FA689C
:100520007B69D018BA687B69D11AD7E90023CDE975
:100530000023034A74F0E0FE00BF1837BD4680BDBB
:10054000D8C4080880B588B002AFF860B960C7E9C0
:100550000023F868EFF7B6FE7861FA687B69D01877
:10056000BA687B69D11AD7E90023CDE90023034A91
:1005700074F0C2FE00BF1837BD4680BDDCC4080859
:10058000B0B588B002AFF860B96087ED010AF868CD
:10059000EFF798FE7861FA687B69D418BA687B69CE
:1005A000D51A7868EFF7FAFF02460B46CDE900232B
:1005B000044A2946204674F09FFE00BF1837BD4606
:1005C000B0BD00BFE0C40808B0B588B002AFF860A5
:1005D000B96087ED010A3A60F868EFF773FE786159
:1005E000FA687B69D418BA687B69D51A7868EFF71E
:1005F000D5FF02460B46CDE900233B68044A294655
:10060000204674F079FE00BF1837BD46B0BD00BF6C
:10061000E4C4080880B588B002AFF860B96087ED1F
:10062000000BF868EFF74EFE7861FA687B69D01826
:10063000BA687B69D11AD7E90023CDE90023034AC0
:1006400074F05AFE00BF1837BD4680BDE0C40808EC
:1006500080B58AB002AF7861396187ED020B7A60AC
:100660007869EFF72FFEF8617A69FB69D0183A696B
:10067000FB69D11AD7E90223CDE900237B68034A3D
:1006800074F03AFE00BF2037BD4680BDE4C40808C0
:1006900080B584B000AF87ED010AC7ED000AF7EE20
:1006A000006A97ED007AC6EE877AC7ED037A97ED78
:1006B000017AD7ED037A67EE277AB0EE670A6EF01B
:1006C00043FFB0EE407AD7ED037AC7EE276AF0EE2B
:1006D000667AB0EE670A1037BD4680BD80B483B03D
:1006E00000AF87ED010A97ED017AD7ED017AB4EEFC
:1006F000677AF1EE10FA14BF01230023DBB218462B
:100700000C37BD465DF8047B704790B583B000AFF1
:1007100087ED000B01231C46D7E90023D7E9000130
:10072000F0F7FCF90346002B01D000231C46E3B28E
:1007300018460C37BD4690BD80B483B000AF034669
:10074000FB71FB792F2B04D9FB79392B01D80123BD
:1007500000E0002318460C37BD465DF8047B704767
:1007600080B483B000AF78607B68002B07DB7B68C8
:10077000092B04DC7B68DBB23033DBB203E07B683F
:10078000DBB23733DBB218460C37BD465DF8047B6D
:10079000704780B485B000AFF860B9607A603B60A4
:1007A000FA687B689A4211DB7A68BB691344FA687D
:1007B0009A420BDABA683B689A4207DB3A68FB69EF
:1007C0001344BA689A4201DA012300E00023184674
:1007D0001437BD465DF8047B704780B58AB000AF22
:1007E000F860B9607A60FB687B62FA68BB681344A2
:1007F0007B6100233B623B6A032B63DC7A6A7B6983
:100800009A4201D1002366E00023FB610023BB6113
:10081000BB69022B2EDC7A6A7B699A4207D1BB69DD
:10082000002B02DD3B6A032B24D0002353E07B6ABC
:100830001B781846FFF780FF0346002B0DD0FA699E
:1008400013469B0013445B0019467B6A5A1C7A626C
:100850001B780B44303BFB6108E0BB69002B03DDD8
:100860007B6A1B782E2B05D0002334E0BB69013353
:10087000BB61CDE7FB69FF2B01D900232BE03B6A6D
:10088000022B05DC7B6A5A1C7A621B782E2B06D160
:100890003B6A032B05D17A6A7B699A4201D0012316
:1008A00000E00023002B01D0002314E0FB69D9B243
:1008B00007F110023B6A13440A461A703B6A01337F
:1008C0003B6298E707F11003184600F07AF80246F9
:1008D0007B681A60012318462837BD4680BD80B466
:1008E00083B000AF78603B1D1B7818460C37BD46BF
:1008F0005DF8047B704780B483B000AF78600B462E
:10090000FB707B68FA781A7000BF0C37BD465DF843
:10091000047B704780B483B000AF78603B1D013327
:100920001B7818460C37BD465DF8047B704780B4D1
:1009300083B000AF78600B46FB707B680133FA78B8
:100940001A7000BF0C37BD465DF8047B704780B459
:1009500083B000AF78603B1D02331B7818460C371C
:10096000BD465DF8047B704780B483B000AF78600B
:100970000B46FB707B680233FA781A7000BF0C37A5
:10098000BD465DF8047B704780B483B000AF7860EB
:100990003B1D03331B7818460C37BD465DF8047BBE
:1009A000704780B483B000AF78600B46FB707B6803
:1009B0000333FA781A7000BF0C37BD465DF8047B2C
:1009C000704780B582B000AF78607B6818787B682C
:1009D000013319787B6802331A787B6803331B78FC
:1009E00000F005F8034618460837BD4680BD90B5AF
:1009F00085B000AF0446084611461A462346FB71EF
:100A00000346BB710B467B7113463B71FA7907F1C4
:100A10000C0311461846FFF76EFFBA7907F10C0375
:100A200011461846FFF783FF7A7907F10C03114648
:100A30001846FFF799FF3A7907F10C03114618465B
:100A4000FFF7AFFFFB6818461437BD4690BD0000A6
:100A5000F0B589B004AFF860B9607A60F868FFF764
:100A60003EFF0646F868FFF755FF0446F868FFF7B3
:100A70006EFF0546F868FFF787FF0346029301956E
:100A800000943346044A7968B86874F035FC00BFB6
:100A90001437BD46F0BD00BF2CC50808B0B588B0FE
:100AA00002AF0346B9607A60FB81B7F90E30002BC4
:100AB00006D17B681C4A1946B868FFF7A4FC2FE0F2
:100AC000B7F90E30002B04DD2B23FB75FB89BB82AD
:100AD00005E02D23FB75FB895B429BB2BB827868E6
:100AE000FC7DB7F91430114A82FB03125211DB1757
:100AF000D31A1BB21D46B7F914300C4A82FB0312FD
:100B00005111DA178A1A642101FB02F29B1A1BB2F7
:100B1000019300952346064A0146B86874F0ECFB41
:100B200000BF1837BD46B0BD38C508081F85EB515A
:100B30003CC5080880B483B000AF87ED010A7B682C
:100B400007EE903AB0EE670A0C37BD465DF8047BBD
:100B5000704780B483B000AF87ED010AD7ED017A0A
:100B600067EEA77AB0EE670A0C37BD465DF8047BE6
:100B7000704780B483B000AF87ED010AB7EE007A0A
:100B8000D7ED017A37EE677AF7EE006AD7ED017A92
:100B900076EEE77A67EE277AB7EE007A77EE677A35
:100BA000B0EE670A0C37BD465DF8047B704780B530
:100BB00082B000AF87ED010AD7ED017AB6EE007A78
:100BC000F4EEC77AF1EE10FA08D5D7ED017A37EED8
:100BD000A77AD7ED017A67EE277A19E0D7ED017A87
:100BE000B8EE007A67EE877AB0EE007A77EE877A11
:100BF000F0EE000AB0EE670A6EF0ECFEB0EE407A5E
:100C0000F0EE006AC7EE267AB7EE007A77EE677AE2
:100C1000B0EE670A0837BD4680BD80B483B000AF30
:100C200087ED010AD7ED017A27EEA77AD7ED017A91
:100C300067EE277AB0EE670A0C37BD465DF8047B95
:100C40007047B0B582B000AF87ED010A38607868B0
:100C5000EFF7A4FC04460D463868EFF78DFC02461A
:100C60000B4643EC112B45EC104B6EF0BBFDB0EE88
:100C7000407AF0EE607AB0EE470AF0EE670A083785
:100C8000BD46B0BD80B582B000AF87ED010AB7EEBA
:100C9000007AD7ED017A77EE677A0320B0EE670A23
:100CA000FFF7CFFF53EC102B4FF000000849EFF790
:100CB00015FB02460B4610461946EFF7BFFF0346E9
:100CC00007EE903AB0EE670A0837BD4680BD00BF18
:100CD0000000F03F80B582B000AF87ED010AD7ED8C
:100CE000017AB6EE007AF4EEC77AF1EE10FA0ED57C
:100CF000D7ED017AB1EE007A27EE877AD7ED017A47
:100D000027EE277AD7ED017A67EE277A19E0D7ED3B
:100D1000017AB8EE007A67EE877AB0EE007A77EE65
:100D2000877AF0EE080AB0EE670A6EF053FEB0EE76
:100D3000407AF0EE006AC7EE267AB7EE007A77EED8
:100D4000677AB0EE670A0837BD4680BD80B483B0CD
:100D500000AF87ED010AD7ED017A27EEA77AD7ED2C
:100D6000017A27EE277AD7ED017A67EE277AB0EE7F
:100D7000670A0C37BD465DF8047B704780B582B0CA
:100D800000AF87ED010AB7EE007AD7ED017A77EE72
:100D9000677AF1EE000AB0EE670A6EF01BFEF0EE25
:100DA000407AB7EE007A77EE677AB0EE670A0837D6
:100DB000BD4680BD80B582B000AF87ED010AD7ED9A
:100DC000017AB6EE007AF4EEC77AF1EE10FA12D597
:100DD000D7ED017AB2EE007A27EE877AD7ED017A65
:100DE00027EE277AD7ED017A27EE277AD7ED017A19
:100DF00067EE277A19E0D7ED017AB8EE007A67EE50
:100E0000877AB0EE007A77EE877AF1EE000AB0EEDC
:100E1000670A6EF0DFFDB0EE407AF0EE006AC7EED2
:100E2000267AB7EE007A77EE677AB0EE670A08376F
:100E3000BD4680BD80B483B000AF87ED010AD7ED19
:100E4000017A27EEA77AD7ED017A27EE277AD7ED38
:100E5000017A27EE277AD7ED017A67EE277AB0EE8E
:100E6000670A0C37BD465DF8047B704780B582B0D9
:100E700000AF87ED010AB7EE007AD7ED017A77EE81
:100E8000677AF1EE040AB0EE670A6EF0A3FDF0EEA9
:100E9000407AB7EE007A77EE677AB0EE670A0837E5
:100EA000BD4680BD80B582B000AF87ED010AD7EDA9
:100EB000017AB6EE007AF4EEC77AF1EE10FA16D5A2
:100EC000D7ED017AB3EE007A27EE877AD7ED017A73
:100ED00027EE277AD7ED017A27EE277AD7ED017A28
:100EE00027EE277AD7ED017A67EE277A19E0D7ED5A
:100EF000017AB8EE007A67EE877AB0EE007A77EE84
:100F0000877AF1EE040AB0EE670A6EF063FDB0EE88
:100F1000407AF0EE006AC7EE267AB7EE007A77EEF6
:100F2000677AB0EE670A0837BD4680BD80B582B0EB
:100F300000AF87ED010AD7ED017A9FED0B7A67EEDE
:100F4000877AF0EE006A87EEA67AB0EE470A6EF076
:100F500075FAF0EE407AB7EE007A77EE677AB0EE87
:100F6000670A0837BD4680BDDB0F494080B582B0B7
:100F700000AF87ED010AD7ED017A9FED097A67EEA0
:100F8000877AF0EE006A87EEA67AB0EE470A6EF036
:100F9000FFFAF0EE407AB0EE670A0837BD4680BD32
:100FA000DB0F494080B582B000AF87ED010AD7ED75
:100FB000017A9FED0D7A67EE877AB0EE670A6EF0E0
:100FC0003DFAF0EE407AB7EE007A77EEC77AF1EEAE
:100FD000677AB0EE007AC7EE876AF0EE667AB0EE16
:100FE000670A0837BD4680BDDB0F494080B582B037
:100FF00000AF87ED010AD7ED017AF5EE407AF1EE08
:1010000010FA12D0D7ED017AB2EE047A67EE877A41
:10101000B2EE047A77EEC77AF0EE670AB0EE000A15
:101020006EF0D8FCF0EE407A01E0DFED037AB0EE2E
:10103000670A0837BD4680BD0000000080B582B059
:1010400000AF87ED010AD7ED017AB7EE007AF4EE32
:10105000477AF1EE10FA12D0D7ED017ABAEE047A9F
:1010600067EE877AF0EE670AB0EE000A6EF0B2FC27
:10107000F0EE407AB7EE007A77EE677A01E0F7EEAD
:10108000007AB0EE670A0837BD4680BD80B582B0F1
:1010900000AF87ED010AD7ED017AF5EE407AF1EE67
:1010A00010FA46D0D7ED017AB7EE007AF4EE477A1F
:1010B000F1EE10FA3AD0D7ED017AB6EE007AF4EEFE
:1010C000C77AF1EE10FA16D5D7ED017AB3EE047AAD
:1010D00067EE877AB2EE047A77EEC77AF0EE670AA7
:1010E000B0EE000A6EF076FCB0EE407AF0EE006AE8
:1010F000C7EE267A1FE0D7ED017ABBEE047A67EEE1
:10110000877AB2EE047A77EE877AF0EE670AB0EE6D
:10111000000A6EF05FFCF0EE407AB0EE007A37EE37
:10112000677AF0EE006AC7EE267A04E0F7EE007AFE
:1011300001E0DFED037AB0EE670A0837BD4680BDF7
:101140000000000080B582B000AF87ED010AF0EE2C
:10115000000A97ED010A6EF03DFCF0EE407AB7EE22
:10116000007A77EE677AB0EE670A6EF08BFCF0EEED
:10117000407AB7EE007A77EE677AB0EE670A083702
:10118000BD4680BD80B582B000AF87ED010AD7EDC6
:10119000017AB7EE007A77EEC77AF0EE000AB0EE89
:1011A000670A6EF017FCF0EE407AB7EE007A77EE41
:1011B000677AB0EE670A6EF065FCF0EE407AB0EE4A
:1011C000670A0837BD4680BD80B582B000AF87EDA5
:1011D000010AD7ED017AB6EE007AF4EEC77AF1EEA5
:1011E00010FA25D5D7ED017A77EEA77A0220B0EE76
:1011F000670AFFF726FD53EC102B4FF00000214942
:10120000EFF76CF802460B4610461946EFF716FD4D
:10121000034600EE103A6EF035FCF0EE407AB7EE81
:10122000007A37EE677AF0EE006AC7EE267A23E09E
:10123000D7ED017AB8EE007A67EE877AB0EE007AE1
:1012400077EE877AF0EE000AB0EE670A6EF0C2FB26
:10125000F0EE407AB7EE007A77EE677AB0EE670A82
:101260006EF010FCF0EE407AB7EE007A37EE877A37
:10127000F0EE006AC7EE267AB0EE670A0837BD4680
:1012800080BD00BF0000F03F80B483B000AF87EDA9
:10129000010AD7ED017A9FED0F7A27EE877AD7ED15
:1012A000017A27EE277AD7ED017A27EE277AD7ED54
:1012B000017ADFED096A67EEA66AD7ED017A66EE7C
:1012C000A77A77EE677AB0EE670A0C37BD465DF80D
:1012D000047B7047B0E62C4060CDD93F80B52DED42
:1012E000028B82B000AF87ED010AD7ED017AB7EE2D
:1012F000007A77EEC77AF0EE080AB0EE670A6EF071
:1013000069FBF0EE407A9FED117A67EE877AB7EECF
:10131000007A37EE878AD7ED017AB7EE007A77EE5A
:10132000C77AF0EE000AB0EE670A6EF053FBF0EEFB
:10133000407A9FED077A67EE877A78EE277AB0EEEB
:10134000670A0837BD46BDEC028B80BDB0E62C4075
:1013500060CDD93F80B582B000AF87ED010AD7EDEF
:10136000017AB6EE007AF4EEC77AF1EE10FA1CD5E7
:10137000D7ED017A77EEA77AF0EE000AB0EE670AB1
:101380006EF028FBB0EE407AD7ED017ADFED1E6AF1
:1013900067EEA67ADFED1D6A77EEE67A27EE277A0A
:1013A000F0EE006AC7EE267A29E0D7ED017A77EEF3
:1013B000A77AB0EE007A77EEC77AF0EE000AB0EEC8
:1013C000670A6EF007FBB0EE407AD7ED017A77EE50
:1013D000A77AF0EE006A77EEE67ADFED0D6A67EE47
:1013E000A67ADFED0A6A77EEA67A67EE277AB0EE84
:1013F000007A37EE877AF0EE006AC7EE267AB0EE12
:10140000670A0837BD4680BDFF12E640FF1226403E
:10141000FF12664080B52DED028B82B000AF87EDE4
:10142000010AD7ED017AF5EE407AF1EE10FA36D0E6
:10143000D7ED017AB7EE007AF4EE477AF1EE10FAC2
:101440002AD0D7ED017AB2EE047A67EE877AB2EE4F
:10145000047A77EEC77AF0EE670AB0EE000A6EF013
:10146000B9FAF0EE407AB1EE678AD7ED017AB2EEC2
:10147000047A67EE877A9FED0E7A77EEC77A9FED52
:101480000D7A67EE877AB0EE670A6EF081F8F0EEBB
:10149000407A68EE277A04E0F7EE007A01E0DFEDAB
:1014A000067AB0EE670A0837BD46BDEC028B80BDF8
:1014B00000002C41920A06400000000080B52DED8E
:1014C000028B82B000AF87ED010AD7ED017AF5EE0D
:1014D000407AF1EE10FA34D0D7ED017AB7EE007A07
:1014E000F4EE477AF1EE10FA28D0D7ED017ABAEE91
:1014F000047A67EE877AF0EE670AB0EE000A6EF0C3
:1015000069FAB0EE408AD7ED017AB2EE047A67EE5E
:10151000877AB6EE087A77EEC77A9FED0E7A67EE95
:10152000877AB0EE670A6EF033F8F0EE407A68EE34
:10153000277AB7EE007A77EE877A04E0F7EE007A42
:1015400001E0DFED057AB0EE670A0837BD46BDEC75
:10155000028B80BD920A06400000000080B52DED90
:10156000028B82B000AF87ED010AD7ED017AF5EE6C
:10157000407AF1EE10FA74D0D7ED017AB7EE007A26
:10158000F4EE477AF1EE10FA68D0D7ED017AB6EEB4
:10159000007AF4EEC77AF1EE10FA2ED5D7ED017A83
:1015A000B3EE047A67EE877AB2EE047A77EEC77A02
:1015B000F0EE670AB0EE000A6EF00CFAB0EE408A68
:1015C000D7ED017AB3EE047A67EE877A9FED297A38
:1015D00077EEC77A9FED287A67EE877AB0EE670AD2
:1015E0006DF0D6FFF0EE407A68EE277AB1EE677ABA
:1015F000F0EE006AC7EE267A35E0D7ED017ABBEE51
:10160000047A67EE877AB2EE047A77EE877AF0EEA4
:10161000670AB0EE000A6EF0DDF9B0EE408AD7ED51
:10162000017AB3EE047A67EE877A9FED127A77EE4D
:10163000C77A9FED117A67EE877AB0EE670A6DF090
:10164000A7FFF0EE407A28EE277AF0EE006AC7EEA8
:10165000267AB7EE007A77EE877A04E0F7EE007A22
:1016600001E0DFED067AB0EE670A0837BD46BDEC53
:10167000028B80BD00003241C3B8B23F00000000C1
:1016800080B582B000AF87ED010AB7EE007AD7EDE2
:10169000017A77EE677AB0EE670A00F00BF8F0EEA9
:1016A000407AB7EE007A77EE677AB0EE670A0837CD
:1016B000BD4680BD80B483B000AF87ED010AD7ED91
:1016C000017A9FED377AF4EEC77AF1EE10FA0AD577
:1016D000D7ED017A9FED337A27EE877AD7ED017A3D
:1016E00067EE277A55E0D7ED017A9FED2F7AF4EE79
:1016F000C77AF1EE10FA16D5D7ED017A9FED2B7A65
:1017000077EEC77AC7ED017AD7ED017A9FED257A9A
:1017100027EE877AD7ED017A67EE277AB6EE087A58
:1017200077EE877A35E0D7ED017A9FED217AF4EEF6
:10173000C77AF1EE10FA16D5D7ED017A9FED1D7A32
:1017400077EEC77AC7ED017AD7ED017A9FED157A6A
:1017500027EE877AD7ED017A67EE277AB6EE0E7A12
:1017600077EE877A15E0D7ED017A9FED137A77EE61
:10177000C77AC7ED017AD7ED017A9FED0A7A27EE95
:10178000877AD7ED017A67EE277A9FED0C7A77EEAC
:10179000877AB0EE670A0C37BD465DF8047B704768
:1017A0008C2EBA3E0000F2408C2E3A3FE9A20B3F4D
:1017B0002FBA683F5D74513F175D743F00007C3F56
:1017C00080B582B000AF87ED010AD7ED017AB6EEA1
:1017D000007AF4EEC77AF1EE10FA16D5D7ED017A59
:1017E00077EEA77AB7EE007A77EE677AB0EE670AFF
:1017F000FFF760FFF0EE407AB7EE007A37EE677AD7
:10180000F0EE006AC7EE267A15E0D7ED017A77EEA2
:10181000A77AB7EE007A77EEC77AB0EE670AFFF7DD
:1018200049FFF0EE407AB7EE007A37EE877AF0EEB5
:10183000006AC7EE267AB0EE670A0837BD4680BD5B
:1018400080B483B000AF786039603B6818460C37CD
:10185000BD465DF8047B704780B483B000AF78600C
:101860007B6800221A707B68FF225A707B68002216
:101870005A8079684FF000024FF00003C1E902235B
:101880007B6818460C37BD465DF8047B704780B511
:1018900082B000AF7860786800F005F87B68184681
:1018A0000837BD4680BD80B582B000AF78607B68E8
:1018B0005B8803F00103002B11D07B689B685A689A
:1018C000013A5A605B68002B0CBF01230023DBB296
:1018D000002B04D07B689B68184600F005FB00BF16
:1018E0000837BD4680BD000080B483B000AF78608B
:1018F000044A7B681A607B6818460C37BD465DF861
:10190000047B704770FF080880B582B000AF786034
:101910007868FFF7E9FF0421786852F019FE7B68C8
:1019200018460837BD4680BD80B582B000AF87ED50
:10193000000B4FF00002084BD7E90001EEF7D0FC96
:1019400002460B4610461946EFF758F9034618466B
:101950000837BD4680BD00BF0000E03F000000002A
:1019600080B582B000AF87ED000B21A3D3E900233F
:10197000D7E90001EFF7E6F80346002B0BD01EA3D2
:10198000D3E90023D7E90001EEF78AFF02460B46B0
:1019900043EC172B1FE01AA3D3E90023D7E900017A
:1019A000EEF79EFC02460B461046194616A3D3E9F5
:1019B0000023EEF775FF02460B4643EC172B9FED15
:1019C0000A1BB0EE470AF0EE670A6DF00BFFB0EEAF
:1019D000407AF0EE607AB0EE470AF0EE670A083718
:1019E000BD4680BDAFF30080333333333333034020
:1019F00012143FC6DCB5A43FD7A3703D0AD72940D7
:101A0000295C8FC2F528AC3FE17A14AE47E1F03F84
:101A100080B584B000AF78607B68184600F074FA37
:101A20007B684FF000021A607B6803F580634FF01B
:101A300000021A600123FB60FB68FF2B4AD8F8689C
:101A4000EEF78AFD26A3D3E90023EEF729FF02462D
:101A50000B4643EC172BB0EE470AF0EE670AFFF790
:101A60007FFF53EC102B10461946EFF7E7F80146BD
:101A70007A68FB689B0013441960F868EEF76CFD08
:101A80004FF00002184BEEF729FC02460B461046B9
:101A9000194613A3D3E90023EEF702FF02460B46D3
:101AA00043EC172BB0EE470AF0EE670AFFF758FF3A
:101AB00053EC102B10461946EFF7C0F801467A6830
:101AC000FB6803F580739B0013441960FB680133C6
:101AD000FB60B1E77B6818461037BD4680BD00BF8C
:101AE0000000000000E06F400000E03F0000000048
:101AF00080B584B000AF78607B68184600F00FFABC
:101B00007B6800221A807B680022A3F80022012350
:101B1000FB60FB68FF2B60DCF868EEF72DFD32A35D
:101B2000D3E90023EEF7BCFE02460B4643EC172B2D
:101B3000B0EE470AF0EE670AFFF712FF51EC100B08
:101B40002BA3D3E90023EEF781FD02460B4643ECBD
:101B5000172BB0EE470AF0EE670AFFF7E5FE0346E3
:101B600099B27B68FA6823F81210F868EEF704FD62
:101B70004FF00002204BEEF7B1FB02460B46104639
:101B8000194619A3D3E90023EEF78AFE02460B4655
:101B900043EC172BB0EE470AF0EE670AFFF7E0FEC2
:101BA00051EC100B12A3D3E90023EEF74FFD0246D0
:101BB0000B4643EC172BB0EE470AF0EE670AFFF72F
:101BC000B3FE034699B27B68FA6802F5807223F887
:101BD0001210FB680133FB609BE77B6818461037E7
:101BE000BD4680BDAFF300800000000000E06F4004
:101BF00000000000E0FFEF400000E03F90B52DED59
:101C0000028B99B004AF786039607B68DA6A3B6810
